:100000000C94C51C0C94F61C0C94F61C0C94F61C59
:100010000C94F61C0C94F61C0C94F61C0C94F61C18
:100020000C94F61C0C94F61C0C94F61C0C94F61C08
:100030000C94F61C0C94F61C0C94F61C0C94F61CF8
:100040000C94F61C0C94EE640C94F61C0C94F61CA8
:100050000C94F61C0C94F61C0C9444D90C9486FA5F
:100060000C94F61C0C94FF590C94F5590C94F61C46
:100070000C94F61C0C94F61C0C94F61C0C94F61CB8
:100080000C94F61C0C94F61C0C94F61C0C94F61CA8
:100090000C94F61C0C94F61C0C94F61C0C94F61C98
:1000A0000C94F61C0C94F61C0C94F61C0C94F61C88
:1000B0000C94F61C0C94F61C0C94F61C0C94F61C78
:1000C0000C94F61C0C94F61C0C94F61C0C943D7BC2
:1000D0000C94137B0C94F61C0C94F61C0C94F61CDC
:1000E0000C94F61C901DD61DDC1D031E101E191E3F
:1000F000241E0B262B2707283228F933F9334D29E4
:10010000F0290727F933F933DA2B872DBF2DF9337F
:10011000BD2FF933F9331231F933F933A131D43129
:10012000F93350320C33CE2DD62DFA2D1E2E522EF1
:10013000F52E092F222F2F2F3C2F502F325A385AAD
:100140004A5A5A5A625A8F5A665A8F5A6A5A6E5A7D
:100150008F5A725A765A7A5A825A8F5A8C5A4EF25B
:1001600051F255F258F25BF285F25FF262F266F2FA
:1001700069F26CF270F273F276F285F27AF27DF245
:1001800080F2D0F2F2F212F337F35CF313F581F35D
:10019000A4F3C7F3ECF311F436F45BF480F413F535
:1001A000A5F4CAF4EFF4D8F5DBF5CAF5CEF5D4F52D
:1001B00012F6DFF5E3F5E9F5EDF5F1F5F7F5FBF509
:1001C000FFF512F605F609F60DF681F986F98BF9B9
:1001D00095F99FF918FAA9F9B1F9B9F9C3F9CDF967
:1001E000D7F9E6F9F0F918FAFAF904FA0EFA084A1A
:1001F000D73B3BCE016E84BCBFFDC12F3D6C74313B
:100200009ABD56833DDA3D00C77F11BED9E4BB4C91
:100210003E916BAAAABE000000803F05A84CCDB25B
:10022000D44EB93836A9020C50B9918688083CA63C
:10023000AAAA2ABE000000803F000C94325A0C94F7
:100240000C330C94DBF50C94031E0C94BF2D0C9412
:10025000D0F20C94D4F50C94101E0C94191E0C942E
:10026000ECF30C9481F90C945A5A0D94CF130C941E
:10027000825A0C940B260C94C7F30C94625A0C947B
:1002800007270C9413F50C9405F60C94F0F90C94D4
:100290008BF90C94385A0C94CAF50C94502F0C948A
:1002A0003C2F0C94BD2F0C94CE2D0C946A5A0C94B8
:1002B00066F20C9458F20C94241E0C9407280C94AB
:1002C0006CF20D94E9130C94665A0C94EE790C942C
:1002D000347A0C94B1F90C94F1F50C94D61D0C946D
:1002E0002B270C94901D0C945BF40C94F0290C9427
:1002F0007A5A0C94DFF50C948C5A0C94DA2B0C94EB
:100300004D290C94D7F90C9455F20C945CF30C9491
:1003100069F20C9480F20C94F52E0C94C3F90C94B1
:1003200012310C94FFF50C94A9F90C9432280C941A
:10033000B9F90C94872D0C94F7F50C94CAF40C942D
:10034000092F0C94817A0C944A5A0C94EFF40C9473
:1003500011F40C94DA790C946E5A0C94D8F50C9430
:10036000CEF50C940EFA0C945FF20C9476F20C9489
:10037000E6F90C94522E0C9450320C9462F20C94C8
:10038000FA2D0C9481F30C94F9330C9495F90C9498
:100390000DF60C947AF20C9470F20C942F2F0C94AE
:1003A0008F5A0C9409F60C944EF20C94CB790C9461
:1003B000F2F20C947DF20C94D62D0C94A1310C9495
:1003C000D4310C949D790C94765A0C94E9F50C94E4
:1003D00051F20C94A4F30C9437F30C94FC790C9424
:1003E000FAF90C94E3F50C94CDF90C9486F90C947D
:1003F00073F20C94EDF50C94DC1D0C94A5F40C94A4
:1004000012F30C94FBF50C949FF90C945BF20C9492
:100410001E2E0C94222F0C9404FA0C9436F40C9497
:1004200012F60C94725A0C9480F40C9418FA0C94F2
:1004300085F24E414E494E495459494E46CDCCCC99
:100440003D0AD7233C17B7D13877CC2B329595E6A8
:10045000241FB14F0A000020410000C84200401C88
:100460004620BCBE4CCA1B0E5AAEC59D7400407AD5
:1004700010F35A00A0724E18090010A5D4E800002D
:10048000E87648170000E40B54020000CA9A3B00CB
:100490000000E1F505000080969800000040420F42
:1004A000000000A08601000000102700000000E806
:1004B00003000000006400000000000A00000000CB
:1004C000000100000000002C76D888DC674F08236C
:1004D000DFC1DFAE59E1B1B796E5E3E453C63AE6D2
:1004E00051997696E8E6C28426EB898C9B62ED40B2
:1004F0007C6FFCEFBC9C9F40F2BAA56FA5F4900501
:100500005A2AF75C936B6CF9676DC11BFCE0E40D34
:1005100047FEF520E6B500D0ED902E030094357728
:10052000050080841E080000204E0A000000C80C50
:10053000333333330F986E12831141EF8D211489B9
:100540003BE65516CFFEE6DB18D1844B381BF77C13
:100550001D901DA4BBE424203284725E228100C958
:10056000F124ECA1E53D274D323520500A4D3234BF
:1005700000526573756D650055492050617573654E
:10058000004E6F204D61746368203A004D33303364
:10059000452D31533635433455004D393939004DE9
:1005A0003530320A4D353030004D3330334530531D
:1005B000323135433855000A202A2A2A726563648D
:1005C00061742E646174615B305D203D0047323898
:1005D0000A4731204631303030205A313000556ED4
:1005E000737570706F72746564204F7074696F6E8C
:1005F0002053656C6563746564004D313930533543
:10060000350A4732380A4732390A4D3430300A4DFC
:10061000313034533231350A4732380A4D313039AE
:10062000533231350A4D34323053310A4731583163
:1006300030305931303046353030300A47315A3059
:100640000A4D3530300A4D31313720536574205A08
:10065000204F666673657400473120463130303074
:10066000205A302E30004732380A47312046313088
:100670003030205A302E30004D353030005A204F67
:100680006666736574203A202573004D353030005E
:100690005A204F6666736574203A202573004732EE
:1006A000385A0A473146313530305A302E300047FB
:1006B00032380A473146313530305A302E30004D0D
:1006C000383400473146313030305A302E30004710
:1006D00032380A473146313030305A302E30005AE5
:1006E000204F6666736574203A202573004D3530BF
:1006F00030004D383400426567696E537769746322
:1007000068007265636461742E61646472203D3DAB
:10071000007265636461742E646174615B305D2096
:100720003D3D0077616974776179203D3D000A2085
:100730002A2A2A4E6F7A7A6C6554656D70537461FB
:100740007475735B325D203D00434F4D4D554E49EE
:10075000434154494F4E0044525952554E00455260
:10076000524F525300494E464F004543484F0047B1
:10077000322F47332062616420706172616D65744D
:100780006572730A00536C6565702E2E2E005A2018
:1007900050726F62652050617374204265640A0074
:1007A0005A2050726F6265205061737420426564F4
:1007B00000486F6D652058592046697273740A00AD
:1007C000486F6D65205859204669727374004D3129
:1007D00031372050726F6265206661696C65642EE6
:1007E0000A4732380A0070726F62655F7265776916
:1007F0007065004469736D69737300473239205224
:1008000065747279696E670050726F62696E6720F5
:100810004661696C6564004D313137204265642062
:100820006C6576656C696E67206661696C65642EBF
:100830000A4730205A31300A4D333030205032359B
:1008400020533838300A4D33303020503530205363
:10085000300A4D3330302050323520533838300A8A
:100860004D333030205035302053300A4D33303046
:100870002050323520533838300A4D333030205034
:1008800035302053300A47342053310070726F6284
:10089000655F6661696C6564004D31313720426582
:1008A00064206C6576656C696E6720646F6E652E7A
:1008B00000205A3A200020593A200042656420580E
:1008C0003A20004D65736820706F696E7420636113
:1008D0006E6E6F74206265207265736F6C766564EE
:1008E0000A004D302F3120427265616B2043616CEC
:1008F0006C656400436F6E74696E7565004D302FD2
:100900003120427265616B2043616C6C6564004EFE
:100910006F204D6F76652E00456E642066696C65AC
:10092000206C6973740A00426567696E2066696CA1
:1009300065206C6973740A004469736D6973730090
:10094000526573756D696E6720534400286E6F2081
:1009500066696C65290043757272656E74206669FC
:100960006C653A20002E0A0044656C6574696F6EF0
:10097000206661696C65642C2046696C653A2000CC
:1009800046696C652064656C657465643A005072F4
:10099000696E742074696D653A20000A537461743D
:1009A000733A2046696C616D656E74207573656479
:1009B0003A20002C204C6F6E67657374206A6F625A
:1009C0003A2000546F74616C2074696D653A2000A0
:1009D00053746174733A20002C204661696C65641D
:1009E0003A20002C2046696E69736865643A2000DD
:1009F0005072696E74733A200053746174733A20B4
:100A000000436F6F6C696E672E2E2E00486561740F
:100A1000696E672E2E2E0045202553006F6B006FE8
:100A20006666006A0765075E07570749074445423F
:100A300055473A004D31313320530042656420431D
:100A40006F6F6C696E672E2E2E00426564204865BC
:100A50006174696E672E2E2E004348414D42455207
:100A60005F54454D5045524154555245004D4F54E9
:100A7000494F4E5F4D4F44455300544845524D41F8
:100A80004C5F50524F54454354494F4E00415554CA
:100A90004F5245504F52545F53445F535441545545
:100AA000530050524F4D50545F535550504F525475
:100AB00000454D455247454E43595F5041525345BD
:100AC0005200434153455F4C494748545F425249A5
:100AD0004748544E45535300544F47474C455F4C8D
:100AE000494748545300534F4654574152455F506D
:100AF0004F574552004255494C445F50455243457B
:100B00004E54004C4556454C494E475F4441544174
:100B1000005A5F50524F4245004155544F4C455684
:100B2000454C005052494E545F4A4F420050524F7C
:100B30004752455353004155544F5245504F52541C
:100B40005F54454D5000564F4C554D455452494306
:100B500000454550524F4D0042494E4152595F4663
:100B6000494C455F5452414E5346455200534552FD
:100B700049414C5F584F4E5F584F464600464952D8
:100B80004D574152455F4E414D453A4D61726C693A
:100B90006E20322E305F44573420544D334420535E
:100BA000534D444E4220534F555243455F434F44AB
:100BB000455F55524C3A68747470733A2F2F6769C9
:100BC000746875622E636F6D2F496E73616E697400
:100BD000794175746F6D6174696F6E2F4D61726CC0
:100BE000696E2F747265652F437265616C697479E3
:100BF0005F4D61726C696E322E302E782050524FEC
:100C0000544F434F4C5F56455253494F4E3A312E45
:100C100030204D414348494E455F545950453A5460
:100C20004D3344203130532050726F204558545278
:100C3000554445525F434F554E543A31205555491E
:100C4000443A63656465326132662D343161322D18
:100C5000343734382D396231322D633535633632CD
:100C60006633363766660A002F2F20003F4A206F12
:100C70007574206F662072616E67652028302E3093
:100C80003120746F20302E33290A0020466C6F7794
:100C90003A200050726F7465637465642050696E09
:100CA0000A00496E76616C696420657874727564B7
:100CB00065720A0020643A0020693A0020703A0008
:100CC00020643A0020693A0020703A006469730099
:100CD000656E0043290A0061626C656420286D69B5
:100CE0006E2074656D702000436F6C6420657874AD
:100CF00072756465732061726520004F4646004F2F
:100D00004E0046696C616D656E742072756E6F750C
:100D1000742064697374616E636520286D6D293A6F
:100D2000200046696C616D656E742072756E6F751A
:100D30007420004D65736820706F696E7420636164
:100D40006E6E6F74206265207265736F6C76656479
:100D50000A004D34323120696E636F7272656374BC
:100D600020706172616D657465722075736167656D
:100D70000A004F666673657473204170706C696514
:100D800064004572723A20546F6F206661722100D0
:100D9000546F6F206661722066726F6D2072656697
:100DA0006572656E636520706F696E740A004545F3
:100DB00050524F4D204F4B0A004572726F72207790
:100DC000726974696E6720746F20454550524F4DAB
:100DD000210A00363726033C3D380E2E303E121ACB
:100DE0001C1808440AFF430809070001627573795B
:100DF0003A2070617573656420666F7220696E7049
:100E000075740A00627573793A2070617573656450
:100E100020666F7220757365720A00627573793A85
:100E20002070726F63657373696E670A0070617515
:100E30007365004D363030002066696C616D656EFB
:100E4000745F72756E6F7574200066696C616D6594
:100E50006E745F72756E6F757420540046696C61B4
:100E60006D656E7452756E6F757420540053544FD7
:100E7000505045442E20005072696E746572207384
:100E8000746F707065642064756520746F2065727E
:100E9000726F72732E2046697820746865206572BF
:100EA000726F7220616E6420757365204D39393917
:100EB00020746F20726573746172742E20285465DB
:100EC0006D706572617475726520697320726573E7
:100ED00065742E2053657420697420616674657290
:100EE0002072657374617274696E67290A004E6FAF
:100EF00020436865636B73756D2077697468206C37
:100F0000696E65206E756D6265722C204C6173741C
:100F1000204C696E653A20004E6F20436865636B14
:100F200073756D2077697468206C696E65206E75C5
:100F30006D6265722C204C617374204C696E653A49
:100F40002000636865636B73756D206D69736D61F7
:100F50007463682C204C617374204C696E653A2070
:100F6000004C696E65204E756D6265722069732054
:100F70006E6F74204C617374204C696E65204E75E1
:100F80006D6265722B312C204C617374204C696E3C
:100F9000653A20004D31313000776169740A004DA7
:100FA000313137004D333100534420726561642084
:100FB0006572726F720A00446F6E65207072696E9E
:100FC00074696E672066696C650A004B494C4C2059
:100FD00063617573656420627920746F6F206D752D
:100FE000636820696E6163746976652074696D65F4
:100FF000202D2063757272656E7420636F6D6D6154
:101000006E643A20006563686F3A004572726F72D1
:101010003A0042696C696E656172204C6576656C58
:10102000696E6720477269643A0A002020506C613B
:101030006E6E657242756666657242797465733A62
:1010400020002046726565204D656D6F72793A20EB
:1010500000436F6D70696C65643A204F6374203291
:101060003720323031390A00204C617374205570BA
:1010700064617465643A20323031392D31302D305D
:1010800035207C20417574686F723A2054696E79FE
:101090004D616368696E657333440A00322E305FB8
:1010A0004457340A004D61726C696E0020536F66BC
:1010B00074776172652052657365740A0020576108
:1010C000746368646F672052657365740A00204218
:1010D000726F776E206F75742052657365740A00A5
:1010E0002045787465726E616C2052657365740A70
:1010F00000506F77657255700A0073746172740ADC
:10110000006175746F25632E67006572726F7220BF
:1011100077726974696E6720746F2066696C650AFE
:1011200000446F6E6520736176696E672066696C36
:10113000652E0A004D323900205A3A0020593A00F3
:1011400020583A00656E6473746F70732068697418
:101150003A200047323858590024F4D43050C38E16
:1011600020C2A24017828B7011127A910D816CD926
:101170000AA861E108C7586607615143061E4B5D26
:1011800005C145A7041A411104093D98037139317D
:10119000034036DB0265339102D4305402802E1DA9
:1011A00002632CEE01752AC501B028A00110278129
:1011B000018F2564012B244B01E0223401AC211F57
:1011C000018D200D01801FFC00841EED00971DDFA6
:1011D00000B81CD200E61BC600201BBC00641AB27B
:1011E00000B219A8000A19A0006A189900D1179135
:1011F0000040178B00B516840031167E00B31579B8
:10120000003A157300C7146F0058146A00EE136695
:10121000008813630025135E00C7125B006C125731
:101220000015125400C111510070114F0021114BD3
:1012300000D61049008D10470046104400021042AD
:1012400000C00F4000800F3E00420F3C00060F3BE5
:1012500000CB0E3800930E37005C0E3500270E349D
:1012600000F30D3200C10D3100900D3000600D2EE5
:1012700000320D2D00050D2C00D90C2B00AE0C29D1
:1012800000850C29005C0C2700350C27000E0C266D
:1012900000E80B2400C40B2400A00B23007D0B23CB
:1012A000005A0B2100390B2100180B2000F80A1FEF
:1012B00000D90A1E00BB0A1E009D0A1D00800A1DDF
:1012C00000630A1C00470A1B002C0A1B00110A1AA3
:1012D00000F7091A00DD091900C4091900AB091942
:1012E00000920917007B091800630917004C0916C2
:1012F0000036091600200916000A091500F5081520
:1013000000E0081400CC081400B8081400A4081465
:1013100000900813007D0812006B08130058081293
:1013200000460812003408110023081100120811A9
:101330000001081100F0071000E0071000D00710AE
:1013400000C0071000B0070F00A107100091070EA2
:101350000083070F0074070F0065070E0057070E84
:101360000049070E003B070D002E070E0020070D59
:101370000013070D0006070D00F9060C00ED060D21
:1013800000E0060C00D4060C00C8060C00BC060CDD
:1013900000B0060C00A4060B0099060C008D060B8D
:1013A0000082060B0077060B006C060B0061060A34
:1013B0000057060B004C060A0042060A0038060ACF
:1013C000002E060A0024060A001A060A0010060962
:1013D0000007060A00FD050900F4050900EB0509F0
:1013E00000E2050900D9050900D0050900C7050973
:1013F00000BE050900B5050800AD050800A50509F2
:10140000009C050800940508008C05080084050868
:10141000007C050800740508006C050700650508D8
:10142000005D050700560508004E05070047050743
:10143000004005080038050700310507002A0507A8
:1014400000230507001C050600160507000F050709
:10145000000805060002050700FB040600F5040766
:1014600000EE040600E8040600E2040700DB0406C0
:1014700000D5040600CF040600C9040600C3040614
:1014800000BD040600B7040600B1040500AC040664
:1014900000A6040600A00405009B040600950405B0
:1014A00000900406008A04050085040500800406F7
:1014B000007A04050075040500700405006B04053E
:1014C0000066040500610405005C0405005704057E
:1014D00000520405004D04050048040500430405BE
:1014E000003E0404003A04050035040500300404FD
:1014F000002C04050027040400230405001E040436
:10150000001A04040016040500110404000D04046C
:1015100000090405000404040000040400FC0304A2
:1015200000F8030400F4030400F0030400EC0304D7
:1015300000E8030400E4030400E0030400DC030407
:1015400000D8030400D4030400D0030400CC030437
:1015500000C8030300C503030024F404D9201BC4FE
:101560000C5C0E9804C4095F0265077101F405F96B
:1015700000FB04B30048048700C103690058035509
:101580000003034500BE023A008402310053022AE0
:10159000002902250004022000E4011C00C80119F2
:1015A00000AF0117009801140084011300710110AD
:1015B000006101100051010E0043010D0036010BC6
:1015C000002B010B0020010B00150109000C010983
:1015D0000003010800FB000800F3000800EB00070F
:1015E00000E4000600DE000600D8000600D2000677
:1015F00000CC000500C7000500C2000500BD0004C6
:1016000000B9000400B5000400B1000400AD0004FE
:1016100000A9000400A5000300A20003009F00042D
:10162000009B000300980003009500020093000354
:1016300000900003008D0002008B00030088000270
:10164000008600020084000300810002007F000287
:10165000007D0002007B000200790002007700019B
:1016600000760002007400020072000100710002A6
:10167000006F0002006D0001006C0002006A0001B2
:1016800000690002006700010066000100650001BA
:1016900000640002006200010061000100600001BE
:1016A000005F0002005D0001005C0001005B0001C2
:1016B000005A0001005900010058000100570001C4
:1016C00000560001005500010054000100530000C5
:1016D00000530001005200010051000100500001C0
:1016E000004F0001004E0000004E0001004D0001BF
:1016F000004C0001004B0000004B0001004A0001BB
:1017000000490001004800000048000100470001B6
:1017100000460000004600010045000000450001B1
:1017200000440001004300000043000100420000AB
:1017300000420001004100000041000100400001A2
:10174000003F0000003F0001003E0000003E00019D
:10175000003D0000003D0001003C0000003C000096
:10176000003C0001003B0000003B0001003A00008B
:10177000003A000100390000003900010038000083
:101780000038000000380001003700000037000179
:101790000036000000360000003600010035000071
:1017A0000035000000350001003400000034000066
:1017B000003400010033000000330000003300015A
:1017C0000032000000320000003200010031000051
:1017D0000031000000310001003000000030000046
:1017E00000300001002F0000002F0000002F00003B
:1017F000002F0001002E0000002E0000002E00012E
:10180000002D0000002D0000002D0000002D000123
:10181000002C0000002C0000002C0000002C000117
:10182000002B0000002B0000002B0000002B00010B
:10183000002A0000002A0000002A0000002A0001FF
:1018400000290000002900000029000000290000F4
:1018500000290001002800000028000000280000E6
:1018600000280000002800010027000000270000D9
:1018700000270000002700000027000100260000CC
:1018800000260000002600000026000000260001BF
:1018900000250000002500000025000000250000B4
:1018A00000250000002500010024000000240000A5
:1018B0000024000000240000002400010023000098
:1018C000002300000023000000230000002300008C
:1018D000002300000023000100220000002200007D
:1018E000002200000022000000220000002200016F
:1018F0000021000000210000002100000021000064
:101900000021000000210000002100010020000053
:101910000020000000200000002000000020000047
:10192000002000000020000000200001001F000037
:10193000001F0000001F0000001F0000001F00002B
:10194000001F0000001F0001001E0000001E00001C
:10195000001E0000001E000000393000003325008A
:101960000087190000B00F0000DB080000BD040074
:1019700000740200003F010000FFFDFCFAF8F6F4DD
:10198000F2F0EEECEAE9E7E5E3E1E0DEDCDAD9D714
:10199000D5D4D2D0CFCDCBCAC8C7C5C3C2C0BFBDB6
:1019A000BCBAB9B7B6B4B3B2B0AFADACAAA9A8A629
:1019B000A5A4A2A1A09E9D9C9A9998979594939274
:1019C000908F8E8D8B8A8988878684838281807FA1
:1019D0007E7D7B7A797877767574737271706F6EAD
:1019E0006D6C6B6A696867666564636261605F5E9F
:1019F0005D5C5B5A59585857565554535251505084
:101A00004F4E4D4C4B4A4A4948474646454443424F
:101A10004241403F3E3E3D3C3B3B3A393838373609
:101A20003535343332323130302F2E2E2D2C2B2BB6
:101A30002A29292827272625252423232221212056
:101A4000201F1E1E1D1C1C1B1B1A191918181716E7
:101A500016151514131312121111100F0F0E0E0D6F
:101A60000D0C0C0B0A0A09090808070706060505EC
:101A700004040303020201000057616974696E6780
:101A800020666F72206865617475702E0A004C655F
:101A90006176696E6720473236003F53706563692F
:101AA0006669656420582C5920636F6F7264696E93
:101AB000617465206F7574206F6620626F756E6447
:101AC000732E0A003F285229657065617420766183
:101AD0006C7565206E6F7420706C61757369626CD3
:101AE000653B206D757374206265206174206C65A0
:101AF00061737420312E0A003F2852296570656198
:101B000074206D75737420626520737065636966F7
:101B1000696564207768656E206E6F7420757369DF
:101B20006E6720616E204C43442E0A003F5370655F
:101B3000636966696564206E6F7A7A6C6520746586
:101B40006D7065726174757265206E6F7420706C53
:101B500061757369626C652E0A003F537065636935
:101B6000666965642066696C616D656E7420736971
:101B70007A65206E6F7420706C61757369626C6534
:101B80002E0A003F53706563696669656420707250
:101B9000696D65206C656E677468206E6F74207067
:101BA0006C61757369626C652E0A003F5072696DD5
:101BB00065206C656E677468206D7573742062654E
:101BC00020737065636966696564207768656E2057
:101BD0006E6F74207573696E6720616E204C43448C
:101BE0002E0A003F537065636966696564206E6FF5
:101BF0007A7A6C652073697A65206E6F7420706CD8
:101C000061757369626C652E0A003F52657472617A
:101C10006374696F6E204D756C7469706C69657260
:101C2000206D7573742062652073706563696669E1
:101C300065642E0A003F53706563696669656420B8
:101C400052657472616374696F6E204D756C74694E
:101C5000706C696572206E6F7420706C6175736949
:101C6000626C652E0A003F5370656369666965643E
:101C7000206C6179657220686569676874206E6F91
:101C80007420706C61757369626C652E0A0043295B
:101C90002E0A003F5370656369666965642062655A
:101CA000642074656D7065726174757265206E6F05
:101CB0007420706C61757369626C65202834302DF6
:101CC00000473236207374617274696E672E2E2E4F
:101CD0000A0043616E6E6F74206F70656E207375BD
:101CE00062646972200053442063617264206F6BE8
:101CF0000A006F70656E526F6F74206661696C6563
:101D0000640A00766F6C756D652E696E6974206665
:101D100061696C65640A00534420696E69742066C9
:101D200061696C0A004D3234004D32332025730056
:101D300057726974696E6720746F2066696C653AC2
:101D400020002E0A006F70656E206661696C656404
:101D50002C2046696C653A20002E0A006F70656E73
:101D6000206661696C65642C2046696C653A2000C8
:101D700046696C652073656C65637465640A002050
:101D800053697A653A200046696C65206F70656E0C
:101D900065643A2000667265736800646F696E67F7
:101DA000002066696C653A20004E6F772000454E32
:101DB0004420535542524F5554494E450A00222063
:101DC000706F73002220706172656E743A22005346
:101DD0005542524F5554494E452043414C4C207476
:101DE00061726765743A2200747279696E67207453
:101DF0006F2063616C6C207375622D67636F64651F
:101E00002066696C6573207769746820746F6F2031
:101E10006D616E79206C6576656C732E204D41582E
:101E2000206C6576656C2069733A310A0053442052
:101E30007072696E74696E67206279746520004EF5
:101E40006F74205344207072696E74696E670A0063
:101E5000486F6D652025732573257320466972735D
:101E60007400220A00556E6B6E6F776E20636F6D83
:101E70006D616E643A20220020746F6F206C6F6E6B
:101E80006720657874727573696F6E2070726576FD
:101E9000656E7465640A0020636F6C6420657874F5
:101EA000727573696F6E2070726576656E746564A5
:101EB0000A007C3C3E5E2B3D3F2F5B5D3B2C2A2283
:101EC0005C0050726F62696E6720506F696E7400BB
:101ED00025532025692F2569002E0A002F005072F6
:101EE0006F62696E67206D65736820706F696E74CC
:101EF0002000202844525952554E2900473239209B
:101F00004175746F20426564204C6576656C696E1E
:101F100067003F20284C2C522C462C4229206F75FC
:101F200074206F6620626F756E64732E0A003F28FE
:101F300056296572626F7365206C6576656C2069E1
:101F40006D706C61757369626C652028302D342961
:101F50002E0A00426164205A2076616C75650A0081
:101F60004E6F2062696C696E656172206772696488
:101F70000A005374616E646172642044657669611D
:101F800074696F6E3A20002052616E67653A2000D6
:101F9000204D61783A2000204D696E3A20004D6551
:101FA000616E3A200046696E6973686564210A00B3
:101FB0002072616E67653A2000206D61783A2000DA
:101FC000206D696E3A2000207369676D613A2000C8
:101FD000206D65616E3A20003A207A3A2000206F29
:101FE000662000205900476F696E6720746F3A20A1
:101FF000580043570A00206469723A0020616E67F6
:102000006C653A005374617274207261646975730F
:102010003A00506F736974696F6E696E67207468F7
:10202000652070726F62652E2E2E0A003F4E756D10
:10203000626572206F66206C65677320696E206D23
:102040006F76656D656E74206E6F7420706C61754F
:102050007369626C652028302D3135292E0A003FC6
:102060002028582C5929206F7574206F6620626FC4
:10207000756E64732E0A003F53616D706C6520733A
:10208000697A65206E6F7420706C61757369626C1B
:10209000652028342D3530292E0A004D3438205A39
:1020A0002D50726F6265205265706561746162695E
:1020B0006C69747920546573740A003F2856296549
:1020C00072626F7365206C6576656C20696D706CEB
:1020D00061757369626C652028302D34292E0A00E1
:1020E000290A002062797465733B206372632000C3
:1020F00053657474696E67732053746F72656420DE
:102100002800454550524F4D206461746173697ACF
:1021100065206572726F722E0A00290A00206279AA
:102120007465733B2063726320002073746F726563
:10213000642073657474696E677320726574726964
:1021400065766564202800202863616C63756C6186
:1021500074656429210A0020213D20004545505224
:102160004F4D20435243206D69736D617463682045
:102170002D202873746F7265642920002053697ABA
:10218000653A2000496E6465783A2000204D6172FE
:102190006C696E3D563730290A00454550524F4D07
:1021A0002076657273696F6E206D69736D617463FB
:1021B000682028454550524F4D3D00204200205098
:1021C000006F6B00526573656E643A200043616E68
:1021D0006E6F74206F70656E207375626469722013
:1021E000002569730025696D2025697300256968DC
:1021F0002025696D2025697300256964202569689B
:102200002025696D20256973002569792025696479
:10221000202569682025696D202569730023646580
:1022200066696E652044454641554C545F00006226
:102230006564004B6420004B6920004B7020005007
:102240004944204175746F74756E652066696E69C6
:1022500073686564212050757420746865206C6112
:102260007374204B702C204B6920616E64204B648A
:1022700020636F6E7374616E74732066726F6D206D
:1022800062656C6F7720696E746F20436F6E66694C
:102290006775726174696F6E2E680A005049442038
:1022A0004175746F74756E65206661696C65642133
:1022B0002074696D656F75740A0045312054484576
:1022C000524D414C2052554E4157415900424544D0
:1022D00020544845524D414C2052554E415741598A
:1022E00000546865726D616C2052756E617761791A
:1022F0000045312048656174696E67204661696CEC
:102300006564004265642048656174696E672046B3
:1023100061696C65640048656174696E6720666117
:10232000696C656400504944204175746F74756E22
:1023300065206661696C6564212054656D70657205
:10234000617475726520746F6F20686967680A0030
:10235000204B643A2000204B693A2000204B703A11
:1023600020000A20436C6173736963205049442044
:102370000A00204B643A2000204B693A2000204B91
:10238000703A20000A204E6F206F76657273686F76
:102390006F740A002054753A2000204B753A2000D3
:1023A000206D61783A2000206D696E3A200020642B
:1023B0003A200020626961733A200050494420416C
:1023C00075746F74756E652073746172740A005051
:1023D0004944204175746F74756E65206661696C3F
:1023E0006564212054656D70657261747572652035
:1023F000746F6F20686967680A005049442041750E
:10240000746F74756E65206661696C656421204225
:102410006164206578747275646572206E756D6292
:1024200065720A002F2F616374696F6E3A006275DE
:1024300074746F6E00656E640070726F6D70745F9F
:102440000073686F77004D38373620526573706FB0
:102450006E64696E672050524F4D50545F00554E68
:102460004B4E4F574E2053544154450047434F4421
:10247000455F494E464F004C43445F5041555345DC
:102480005F524553554D450046494C414D454E54CC
:102490005F52554E4F55545F434F4E54494E55452C
:1024A0000046494C414D454E545F52554E4F555490
:1024B000004D323400436F6E74696E756500446977
:1024C0007361626C6552756E6F75740050757267DA
:1024D00065204D6F726500506175736564007061B1
:1024E0007573656400486F74656E6420746F6F2047
:1024F000636F6C640A004469736D697373005061A3
:1025000075736500507265737320627574746F6EB5
:1025100020286F72204D3130382920746F20726569
:1025200073756D650A00496E736572742066696C17
:10253000616D656E7420616E6420707265737320C6
:10254000627574746F6E20286F72204D3130382997
:102550000A00436F6E74696E756500526568656147
:102560007420446F6E6500526568656174696E67BA
:102570002E2E2E00526568656174696E670048658D
:102580006174657254696D656F7574005265686534
:1025900061740048656174657254696D656F757426
:1025A00000507265737320627574746F6E20286FAB
:1025B00072204D3130382920746F20686561742095
:1025C0006E6F7A7A6C650A004E6F7A7A6C6520506D
:1025D00061726B656400436F6E74696E7565004E61
:1025E0006F7A7A6C65205061726B656400486F7415
:1025F000656E6420746F6F20636F6C640A0072658F
:1026000073756D656400626567696E00436F6E7413
:10261000696E75650044697361626C6552756E6FB1
:1026200075740050757267654D6F72650050617505
:10263000736564004C6F61642046696C616D656E02
:102640007400436F6E74696E7565004C6F61642031
:1026500046696C616D656E74205400496E736572D5
:10266000742066696C616D656E7420616E642070A3
:102670007265737320627574746F6E20286F722098
:102680004D313038290A004469736D697373005203
:102690006573756D696E67005A5F53544F505F5094
:1026A000494E005A5F535445505F50494E005A5F9F
:1026B0004D494E5F50494E005A5F454E41424C4590
:1026C0005F50494E005A5F4449525F50494E005A8C
:1026D0005F43535F50494E00595F53544F505F5012
:1026E000494E00595F535445505F50494E00595F61
:1026F0004D494E5F50494E00595F454E41424C4551
:102700005F50494E00595F4449525F50494E00594D
:102710005F43535F50494E00585F53544F505F50D2
:10272000494E00585F535445505F50494E00585F22
:102730004D494E5F50494E00585F454E41424C4511
:102740005F50494E00585F4449525F50494E00580F
:102750005F43535F50494E0053535F50494E0053FF
:102760004552564F335F50494E00534552564F32F3
:102770005F50494E00534552564F315F50494E000D
:10278000534552564F305F50494E00534453530007
:1027900053445F4445544543545F50494E005343AE
:1027A0004B5F50494E0052414D50535F44395F508A
:1027B000494E0052414D50535F44385F50494E00DE
:1027C00052414D50535F4431305F50494E004D4FA0
:1027D00053495F50494E004D4F534645545F445F47
:1027E00050494E004D49534F5F50494E004D41589E
:1027F000363637355F53535F50494E004C45445F82
:1028000050494E004845415445525F4245445F504F
:10281000494E004845415445525F305F50494E0093
:1028200046494C5F52554E4F55545F50494E0046F5
:10283000414E315F50494E0046414E5F50494E0077
:1028400045315F535445505F50494E0045315F4517
:102850004E41424C455F50494E0045315F4449521C
:102860005F50494E0045315F43535F50494E00452C
:10287000305F535445505F50494E0045305F454EE0
:1028800041424C455F50494E0045305F4449525FDC
:1028900050494E0045305F43535F50494E00455FFD
:1028A0004D5558325F50494E00455F4D5558315F88
:1028B00050494E00455F4D5558305F50494E0042DB
:1028C00045455045525F50494E004156525F535363
:1028D0005F50494E004156525F53434B5F50494E43
:1028E000004156525F4D4F53495F50494E0041568B
:1028F000525F4D49534F5F50494E0054454D505F14
:102900004245445F50494E0054454D505F315F5041
:10291000494E0054454D505F305F50494E00464986
:102920004C57494454485F50494E00545844005253
:1029300058440020202000202020416E616C6F67E9
:1029400020696E203D2025356C64003C756E7573E2
:1029500065642F756E6B6E6F776E3E002028412583
:102960003264292020002533642000257350494E0D
:102970003A20004F7574707574203D2000496E70C8
:10298000757420203D2000416E616C6F6720696E78
:10299000203D2025356C640070726F74656374652A
:1029A000642000202841253264292020002533643A
:1029B0002000257350494E3A20002F2900012B2971
:1029C00001011E293B001329430008294500FB286B
:1029D0004400EE283201E1283301D5283401CA2809
:1029E0003501BF282501B4282801A9282A019E28DD
:1029F0002C0194282A0189281C017B2818016F28A2
:102A00001A0165282C015A2822014C281E01402851
:102A10002401382809012F28070120280201132842
:102A20000A0104280801FC270D01ED274201E427D3
:102A30003201D7270701CE273301C0270A01B32768
:102A40000801A62709019E273401902731018B2711
:102A5000350180270B01752706016A2705015F27CD
:102A60000401582735014F273501452737013827FD
:102A700026012E27030123273601182703010F27DC
:102A8000310105273D01F8263801EE260E01E32627
:102A90003C01D8260E01CF262801C5263001B826D4
:102AA0003E01AE261201A3262E0198261201446F84
:102AB0006E652E0A00534552564F206E6F74207378
:102AC00065742075702E0A004D3433205761697487
:102AD0002043616C6C656400436F6E74696E75654C
:102AE000004D343320576169742043616C6C656418
:102AF000005761746368696E672070696E730A00BD
:102B000064697300656E0061626C65640A00656EDD
:102B10006473746F70206D6F6E69746F7220002023
:102B20004500205A00205900204D393220580020FD
:102B30005A0020590020580020204D61783A20008A
:102B4000200020204D696E3A2000536F6674206586
:102B50006E6473746F70733A2000473238002049F6
:102B60006E76616C69642065787472756465722034
:102B700000205A3A0020593A0020436F756E7420A5
:102B8000583A0020453A00205A3A0020593A005855
:102B90003A0020746F6F206C6F6E672065787472D6
:102BA0007573696F6E2070726576656E7465640A00
:102BB0000020636F6C6420657874727573696F6E42
:102BC0002070726576656E7465640A00000000000E
:102BD00000000000000000000000484200004842E1
:102BE000000080405761726E696E673A20486F6DD1
:102BF000696E672042756D702044697669736F72E3
:102C0000203C20310A000202040000A0400000A085
:102C1000400000004000809D4300009B430000C82E
:102C200043FFFFFF000000010000000100008000E2
:102C3000555555000000400033333300AAAA2A003E
:102C40004992240000002000C7711C0099991900C6
:102C5000D1451700555515003BB11300244912000A
:102C600011111100000010000F0F0F00E3380E00CB
:102C700043790D00CCCC0C00C3300C00E8A20B0053
:102C800064210B00AAAA0A00703D0A009DD8090021
:102C9000427B090092240900DCD3080088880800E0
:102CA0001042080000000800F0C1070087870700F5
:102CB00075500700711C07003EEB0600A1BC060022
:102CC0006990060066660600703E06006118060000
:102CD00017F4050074D105005BB00500B290050043
:102CE000627205005555050078390500B81E0500CB
:102CF000050505004EEC040087D40400A1BD0400C6
:102D000090A7040049920400C17D0400EE6904000C
:102D1000C7560400444404005C3204000821040047
:102D200041100400000004003FF00300F8E003003D
:102D300026D20300C3C30300CCB503003AA80300A6
:102D40000A9B0300388E0300C08103009F750300B7
:102D5000D0690300505E03001D5303003448030094
:102D6000913D03003333030016290300381F03008D
:102D700097150300300C0300030303000BFA020055
:102D800049F10200BAE802005CE002002DD802001E
:102D90002DD0020059C80200B0C0020031B90200B3
:102DA000DAB10200AAAA0200A0A30200BC9C0200A1
:102DB000FA9502005C8F0200DF8802008282020026
:102DC000457C02002776020027700200436A020059
:102DD0007C640200D05E02003F590200C85302002A
:102DE00070012C0190012701B0012201C0011D01D9
:102DF000F00118011002130130020E0160020901F6
:102E000090020401C002FF000003FA004003F50035
:102E10008003F000D003EB002004E6007004E10022
:102E2000E004DC004005D700C005D2004006CD001C
:102E3000D006C8008007C3003008BE00F008B90003
:102E4000C009B400B00AAF00B00BAA00D00CA500B6
:102E5000000EA000500F9B00C01096005012910071
:102E600000148C00C0158700B0178200B0197D00D7
:102E7000D01B7800001E730040206E009022690075
:102E8000F024640040275F0090295A00E02B550091
:102E9000102E500020304B0010324600E03341002D
:102EA00090353C001037370070383200A0392D00C3
:102EB000B03A2800A03B2300603C1E00103D1900E2
:102EC000903D1400103E0F00703E0A00C03E050009
:102ED000003F0000403FFBFF803FF6FFC03FF1FF97
:102EE000202D20496E76616C696420657874727556
:102EF000646572206E756D62657220210A00100093
:102F0000C90210012C014001220170011801B00119
:102F10000E01F00104015002FA00B002F00030038B
:102F2000E600D003DC009004D2007005C800A006C3
:102F3000BE000008B400B009AA00D00BA000600ECB
:102F4000960060118C000015820020197800C01DC9
:102F50006E00A0226400B0275A00902C500000316F
:102F60004600E0343C0010383200903A2800603CC3
:102F70001E00A03D1400803E0A00203F00004531A5
:102F800020544845524D414C2052554E41574159CD
:102F90000042454420544845524D414C2052554E24
:102FA0004157415900546865726D616C2052756ECD
:102FB00061776179004531204572723A204D415860
:102FC00054454D50004572723A204D415854454D7C
:102FD0005020424544004D415854454D5020747294
:102FE00069676765726564004531204572723A20F1
:102FF0004D494E54454D50004572723A204D494E50
:1030000054454D5020424544004D494E54454D5085
:1030100020747269676765726564000A0A0020207F
:103020005A5F4D494E3A002020595F4D494E3A00B3
:103030002020585F4D494E3A004D383420582059D1
:10304000205A204500202F002042403A0020403ADC
:103050000020573A0020573A00496E76616C696447
:103060002065787472756465720A00446966663A10
:10307000200046726F6D5374703A0053746570701F
:1030800065723A00556E4C6576656C3A004C657613
:10309000656C65643A005261773A20202020000A6E
:1030A0004C6F676963616C3A004361703A0042613A
:1030B000627973746570205A0050726F6265204F98
:1030C0006666736574205A0050726F6265204F66A1
:1030D000667365745A3A2000290A0020746F200034
:1030E0003F5A206F7574206F662072616E6765208D
:1030F0002800290A0020746F20003F59206F757442
:10310000206F662072616E676520282D00290A00F5
:1031100020746F20003F58206F7574206F662072F6
:10312000616E676520282D00205A002059005072DA
:103130006F6265204F6666736574205800220A002E
:10314000656E7175657565696E672022000A206974
:103150006E6974207A70726F62655F7A6F666673EB
:103160006574203D2000454550524F4D20496E6901
:103170007469616C697A65640A0048617264636F9E
:103180006465642044656661756C7420536574746D
:10319000696E6773204C6F616465640A000000FA11
:1031A000430000FA430000204100008C420000A0D0
:1031B000420000A0420000C84300000C43EE0200A1
:1031C00000EE020000640000003C0000003A0A002B
:1031D00020204D363033200020440020204D343153
:1031E0003220530046696C616D656E742072756E95
:1031F0006F75742073656E736F723A0A0020550004
:103200004C0046696C616D656E74206C6F61642F53
:10321000756E6C6F6164206C656E677468733A0AD2
:1032200000205A0020590020204D38353120580008
:103230005A2D50726F6265204F6666736574002068
:10324000440020490020204D3330342050002044D9
:103250000020490020204D33303120500050494497
:103260002073657474696E67733A0A00205A0020EF
:103270004A0020204732392057204900205A002098
:10328000204D3432302053004175746F2042656404
:10329000204C6576656C696E673A0A00205A0020FA
:1032A000590020204D323036205800486F6D65207F
:1032B0006F66667365743A0A00204A002054002045
:1032C000530020204D323035204200204A3C6A75A0
:1032D0006E635F6465763E00416476616E6365642B
:1032E0003A20423C6D696E5F7365676D656E745F11
:1032F00074696D655F75733E20533C6D696E5F66E2
:10330000656564726174653E20543C6D696E5F74DE
:10331000726176656C5F66656564726174653E00B6
:1033200020540020520020204D32303420500041E3
:103330006363656C65726174696F6E2028756E6970
:1033400074732F7332293A20503C7072696E745F27
:10335000616363656C3E20523C7265747261637494
:103360005F616363656C3E20543C74726176656C8A
:103370005F616363656C3E0A00204500205A0020AF
:10338000590020204D3230312058004D6178696D50
:10339000756D20416363656C65726174696F6E2041
:1033A00028756E6974732F7332293A0A002045001C
:1033B000205A0020590020204D3230332058004D33
:1033C0006178696D756D2066656564726174657399
:1033D0002028756E6974732F73293A0A0053746537
:1033E00070732070657220756E69743A0A0020202F
:1033F0004D3230302044300A0020204D3230302011
:1034000044002044697361626C65640A0046696C1B
:10341000616D656E742073657474696E67733A00CC
:1034200020286D6D29002020473231202020203BAC
:1034300020556E69747320696E206D6D00486F6D44
:10344000696E67204661696C6564006F70656E0027
:10345000545249474745524544003A200066696C3A
:10346000616D656E74007A5F6D696E00795F6D697C
:103470006E00785F6D696E005265706F7274696E70
:103480006720656E6473746F7020737461747573F4
:103490000A002E0A006F70656E206661696C6564B3
:1034A0002C2046696C653A2000706F7765726F66F4
:1034B00066004B494C4C45442E20005072696E7496
:1034C00065722068616C7465642E206B696C6C2871
:1034D000292063616C6C6564210A0020540020522D
:1034E00000416363656C65726174696F6E3A205068
:1034F0000050574D3A20202534640050574D3A2053
:10350000202534640050574D3A2020253464005063
:10351000574D3A20202534640050574D3A2020253D
:1035200034640050574D3A20202534640050574DE4
:103530003A20202534640050574D3A202025346429
:103540000050574D3A20202534640050574D3A2002
:10355000202534640050574D3A2020253464005013
:10356000574D3A20202534640050574D3A202025ED
:1035700034640050574D3A20202534640050574D94
:103580003A20202534640050574D3A2020253464D9
:10359000003A200020202020434F4D002020206EA4
:1035A0006F6E2D7374616E646172642050574D208C
:1035B0006D6F646500202020636F6D7061726520FF
:1035C000696E7465727275707420656E61626C6587
:1035D00064002020206F766572666C6F7720696EBC
:1035E0007465727275707420656E61626C656400DA
:1035F0003A20002020202054494D534B00423A20CD
:1036000000202020205443435200413A2000202033
:10361000202054434352002020202043533A2000CE
:103620002020202057474D3A200050574D3A202067
:103630002534640050574D3A20202534640047005B
:103640004800000088008A008C00B300B40000002D
:1036500098009A009C00A800AA00AC0028012A014A
:103660002C012020202054494D45520044004500A3
:103670006E00800081006F00B000B100700090000B
:1036800091007100A000A1007200200121017300CF
:1036900020697320616C736F207469656420746F96
:1036A00020746869732070696E0054494D45523129
:1036B00043000A202E002020002020506F72743A10
:1036C000200000002100240027002A002D003000E7
:1036D000330001010000040107010A01000022007B
:1036E000250028002B002E003100340002010000CC
:1036F000050108010B01000020002300260029001D
:103700002C002F0032000001000003010601090116
:1037100005050505070508080808020202020A0A4D
:10372000080804040404010101010101010103036B
:10373000030303030303040707070C0C0C0C0C0C16
:103740000C0C0202020206060606060606060B0B13
:103750000B0B0B0B0B0B0102102020080810204054
:103760001020408002010201080402010102040845
:1037700010204080804020100804020180040201D3
:10378000804020100804020108040201010204081C
:1037900010204080010204081020408000000A0B25
:1037A00002090C0D0E0807030401000000000000D0
:1037B0000000000000000000000000000000000009
:1037C00000000000000000001211100000000000C6
:1037D00000000000000000000000000000000000E9
:1037E000000050726F62696E67204661696C6564A3
:1037F0000A0050726F62696E67204661696C656489
:1038000000205A3A200020593A200042656420588E
:103810003A2000544D3344203130532050726F20F1
:1038200052656164792E005072696E74696E672EFC
:103830002E2E005072696E7420506175736564009D
:1038400063616E63656C005072696E742041626FD3
:1038500072746564004469736D697373005549201F
:1038600041626F7274656400726573756D65004DB9
:1038700032340000809D4300009B430000C8430099
:103880000000000000000000000000626564002CE1
:103890002073797374656D2073746F707065642123
:1038A000204865617465725F49443A20004265644E
:1038B0002048656174696E67204661696C656400C3
:1038C00048656174696E67206661696C6564004271
:1038D000454420544845524D414C2052554E415785
:1038E000415900546865726D616C2052756E617744
:1038F00061790045312048656174696E67204661D1
:10390000696C65640048656174696E672066616909
:103910006C656400453120544845524D414C20525D
:10392000554E4157415900546865726D616C205283
:10393000756E61776179004F46460A00466164659D
:10394000204865696768742000426564204C65768C
:10395000656C696E6720004661696C656420746FF0
:1039600020656E61626C6520426564204C657665F9
:103970006C696E670A00496E76616C6964206D65DA
:1039800073682E0A00006101350111241FBECFEFBC
:10399000D1E2DEBFCDBF00E00CBF17E0A0E0B2E097
:1039A000E8E9F9E402E00BBF02C007900D92AE3BDC
:1039B000B107D9F72DE1AEEBB7E001C01D92A233FC
:1039C000B207E1F71CE1C4ECDCE100E006C021979E
:1039D0000109802FFE010F94F520C33CD10780E040
:1039E0000807A9F70F94210B0D94BA240C9400003A
:1039F0002F923F924F925F926F927F928F929F92FF
:103A0000AF92BF92CF92DF92EF92FF920F931F93EC
:103A1000CF93DF93CDB7DEB7A7970FB6F894DEBF8D
:103A20000FBECDBF80910901817091E09827209150
:103A3000DD07921781F19093DD07811116C00E9476
:103A40001A7C8091791683FF09C087E993E00E9470
:103A5000F75261E080E00E9498FE1DC060E081E0C6
:103A60000E9498FE80EB93E014C00091791603FB4E
:103A7000002700F90E94A97B80917916877F8093A7
:103A80007916002341F060E081E00E9498FE89EC05
:103A900093E00E94F7528091DC0781110C946C38FE
:103AA0008091DA079091DB079C012F5F3F4F3093A5
:103AB000DB072093DA07883E934010F40C946C38AF
:103AC00081E08093DC071092DB071092DA07809187
:103AD000AA0A882309F48CC30E9482AD811188C38D
:103AE0008091D9078F5F8093D9078091D907853658
:103AF00020F01092D9071092AA0AE091AA0A8E2FFC
:103B0000EE0F990BAA0BBB0BFC013197E730F105C7
:103B100008F0A0C08827EE58FF4F8F4F0D94F52076
:103B20000E947AAD882309F495C081E08093260233
:103B30008CED93E00E94F75280E190E09093FE14A8
:103B40008093FD1485E08093F11402E80093F4144F
:103B500084E190E1A0E0B0E08093F5149093F61436
:103B6000A093F714B093F8140E9419ED81E09AE540
:103B70009093FE148093FD1486E390E090930015DB
:103B80008093FF1487E08093F1140093F41484E889
:103B900090E0A0E0B0E08093F5149093F614A09329
:103BA000F714B093F8140E9419ED52C00E947AAD38
:103BB000882309F44FC048C08AEE93E00E94F75270
:103BC00081E09AE59093FE148093FD1480E490E0E8
:103BD000909300158093FF1407E00093F11482E89E
:103BE0008093F41484E890E0A0E0B0E08093F514B2
:103BF0009093F614A093F714B093F8140E9419ED63
:103C00000093AA0A27C08091D807882319F10E943F
:103C10007AAD8823F9F00E9482AD81111BC0EBC2FE
:103C20000E947AAD8823B1F00E9482AD811112C04A
:103C300010C30E9482AD81110DC042E060E070E0CF
:103C4000CB010E9498AD04C00E9482AD811102C0D8
:103C50001092AA0A80912602882309F4B1C28091A9
:103C6000A60A9091A70A892B09F08FC18091D507E8
:103C70009091D607892B09F01EC184E096E09093BD
:103C8000FE148093FD1480EA90E8909300158093D1
:103C9000FF1417E01093F11402E80093F41480EA83
:103CA00090E0A0E0B0E08093F5149093F614A09318
:103CB000F714B093F8140E9419ED809106029091C8
:103CC0000702A0910802B09109020097A105B10571
:103CD00011F51092FE141092FD1415E01093F114DA
:103CE0000093F4148AE890E1A0E0B0E08093F5142A
:103CF0009093F614A093F714B093F8140E9419ED62
:103D000089E090E09093FE148093FD141093F114D9
:103D10000093F41440C00196A11DB11D65E0B69555
:103D2000A795979587956A95D1F70197A109B1094C
:103D3000009721E0A207B10558F0B093FE14A093BC
:103D4000FD14909300158093FF141093F11407C095
:103D50009093FE148093FD1485E08093F11412E893
:103D60001093F4148AE890E1A0E0B0E08093F51499
:103D70009093F614A093F714B093F8140E9419EDE1
:103D800088E090E09093FE148093FD1485E080938A
:103D9000F1141093F4148CE890E1A0E0B0E080936B
:103DA000F5149093F614A093F714B093F8140E94AE
:103DB00019ED8091060290910702A0910802B0913E
:103DC0000902009731E0A307B10550F0B093FE144B
:103DD000A093FD14909300158093FF1487E005C015
:103DE0009093FE148093FD1485E08093F11482E893
:103DF0008093F41488E890E1A0E0B0E08093F5149B
:103E00009093F614A093F714B093F8140E9419ED50
:103E10008091060290910702A0910802B0910902D8
:103E2000BA2FA92F982F88270097E1E0AE07B10598
:103E300050F0B093FE14A093FD149093001580935E
:103E4000FF1487E005C09093FE148093FD1485E075
:103E50008093F11412E81093F41481EA90E0A0E04A
:103E6000B0E08093F5149093F614A093F714B093F8
:103E7000F8140E9419ED80915617882319F082E0FA
:103E800090E002C083E090E09093FE148093FD14D4
:103E900085E08093F1141093F41485E490E1A0E0A0
:103EA000B0E08093F5149093F614A093F714B093B8
:103EB000F8140E9419ED0091D5071091D607053628
:103EC00011057CF41093FE140093FD1485E080939B
:103ED000F11482E88093F41480E090E1A0E0B0E077
:103EE00011C0C801845691099093FE148093FD146B
:103EF00085E08093F11482E88093F41481E090E1EE
:103F0000A0E0B0E08093F5149093F614A093F7141A
:103F1000B093F8140E9419ED0F5F1F4F1093D6074E
:103F20000093D507093C110564F188EF93E00E94E6
:103F3000F75281E090E09093A70A8093A60A8093BD
:103F4000260281E09AE59093FE148093FD148DE2A1
:103F500090E0909300158093FF1487E08093F11414
:103F600082E88093F41484E890E0A0E0B0E08093CD
:103F7000F5149093F614A093F714B093F8140E94DC
:103F800019ED1092DC070C946C3880915F149091BD
:103F90006014891B8F7009F0DAC10E9450508111A2
:103FA000D6C18091791682FDD2C17DC184E690E0B0
:103FB0009093FE148093FD141093F1140093F41465
:103FC0008EE090E1A0E0B0E08093F5149093F614B9
:103FD000A093F714B093F8140E9419EDC601825310
:103FE0009048880F991F9093FE148093FD141093AE
:103FF000F1140093F4148FE090E1A0E0B0E080931E
:10400000F5149093F614A093F714B093F8140E944B
:1040100019ED0E9469FD90E09093FE148093FD14C9
:1040200085E08093F11482E88093F41486E190E1B6
:10403000A0E0B0E08093F5149093F614A093F714E9
:10404000B093F8140E9419ED20E030E048EC52E4FF
:104050006091EE167091EF168091F0169091F11626
:104060000F947A1A0F946A227093FE146093FD14D1
:1040700015E01093F11402E80093F41486E290E145
:10408000A0E0B0E08093F5149093F614A093F71499
:10409000B093F8140E9419ED20E030E0A90160917E
:1040A000850B7091860B8091870B9091880B0F94F4
:1040B000FE200F946A227093FE146093FD141093F7
:1040C000F1140093F41486E390E1A0E0B0E0809353
:1040D000F5149093F614A093F714B093F8140E947B
:1040E00019ED6091900870919108809192089091DB
:1040F00093080F946A227093FE146093FD1410933A
:10410000F1140093F4148CE390E1A0E0B0E080930C
:10411000F5149093F614A093F714B093F8140E943A
:1041200019ED8091890B90918A0B9093FE148093E6
:10413000FD141093F1140093F41484E390E1A0E0D3
:10414000B0E08093F5149093F614A093F714B09315
:10415000F8140E9419ED809194089091950890931D
:10416000FE148093FD141093F1140093F4148AE369
:1041700090E1A0E0B0E08093F5149093F614A09342
:10418000F714B093F8140E9419ED0091D1070111B2
:104190007FC18091D30781117BC18091D8078111A4
:1041A0003CC28091A5149091A614A091A714B0913F
:1041B000A8148C34F0E19F07A105B10509F052C2A3
:1041C00081E4C82E85E1D82E0AE18BE493E10E94B8
:1041D000FC79E090C607F090C707181619060CF096
:1041E0009DC31AE1E116F10414F40C940C3496C347
:1041F0001092D9077ACC8AEA95E00E94F752809112
:10420000D70790E0A0E0B0E0895B9F4FAE4FB54A82
:1042100021E03AE53093FE142093FD1490930015AD
:104220008093FF1487E08093F11482E88093F41464
:1042300084E890E0A0E0B0E08093F5149093F61449
:10424000A093F714B093F8140E9419ED1092D807B8
:10425000FFCC81E0809326021092AA0A88EB95E0B9
:104260000E94F75281E09AE59093FE148093FD142A
:104270008EE490E0909300158093FF1487E0809384
:10428000F11482E88093F41484E890E0A0E0B0E0B8
:104290008093F5149093F614A093F714B093F81448
:1042A0000E9419EDD7CC00919008109191082091AF
:1042B00092083091930808A319A32AA33BA3609105
:1042C000940870919508072E000C880B990B0F9499
:1042D0001B1A6B017C0120E030E040E050E40F94B9
:1042E000FD2028A139A14AA15BA10F945E231816D5
:1042F0000CF433C220E030E0A9016091850B70918D
:10430000860B8091870B9091880B0F94FE206CA3F5
:104310007DA38EA39FA36091890B70918A0B072EBA
:10432000000C880B990B0F941B1A4B015C0120E0C9
:1043300030E040E251E40F94FD202CA13DA14EA1BC
:104340005FA10F945E2318160CF407C226C28CE0FE
:1043500090E09093FE148093FD1405E00093F11417
:1043600082E88093F41484E190E1A0E0B0E08093CF
:10437000F5149093F614A093F714B093F8140E94D8
:1043800019ED0E9496FB20E13EE040E050E00F94E2
:104390006A202115310511E04107510560F0509365
:1043A000FE144093FD14309300152093FF1487E012
:1043B0008093F11406C03093FE142093FD140093F3
:1043C000F11402E80093F41480E190E1A0E0B0E081
:1043D0008093F5149093F614A093F714B093F81407
:1043E0000E9419ED0E9496FB20E13EE040E050E083
:1043F0000F946A202CE330E040E050E00F946A20F4
:104400003093FE142093FD1415E01093F1140093E3
:10441000F41482E190E1A0E0B0E08093F514909371
:10442000F614A093F714B093F8140E9419ED0E94AB
:1044300069FD882391F00E9469FD8F5F8093D40706
:10444000C82ED12C833308F0B1CDC601880F991F37
:104450009093FE148093FD1404C01092FE141092E9
:10446000FD141093F1140093F4148EE090E1A0E099
:10447000B0E08093F5149093F614A093F714B093E2
:10448000F8140E9419ED1092FE141092FD14AFCD95
:1044900020E030E0A9016091850B7091860B80913E
:1044A000870B9091880B0F94FE2020E030E048ECC1
:1044B00052E40F947A1A6B017C016091890B709120
:1044C0008A0B072E000C880B990B0F941B1A9B016B
:1044D000AC01C701B6010F94F8210F947122643624
:1044E000710510F064E670E07093FE146093FD14A3
:1044F00095E0A92EA092F11422E8B22EB092F41405
:1045000084E290E1A0E0B0E08093F5149093F6147B
:10451000A093F714B093F8140E9419ED20E030E056
:10452000A9016091850B7091860B8091870B90910A
:10453000880B0F94FE206B017C0120E030E04AE202
:1045400053E40F945E2318160CF069C1002309F49C
:1045500066C11092D10720E030E040E251E4609162
:10456000C9077091CA078091CB079091CC070F942F
:104570007A1A0F946A227093FE146093FD14A0922D
:10458000F114B092F41484E590E1A0E0B0E08093DF
:10459000F5149093F614A093F714B093F8140E94B6
:1045A00019ED20E030E040E251E46091CD077091D8
:1045B000CE078091CF079091D0070F947A1A0F946D
:1045C0006A227093FE146093FD14A092F114B092CD
:1045D000F41488E590E1A0E0B0E08093F5149093A6
:1045E000F614A093F714B093F8140E9419ED86EC1A
:1045F00095E00E94F75281E09AE59093FE14809333
:10460000FD1481E490E0909300158093FF1487E0FF
:104610008093F114B092F41451C18091C80701E065
:10462000080F0093C80790E09093FE148093FD1448
:1046300085E08093F11482E88093F41482E490E1A1
:10464000A0E0B0E08093F5149093F614A093F714D3
:10465000B093F8140E9419ED0A3008F4A2CD10921C
:10466000C8079FCD8A349041A105B10509F4A8CDB2
:1046700020E030E040E251E460913E1770913F1736
:1046800080914017909141170F947A1A0F946A22E3
:104690007093FE146093FD1415E01093F11402E87A
:1046A0000093F41488E490E1A0E0B0E08093F51466
:1046B0009093F614A093F714B093F8140E9419ED98
:1046C00020E030E040E251E46091421770914317DE
:1046D00080914417909145170F947A1A0F946A228B
:1046E0007093FE146093FD141093F1140093F4146E
:1046F0008AE490E1A0E0B0E08093F5149093F61482
:10470000A093F714B093F8140E9419ED20E030E064
:1047100040E251E460914617709147178091481725
:10472000909149170F947A1A0F946A227093FE148D
:104730006093FD141093F1140093F4148CE490E151
:10474000A0E0B0E08093F5149093F614A093F714D2
:10475000B093F8140E9419ED33CD8DE090E0909362
:10476000FE148093FD1485E08093F11482E8809319
:10477000F41484E190E1A0E0B0E08093F51490930C
:10478000F614A093F714B093F8140E9419ED8091D9
:10479000A90A811141C081E03FC020E030E040E043
:1047A00050E4C701B6010F94FE2028A139A14AA107
:1047B0005BA10F94141A87FD10C020E030E040E2A6
:1047C00051E4C501B4010F94FE202CA13DA14EA1DE
:1047D0005FA10F94141A87FF37CC84E190E0909387
:1047E000FE148093FD1485E08093F11482E8809399
:1047F000F41484E190E1A0E0B0E08093F51490938C
:10480000F614A093F714B093F8140E9419ED809158
:10481000A90A811101C082E08093A90A15CC609198
:10482000890B70918A0B072E000C880B990B0F9443
:104830001B1A9B01AC01C701B6010F945E23609166
:10484000D30787FD4AC0662309F4A7CC062E000CC7
:10485000770B8EE297E00E94D7511092D307109207
:10486000D6071092D50784E090E09093FE148093D1
:10487000FD1485E08093F11402E80093F4148EE8AF
:1048800090E1A0E0B0E08093F5149093F614A0932B
:10489000F714B093F8140E9419ED81E09AE5909313
:1048A000FE148093FD1483E590E0909300158093AF
:1048B000FF1487E08093F1140093F41484E890E0EF
:1048C000A0E0B0E08093F5149093F614A093F71451
:1048D000B093F8140E9419ED60CC662309F45DCC06
:1048E0008091D5079091D6079C012F5F3F4F309361
:1048F000D6072093D50765E070E00F94E1209093F0
:10490000FE148093FD1485E08093F11482E8809377
:10491000F4148EE890E1A0E0B0E0D4CF1E141F04A0
:104920000CF02FCB9091A21480914115981322C0C6
:104930009091A3148091421598131CC003E0E016D7
:10494000F104C4F0909143159093A1148091441503
:104950008093A4149330D1F4982F9D7F9038B1F4B4
:10496000909145159F3409F05FC0909146159B3496
:1049700009F05AC08AE1E1E4F5E1DF011D928A9570
:10498000E9F71092C7071092C607FBCA833809F0EF
:104990004BC08091451590914615982789279827F7
:1049A000A0E0B0E08093A5149093A614A093A71460
:1049B000B093A8144091471550E060E070E0409338
:1049C000A9145093AA146093AB147093AC1408E428
:1049D000A02E05E1B02E80E090E0DC018417950761
:1049E000A607B70708F04EC06C017D01F694E79466
:1049F000D794C79496012A5F3F4F220F331FF901C6
:104A0000EF55FB4E7F01F501208130E0322F222748
:104A10000181202BF701318320830296A11DB11D56
:104A2000F2E0AF0EB11CDACF813861F58091451507
:104A300090E0A0E0B0E08093A5149093A614A0931A
:104A4000A714B093A81480914615482F50E060E059
:104A500070E04093A9145093AA146093AB14709320
:104A6000AC14A7E4B5E1EDEAF4E190E020E030E039
:104A70002817390739F04D9150E0419351932F5F3A
:104A80003F4FF6CF8AE1E1E4F5E1DF011D928A951F
:104A9000E9F71092C7071092C60789E094E00E94D8
:104AA000F7526091AA0A161664F4062E000C770BD2
:104AB00083E297E00E94D7518AE00E94A0500C94B4
:104AC000FD336091AD147091AE1481E197E00E94C6
:104AD000AE518AE00E94A0504091A5145091A614B6
:104AE0006091A7147091A81482E097E00E949D51F4
:104AF0008AE00E94A0508091A5149091A614A091E4
:104B0000A714B091A814E5E7F2E000E010E04191AD
:104B10005191619171914115510561057105D1F175
:104B2000481759076A077B0791F5AC01BD0148504A
:104B3000504161097109453051056105710568F100
:104B4000AC01BD01477F423350416105710541F120
:104B50008433F0E19F07A105B10511F1AC01BD015E
:104B6000465450416109710947305105610571058D
:104B7000D0F0AC01BD014455504161097109453087
:104B800051056105710588F402E110E00EC00F5F68
:104B90001F4FBDCF0FEF1FEF08C003E010E005C0AF
:104BA00008E010E002C00FE010E08A509042A10936
:104BB000B109833D9105A105B10530F00F3F2FEFFD
:104BC000120721F40C94FD3309E110E0AAE2CA2E89
:104BD000A4E0DA2EF60181916F01882319F00E947A
:104BE000A050F8CFB801012E000C880B990B0E9441
:104BF000BB510E94F15286EF96E00E94F7520A31B3
:104C0000110510F00C94F933F8018827E758FF4F8D
:104C10008F4F0D94F5208091AD149091AE1481309A
:104C20009105E1F4109226028FEF8093B51960E0B0
:104C300080E00E9498FE08E314E0D8018D918D0178
:104C4000882319F00E94A050F8CF81E09AE5909354
:104C5000FE148093FD148EE290E0AFC08230910587
:104C600009F0C5C081E0809326020E94DAFD82EF40
:104C700096E09093CA088093C9088BE090E09093E7
:104C8000FE148093FD1405E00093F11412E81093D4
:104C9000F41480E092E1A0E0B0E08093F5149093EA
:104CA000F614A093F714B093F8140E9419ED109223
:104CB000FE141092FD140093F1141093F4148EE07E
:104CC00090E1A0E0B0E08093F5149093F614A093E7
:104CD000F714B093F8140E9419ED1092FE1410927C
:104CE000FD140093F1141093F4148FE090E1A0E010
:104CF000B0E08093F5149093F614A093F714B0935A
:104D0000F8140E9419ED1092FE141092FD140093F5
:104D1000F1141093F41486E190E1A0E0B0E08093E8
:104D2000F5149093F614A093F714B093F8140E941E
:104D300019ED62E070E080E090E00E945CAE1092BD
:104D4000FE141092FD140093F1141093F41480E1FA
:104D500090E1A0E0B0E08093F5149093F614A09356
:104D6000F714B093F8140E9419ED1092FE141092EB
:104D7000FD140093F1141093F41482E190E1A0E08B
:104D8000B0E08093F5149093F614A093F714B093C9
:104D9000F8140E9419ED02E614E0F80181918F01E8
:104DA000882319F00E94A050F8CF81E09AE59093F3
:104DB000FE148093FD148DE290E090930015809393
:104DC000FF1487E08093F11482E88093F41484E860
:104DD00090E0A0E0B0E08093F5149093F614A093D7
:104DE000F714B093F8140E9419ED0C94FD3383303E
:104DF000910549F581E0809326020CE814E0D80182
:104E00008D918D018823C9F00E94A050F8CF809128
:104E1000A5149091A614A091A714B091A814823360
:104E200030E19307A105B10509F077C48091AD1475
:104E30009091AE14009709F035C480910502882343
:104E400009F405C315C3049711F00C94FD331092B7
:104E500026020C94FD338091AD149091AE148130F4
:104E60009105D1F41092260280910502882319F051
:104E700082E090E002C083E090E09093FE14809383
:104E8000FD1485E08093F11482E88093F4148EE1A0
:104E900090E1A0E0B0E09FCF8230910519F506EBDC
:104EA00014E0F80181918F01882319F00E94A0502D
:104EB000F8CF81E0809326028091A90A843049F0DE
:104EC00081E09AE59093FE148093FD1485E390E0D1
:104ED00074CF81E09AE59093FE148093FD1486E3ED
:104EE00090E06BCF8330910509F04CC02091050212
:104EF000222319F19093FE148093FD1485E0809392
:104F0000F11482E88093F4148EE190E1A0E0B0E027
:104F10008093F5149093F614A093F714B093F814BB
:104F20000E9419ED40E060E070E088EC92E40E949D
:104F300049FE109205020C94FD3382E090E09093BC
:104F4000FE148093FD1485E08093F11482E8809331
:104F5000F4148EE190E1A0E0B0E08093F51490931A
:104F6000F614A093F714B093F8140E9419ED40E0E2
:104F700060E070E0CB010E9449FE81E08093050271
:104F80000C94FD33049711F00C94FD338091A30829
:104F90008823F1F082E090E09093FE148093FD145A
:104FA00085E08093F11482E88093F4148FE190E11E
:104FB000A0E0B0E08093F5149093F614A093F7145A
:104FC000B093F8140E9419ED1092A3080C94FD33CD
:104FD00083E090E09093FE148093FD1485E080932D
:104FE000F11482E88093F4148FE190E1A0E0B0E046
:104FF0008093F5149093F614A093F714B093F814DB
:105000000E9419ED81E08093A3080C94FD33009178
:10501000AD141091AE14B80180E090E00F94191A0D
:105020006B017C0120E030E040E251E40F94141A5F
:1050300087FD0DC020E030E04AEF53E4C701B60120
:105040000F945E23181634F0902F812F05C09AE03C
:1050500080E002C094EF81E0909354028093550267
:105060000C94FD338091A5149091A614A091A714DF
:10507000B091A8148830F0E19F07A105B10509F0AF
:1050800050C081E09AE59093FE148093FD148DE268
:1050900090E0909300158093FF1487E08093F114C3
:1050A00012E81093F41484E890E0A0E0B0E080935C
:1050B000F5149093F614A093F714B093F8140E948B
:1050C00019ED1092FE141092FD1405E00093F114F6
:1050D0001093F41480E190E1A0E0B0E08093F51427
:1050E0009093F614A093F714B093F8140E9419ED5E
:1050F0001092FE141092FD140093F1141093F41406
:1051000082E190E1A0E0B0E08093F5149093F61472
:10511000A093F714B093F8140E9419ED0E94DAFDE1
:105120008FC08A3000E19007A105B105E1F58091BB
:10513000AD149091AE14813F910511F00C94FD33A4
:1051400081E09AE59093FE148093FD1486E390E04D
:10515000909300158093FF1487E08093F11482E808
:105160008093F41484E890E0A0E0B0E08093F5141C
:105170009093F614A093F714B093F8140E9419EDCD
:1051800041E755E068E775E084E00E9456BA60E0C8
:1051900083E398E30E949BFD87E695E09093CA081D
:1051A0008093C9084DC08C309041A105B10509F02C
:1051B00047C08091AD149091AE14019709F040C0A2
:1051C0000F94D0141092A90A81E0809326028CE0FB
:1051D00090E09093FE148093FD1485E08093F11489
:1051E00012E81093F41484E190E1A0E0B0E0809321
:1051F000F5149093F614A093F714B093F8140E944A
:1052000019ED81E09AE59093FE148093FD1485E3F7
:1052100090E0909300158093FF1487E08093F11441
:105220001093F41484E890E0A0E0B0E08093F514CB
:105230009093F614A093F714B093F8140E9419ED0C
:105240008091A5149091A614A091A714B091A814D0
:105250008C309041A105B10511F00C94FD33809183
:10526000AD149091AE14029711F00C94FD330F948D
:10527000D01481E08093D3071092A90A809326026C
:105280001092D6071092D50781E09AE59093FE140C
:105290008093FD1482E590E090CD2091AD14309183
:1052A000AE14B90180E090E037FF09C00F94191ADD
:1052B00020E030E040E857E40F94FD2002C00F9456
:1052C000191A20E030E048EC52E40F94F8216B0109
:1052D0007C0120E030E040EA51EC0F945E2387FD32
:1052E00031C020E030E040EA51E4C701B6010F943C
:1052F000141A18163CF1A70196016091EE167091F0
:10530000EF168091F0169091F1160F94FD2020E099
:1053100030E048EC53E40F947A1A90580F946A22C4
:10532000CB010E9477F0C092EE16D092EF16E09279
:10533000F016F092F1168DEE96E09093CA088093E5
:10534000C90828C020E030E048EC52E46091EE1635
:105350007091EF168091F0169091F1160F947A1AD1
:105360000F946A227093FE146093FD1485E080937D
:10537000F11482E88093F41486E290E1A0E0B0E0BA
:105380008093F5149093F614A093F714B093F81447
:105390000E9419ED6091EE167091EF168091F01653
:1053A0009091F1168E010B5E1F4F23E041E00F94A8
:1053B000EC149F938F938FED96E09F938F930451FE
:1053C00011091F930F930F94AC19C8010E9436AFB7
:1053D0000F900F900F900F900F900F900C94FD3343
:1053E0008091AD149091AE14009729F481E08093E0
:1053F00026020C94FD3381309105B1F480910502B1
:10540000882349F081E09AE59093FE148093FD147F
:105410008CE390E0D2CC81E09AE59093FE148093E7
:10542000FD148BE390E0C9CC82309105F9F2833012
:10543000910539F58091050240E0882389F060E00C
:1054400070E088EC92E40E9449FE1092050281E02F
:105450009AE59093FE148093FD1489E390E0ADCC1F
:1054600060E070E0CB010E9449FE81E0809305027C
:1054700081E09AE59093FE148093FD148AE390E016
:105480009CCC8530910599F50E948EFE84EB90E0CE
:105490000E94E4DB10928E1210928F1210929012E2
:1054A00010929112109292120E943BDB86E490E0DF
:1054B0000E94D86E84EB90E09093FE148093FD14CC
:1054C00005E00093F11412E81093F41484E390E1E2
:1054D000A0E0B0E08093F5149093F614A093F71435
:1054E000B093F8140E9419ED86E490E035C0863040
:1054F0009105D9F50E948EFE80EF90E00E94E4DBDA
:1055000010928E1210928F1210929012109291128D
:10551000109292120E943BDB8EE690E00E94D86EC1
:1055200080EF90E09093FE148093FD1405E00093CB
:10553000F11412E81093F41484E390E1A0E0B0E0D9
:105540008093F5149093F614A093F714B093F81485
:105550000E9419ED8EE690E09093FE148093FD1466
:105560000093F1141093F414D3C0813F910511F00E
:105570000C94FD3340E060E070E0CB010E9449FEF6
:1055800041E060E070E0CB010E9449FE109205020C
:105590000E948EFE80E090E00E94E4DB10928E126A
:1055A00010928F12109290121092911210929212E9
:1055B0000E943BDB80E090E00E94D86E1092FE14C7
:1055C0001092FD1405E00093F11412E81093F41406
:1055D00084E390E1A0E0B0E08093F5149093F6149A
:1055E000A093F714B093F8140E9419ED61E070E0F5
:1055F00080E090E00E945CAE1092FE141092FD14C8
:105600000093F1141093F4148AE390E1A0E0B0E069
:105610008093F5149093F614A093F714B093F814B4
:105620000E9419ED61E070E080E090E00E945CAEC5
:1056300084E190E09093FE148093FD140093F114A4
:105640001093F41484E190E1A0E0B0E08093F514AD
:105650009093F614A093F714B093F8140E9419EDE8
:1056600081E09AE59093FE148093FD1489E390E025
:10567000909300158093FF1487E08093F1141093AA
:10568000F41484E890E0A0E0B0E08093F5149093E7
:10569000F614A093F714B093F8140E9419ED82E069
:1056A0000C94F63381309105A9F40E948EFE80E0BF
:1056B00090E00E94E4DB1092FE141092FD1485E04D
:1056C0008093F11482E88093F41484E390E1A0E0E5
:1056D000B0E081CB029711F00C94FD3310928E1242
:1056E00010928F12109290121092911210929212A8
:1056F0000E943BDB80E090E00E94D86E1092FE1486
:105700001092FD1485E08093F11482E88093F414E4
:105710008AE390E1A0E0B0E05ECB8433E0E19E0755
:10572000A105B105D9F40091AD141091AE140E94F9
:105730008EFEB80180E090E00F94191A20E030E06E
:1057400046E953E40F945E23181614F0C80102C012
:105750008CE291E00E94E4DB0C94FD338A339041AB
:10576000A105B10511F00C94FD330091AD14109119
:10577000AE1410928E1210928F12109290121092FC
:105780009112109292120E943BDBB80180E090E0EF
:105790000F94191A20E030E04CE053E40F945E239C
:1057A000181614F0C80102C08CE890E00E94D86E70
:1057B0000C94FD338091AD149091AE14009709F4D0
:1057C00015CE8130910509F04CC080915617882381
:1057D00019F083E090E002C082E090E09093FE1424
:1057E0008093FD1485E08093F11482E88093F41493
:1057F00085E490E1A0E0B0E08093F5149093F61476
:10580000A093F714B093F8140E9419ED8AE090E089
:105810009093FE148093FD1485E08093F11482E848
:105820008093F41480E092E1A0E0B0E08093F5145E
:105830009093F614A093F714B093F8140E9419ED06
:105840000E947AAD811103C08FEC96E002C083EC18
:1058500096E09093CA088093C90882E08093AA0AD0
:1058600085C18230910509F0ADC081E080932602A8
:1058700088E0E9ECF7E0DF011D928A95E9F780E026
:1058800090E0A0E2B1E48093C9079093CA07A09387
:10589000CB07B093CC078093CD079093CE07A0930E
:1058A000CF07B093D00784E690E09093FE148093E6
:1058B000FD1405E00093F11412E81093F41484E54C
:1058C00090E1A0E0B0E08093F5149093F614A093DB
:1058D000F714B093F8140E9419ED20E030E040E294
:1058E00051E46091CD077091CE078091CF079091E0
:1058F000D0070F947A1A0F946A227093FE14609363
:10590000FD140093F1141093F41488E590E1A0E0E5
:10591000B0E08093F5149093F614A093F714B0932D
:10592000F8140E9419ED20E030E0A9016091850B88
:105930007091860B8091870B9091880B0F94FE20BD
:105940000F946A227093FE146093FD140093F11477
:105950001093F41486E390E1A0E0B0E08093F51496
:105960009093F614A093F714B093F8140E9419EDD5
:105970008091890B90918A0B9093FE148093FD1473
:105980000093F1141093F41484E390E1A0E0B0E0EC
:105990008093F5149093F614A093F714B093F81431
:1059A0000E9419ED62E070E080E090E00E945CAE41
:1059B00081E09AE59093FE148093FD1481E490E0D9
:1059C0000C9439358330910509F085C01092D707C2
:1059D00020E030E040E251E460913E1770913F17C3
:1059E00080914017909141170F947A1A0F946A2270
:1059F0007093FE146093FD1405E00093F11412E817
:105A00001093F41488E490E1A0E0B0E08093F514E2
:105A10009093F614A093F714B093F8140E9419ED24
:105A200020E030E040E251E460914217709143176A
:105A300080914417909145170F947A1A0F946A2217
:105A40007093FE146093FD140093F1141093F414FA
:105A50008AE490E1A0E0B0E08093F5149093F6140E
:105A6000A093F714B093F8140E9419ED20E030E0F1
:105A700040E251E4609146177091471780914817B2
:105A8000909149170F947A1A0F946A227093FE141A
:105A90006093FD140093F1141093F4148CE490E1DE
:105AA000A0E0B0E08093F5149093F614A093F7145F
:105AB000B093F8140E9419ED62E070E080E090E08D
:105AC0000E945CAE81E09AE59093FE148093FD14F1
:105AD00087E490E0CEC78430910509F48EC6853006
:105AE000910549F44EE750E160E070E08DED94E0FF
:105AF0000E94D7ED82C6069709F07FC68FEB96E02D
:105B00009093CA088093C9088BE090E02BC28091E3
:105B1000AD149091AE14019711F51092260281E018
:105B20009AE59093FE148093FD148FE390E0909398
:105B300000158093FF1487E08093F11482E880932E
:105B4000F41484E890E0A0E0B0E08093F514909322
:105B5000F614A093F714B093F8140E9419ED8091F5
:105B6000AD149091AE14029709F047C681E09AE512
:105B70009093FE148093FD1480E490E01EC9E091A0
:105B8000AD14F091AE143197EB30F10508F0E4C19B
:105B90008827ED56FF4F8F4F0D94F52080914913C4
:105BA00080FF65C6869580FD65C661C62DEC3CEC20
:105BB0004CEC5DE36091EE167091EF168091F0165B
:105BC0009091F1160F94FE206B017C0120E030E0F3
:105BD00040EA51EC0F945E2387FDC2C120E030E023
:105BE00040EA51E4C701B6010F94141A18160CF0DC
:105BF00048C6B6C12DEC3CEC4CEC5DE36091EE1672
:105C00007091EF168091F0169091F1160F94FD208F
:105C10006B017C0120E030E040EA51EC0F945E2300
:105C200087FD9EC120E030E040EA51E4C701B601A3
:105C30000F94141A18160CF09BC692C180E00E94B3
:105C400060BF0E947AAD811103C086E696E002C073
:105C500088E596E09093CA088093C90882E0809313
:105C6000AA0A81E09AE59093FE148093FD1484E5DE
:105C700090E0909300158093FF1487E08093F114D7
:105C800082E88093F41484E890E0A0E0B0E0809390
:105C9000F5149093F614A093F714B093F8140E949F
:105CA00019ED5EC183E08093AA0A83E090E09093AF
:105CB000FE148093FD1485E08093F11482E88093B4
:105CC000F4148DE890E1A0E0B0E08093F514909397
:105CD000F614A093F714B093F8140E9419EDE12C78
:105CE000F12C00E0DD24D394AA24A39475E0972E30
:105CF000E5E08E2EF2E87F2EDD2031F0CC24C39437
:105D000065E0B62E10E005C0CC24CA94BB24BA943A
:105D100014E0DA24B116D1F1802F90E04897A4F571
:105D20000F5FF701919EE00DF11D1124EE0FFF1F93
:105D3000EE0FFF1FE452FD4E20E030E04AE754E44E
:105D400060817181828193810F947A1A0F946A2203
:105D50007093FE146093FD148092F1147092F41409
:105D6000802F90E08158974F880F991F092E000CC3
:105D7000AA0BBB0B8093F5149093F614A093F71421
:105D8000B093F8140E9419ED1C0DC4CFBFEFEB1AAD
:105D9000FB0AE5E0EE16F10409F0AECF81E09AE5EA
:105DA0009093FE148093FD1485E590E09093001588
:105DB0008093FF1487E08093F11482E88093F414B9
:105DC00084E890E0A0E0B0E08093F5149093F6149E
:105DD000A093F714B093F8140E9419ED8AEF95E0A0
:105DE0009093CA088093C908BBC042E060E070E0AD
:105DF00080E890E40E9498AD40E060E070E08DE1C2
:105E000093E40E9498AD41E060E070E08BE193E4A0
:105E100013C042E060E070E080E890E40E9498AD3A
:105E200040E060E070E080EB91E40E9498AD41E0DA
:105E300060E070E080EB91E40E9498AD86E0809392
:105E4000AA0A8EC042E060E070E080E890E40E9420
:105E500098AD40E060E070E882E993E4E6CF42E08C
:105E600060E070E080E890E40E9498AD40E060E07F
:105E700070E882E993E40CC042E060E070E080E802
:105E800090E40E9498AD40E060E070E080EB91E427
:105E90000E9498AD41E060E070E080E993E4CCCFEF
:105EA0008091561781111CC083E090E09093FE14FE
:105EB0008093FD1485E08093F11482E88093F414BC
:105EC00085E490E1A0E0B0E08093F5149093F6149F
:105ED000A093F714B093F8140E9419ED81E01BC051
:105EE00082E090E09093FE148093FD1485E080930F
:105EF000F11482E88093F41485E490E1A0E0B0E02E
:105F00008093F5149093F614A093F714B093F814BB
:105F10000E9419ED80E00E9460BF20E030E048EC74
:105F200052E46091EE167091EF168091F016909108
:105F3000F1160F947A1A0F946A227093FE146093EC
:105F4000FD1485E08093F11482E88093F41486E2D6
:105F500090E1A0E0B0E09BCE8EED95E00E94F7527C
:105F60008AE090E09093FE148093FD1485E0809386
:105F7000F11482E88093F4144FC184E08093AA0A5C
:105F80008091A5149091A614A091A714B091A81483
:105F90006091AD147091AE148834F0E19F07A105B3
:105FA000B10509F453C08A3400E19007A105B10599
:105FB00009F455C08C3410E19107A105B10509F42D
:105FC00057C086349041A105B10509F059C063302E
:105FD0007105B9F58DEC95E09093CA088093C908D6
:105FE00081E08093D807809326021092C80781E051
:105FF0009AE59093FE148093FD148AE490E09093C8
:1060000000158093FF1487E08093F11412E8109339
:10601000F41484E890E0A0E0B0E08093F51490934D
:10602000F614A093F714B093F8140E9419ED8AE0C7
:1060300090E09093FE148093FD1485E08093F1141A
:10604000E9C06093D7071092AA0AD7C3412C30E861
:10605000532E3DE9632E33E4732E312C11C0412CB5
:10606000512C2BE9622E23E4722E3324339408C082
:10607000412C512C88EC682E83E4782E92E0392E46
:1060800080E090E00F94191A20E030E040E251E403
:106090000F94F8216B017C0120E030E0A9010F94FE
:1060A000141A87FF09C01092C2071092C3071092FA
:1060B000C4071092C50719C0A3019201C701B60118
:1060C0000F945E2318164CF0C092C207D092C307FB
:1060D000E092C407F092C50708C04092C2075092F0
:1060E000C3076092C4077092C5076091C2077091A0
:1060F000C3078091C4079091C507432D0E9498ADB6
:1061000061E070E080E090E00E945CAE20E030E072
:1061100040E251E460913E1770913F178091401723
:10612000909141170F947A1A0F946A227093FE147B
:106130006093FD1405E00093F11412E81093F41439
:1061400088E490E1A0E0B0E08093F5149093F61419
:10615000A093F714B093F8140E9419ED20E030E0FA
:1061600040E251E4609142177091431780914417C7
:10617000909145170F947A1A0F946A227093FE1427
:106180006093FD140093F1141093F4148AE490E1E9
:10619000A0E0B0E08093F5149093F614A093F71468
:1061A000B093F8140E9419ED20E030E040E251E491
:1061B0006091461770914717809148179091491741
:1061C0000F947A1A0F946A227093FE146093FD1450
:1061D0000093F1141093F4148CE490E1A0E0B0E08B
:1061E0008093F5149093F614A093F714B093F814D9
:1061F0000E9419ED61E070E080E090E00E945CAEEA
:106200001092AA0A8AE090E09093FE148093FD1405
:106210000093F1141093F41480E092E1A0E0B0E058
:106220000C94EB268091A5149091A614A091A7142C
:10623000B091A814863530E19307A105B10509F0A6
:1062400046C020E030E0A9016091850B7091860B7B
:106250008091870B9091880B0F94FE2020E030E016
:106260004AE253E40F94141A2091AD143091AE1405
:1062700087FF0AC42530310508F006C48AEA90E099
:106280009093FE148093FD1485E08093F11412E83E
:106290001093F41480E290E1A0E0B0E08093F51454
:1062A0009093F614A093F714B093F8140E9419ED8C
:1062B00065E070E080E090E00E945CAE81E09AE5ED
:1062C0009093FE148093FD1482E490E0D2C3843551
:1062D000E0E19E07A105B105B9F46091AD1470919C
:1062E000AE1480E090E00F94191A20E030E040E214
:1062F00051E40F94F8216093C9077093CA07809303
:10630000CB079093CC0779C288359041A105B105A0
:1063100009F073C26091AD147091AE1480E090E00A
:106320000F94191A20E030E040E251E40F94F82174
:106330006093CD077093CE078093CF079093D007DB
:106340005CC26091AD147091AE1487EB95E00E9431
:10635000AE518091AD149091AE1482309105A1F0B0
:1063600038F4009771F00197E1F486E095E043C2BC
:106370008430910579F058F0059799F48CE895E010
:106380000BC080EF94E037C289EA95E005C08FE941
:1063900095E002C08AE995E09093CA088093C90805
:1063A0002CC28AE195E027C289E295E00E94F7526B
:1063B0008091AD149091AE148130910519F46499D7
:1063C000E4C41BC2892B09F018C287E395E00E9440
:1063D000F7528091BE07813039F58DE495E00E9437
:1063E000F75281E09AE59093FE148093FD148EE2BB
:1063F00090E0909300158093FF1487E08093F11450
:1064000082E88093F41484E890E0A0E0B0E0809308
:10641000F5149093F614A093F714B093F8140E9417
:1064200019ED1092A80A35C0823069F481E695E032
:106430000E94F75281E09AE59093FE148093FD1438
:1064400086E390E00EC0833031F585E795E00E9449
:10645000F75281E09AE59093FE148093FD1481E455
:1064600090E0909300158093FF1487E08093F114DF
:1064700082E88093F41484E890E0A0E0B0E0809398
:10648000F5149093F614A093F714B093F8140E94A7
:1064900019ED10923C171092BE070E94DAFDADC1B3
:1064A0008091AD149091AE148F3F910531F028F09A
:1064B0008FEF90E0A0E0B0E002C0A0E0B0E08093F9
:1064C000060290930702A0930802B09309028091FC
:1064D000060290910702A0910802B091090200976C
:1064E000A105B10509F51092FE141092FD1405E006
:1064F0000093F11412E81093F4148AE890E1A0E0FC
:10650000B0E08093F5149093F614A093F714B09331
:10651000F8140E9419ED89E090E09093FE148093A6
:10652000FD140093F1143DC00196A11DB11D05E0BD
:10653000B695A795979587950A95D1F70197A109E3
:10654000B109009701E0A007B10550F0B093FE1427
:10655000A093FD14909300158093FF1487E005C06D
:106560009093FE148093FD1485E08093F11412E85B
:106570001093F4148AE890E1A0E0B0E08093F51461
:106580009093F614A093F714B093F8140E9419EDA9
:1065900088E090E09093FE148093FD1485E0809352
:1065A000F1141093F4148CE890E1A0E0B0E0809333
:1065B000F5149093F614A093F714B093F8140E9476
:1065C00019ED8091060290910702A0910802B09106
:1065D0000902BA2FA92F982F8827009711E0A10749
:1065E000B10550F0B093FE14A093FD1490930015E4
:1065F0008093FF1487E005C09093FE148093FD14F0
:1066000085E08093F11482E88093F41481EA90E0AD
:10661000A0E0B0E00C94EB2689E895E00E94F752E8
:106620000E946EAD4091A5145091A6146091A714DC
:106630007091A814882339F0433D20E25207610588
:10664000710509F4E8C3423D50426105710509F046
:10665000D4C08091AD149091AE14019709F033C568
:106660000E946EAD882309F42EC58091B51987FD6F
:10667000C4C0A2E18A02C00111248059944E0E9434
:10668000C27BC12C90E2D92EE12CF12C05E012E85E
:106690001092FE141092FD140093F1141093F41450
:1066A000C092F514D092F614E092F714F092F81418
:1066B0000E9419EDBFEFCB1ADB0AEB0AFB0AEAE0F6
:1066C000CE16E0E2DE06E104F10411F70091B519FF
:1066D000F2E10F0280011124085F154EF8010190CC
:1066E0000020E9F7C8018E1B9F0B439697FD01968A
:1066F0007C01F594E7941E141F040CF0DEC49E0187
:106700002F5F3F4F690184E1D9011D928A95E9F716
:10671000A7016AE975E0C9010F947124B801C601A7
:106720008E0D9F1D0F945C2440E050E260E070E00D
:10673000C6010E94D7ED62E070E080E090E00E9428
:106740005CAE40E060E070E08FE793E40E9449FEB9
:1067500041E060E070E08FE793E40E9449FE109210
:1067600005028DE090E09093FE148093FD1485E087
:106770008093F11412E81093F41484E190E1A0E006
:10678000B0E08093F5149093F614A093F714B093AF
:10679000F8140E9419ED62E070E080E090E00E9441
:1067A0005CAE81E09AE59093FE148093FD1485E33E
:1067B00090E0909300158093FF1487E08093F1148C
:1067C0001093F41484E890E0A0E0B0E08093F51416
:1067D0009093F614A093F714B093F8140E9419ED57
:1067E00081E0809326028093A80A83E08093A90A1F
:1067F00004C081E895E00E94F75280E5E1EAF4E107
:10680000DF011D928A95E9F78AE58093A21485EA53
:106810008093A3140C94C11F8BE493E10E94DA7956
:10682000F701EF5BFA4E8083809141158A3581F044
:106830001E141F0414F00C94E520D601E02F1D92C5
:10684000EA95E9F71092C7071092C6070C94E52065
:1068500062E070E080E090E00E945CAEFFEFEF1A33
:10686000FF0AF092C707E092C6070C94E5208FEA72
:1068700096E002C08EE996E09093CA088093C9081A
:106880004CCB88E290E00E9477F02DEC3CEC4CEC95
:106890005DE36091EE167091EF168091F016909185
:1068A000F1160F94FE206B017C0120E030E040EAFD
:1068B00051EC0F945E2387FD12C020E030E040EAE7
:1068C00051E4C701B6010F94141A181644F0C0928F
:1068D000EE16D092EF16E092F016F092F11620E04C
:1068E00030E048EC52E46091EE167091EF16809122
:1068F000F0169091F1160F947A1A0F946A22709301
:10690000FE146093FD1485E08093F11482E8809377
:10691000F41486E290E1A0E0B0E08093F514909347
:10692000F614A093F714B093F8140E9419ED609137
:10693000EE167091EF168091F0169091F1168E017F
:106940000B5E1F4F23E041E00F94EC149F938F9355
:1069500080E996E09F938F93045111091F930F9341
:106960000F94AC19C8010E9436AF8BE896E076C050
:1069700088ED9FEF0E9477F02DEC3CEC4CEC5DE352
:106980006091EE167091EF168091F0169091F116CD
:106990000F94FD206B017C0120E030E040EA51ECD7
:1069A0000F945E2387FD12C020E030E040EA51E4FE
:1069B000C701B6010F94141A181644F0C092EE16CF
:1069C000D092EF16E092F016F092F11620E030E04F
:1069D00048EC52E46091EE167091EF168091F0163B
:1069E0009091F1160F947A1A0F946A227093FE1404
:1069F0006093FD1485E08093F11482E88093F41491
:106A000086E290E1A0E0B0E08093F5149093F61454
:106A1000A093F714B093F8140E9419ED6091EE164C
:106A20007091EF168091F0169091F1168E010B5E29
:106A30001F4F23E041E00F94EC149F938F938DE759
:106A400096E09F938F93045111091F930F930F9416
:106A5000AC19C8010E9436AF88E796E09093CA0847
:106A60008093C9080F900F900F900F900F900F9088
:106A700077CA909300158093FF1487E08093F114F8
:106A80001093F4140C94E7262430310539F5209145
:106A90004A1730914B1740914C1750914D17609108
:106AA000CD077091CE078091CF079091D0070F94BA
:106AB000FE2060934A1770934B1780934C17909366
:106AC0004D1780E090E0A0E8BFE389839A83AB8311
:106AD000BC83CE0101960E9413D0BBC02530310586
:106AE00008F4FDC02630310509F43CC108F02EC180
:106AF00081E08093D1070E948EFE8EEB90E00E9491
:106B0000E4DB20E030E0A9016091850B7091860BF9
:106B10008091870B9091880B0F94FE2020E030E04D
:106B200048EC52E40F947A1A6B017C016091890B56
:106B300070918A0B072E000C880B990B0F941B1A6F
:106B40009B01AC01C701B6010F94F8210F9471228B
:106B50006436710510F064E670E07093FE14609383
:106B6000FD1405E00093F11412E81093F41484E28C
:106B700090E1A0E0B0E08093F5149093F614A09318
:106B8000F714B093F8140E9419ED20E030E0A90149
:106B90006091850B7091860B8091870B9091880B8B
:106BA0000F94FE200F946A227093FE146093FD14DC
:106BB0000093F1141093F41486E390E1A0E0B0E0A8
:106BC0008093F5149093F614A093F714B093F814EF
:106BD0000E9419ED8091890B90918A0B9093FE147D
:106BE0008093FD140093F1141093F41484E390E166
:106BF000A0E0B0E08093F5149093F614A093F714FE
:106C0000B093F8140E9419ED65E070E080E090E028
:106C10000E945CAE81E09AE59093FE148093FD148F
:106C200084E490E0909300158093FF1487E08093B4
:106C3000F1141093F41484E890E0A0E0B0E08093A5
:106C4000F5149093F614A093F714B093F8140E94DF
:106C500019ED20E030E040E251E46091C907709105
:106C6000CA078091CB079091CC070F947A1A0F94A2
:106C70006A227093FE146093FD1405E00093F114F2
:106C800012E81093F41484E590E1A0E0B0E0809362
:106C9000F5149093F614A093F714B093F8140E948F
:106CA00019ED20E030E040E251E46091CD077091B1
:106CB000CE078091CF079091D0070F947A1A0F9446
:106CC0006A227093FE146093FD140093F1141093E4
:106CD000F41488E590E1A0E0B0E00C94EB262230BB
:106CE000310589F420914A1730914B1740914C1788
:106CF00050914D176091C9077091CA078091CB07D9
:106D00009091CC07D4CE2330310598F02091CD0757
:106D10003091CE074091CF075091D00760914A172C
:106D200070914B1780914C1790914D170F94FD2047
:106D3000C0CE2130310509F08CCF2091C9073091A8
:106D4000CA074091CB075091CC07E8CF213F3105CE
:106D500009F07FCF1092D10761E070E080E090E011
:106D60000E945CAE81E09AE59093FE148093FD143E
:106D700081E490E0909300158093FF1487E0809366
:106D8000F11482E88093F41456CF87EE95E00E94C8
:106D9000F75281E00E943FB98DE090E09093FE149D
:106DA0008093FD1485E08093F11412E81093F4149D
:106DB00084E190E1A0E0B0E08093F5149093F614A4
:106DC000A093F714B093F8140E9419ED83E0809318
:106DD000A90A81E09AE59093FE148093FD1485E35F
:106DE00090E0909300158093FF1487E08093F11456
:106DF0001093F41484E890E0A0E0B0E08093F514E0
:106E00009093F614A093F714B093F8140E9419ED20
:106E10001092BE07F2CC8FEF95E00E94F75280915E
:106E2000B6199091B71999272091AD143091AE14ED
:106E30008217930708F4E1CC82E995E00E94F752AB
:106E40008091AD1481508093B519A4ED8A2EA0E2F3
:106E50009A2EA12CB12C05E012E81092FE1410928B
:106E6000FD140093F1141093F4148092F514909291
:106E7000F614A092F714B092F8140E9419ED3FEFA7
:106E8000831A930AA30AB30A8EED881680E2980645
:106E9000A104B10411F78091B519A2E18A02C001E1
:106EA0001124FC01E85FF54E7F0101900020E9F715
:106EB000C7018E1B9F0B439697FD01968C0115957C
:106EC000079510161106FCF49E012F5F3F4F6901D4
:106ED00084E1D9011D928A95E9F7A8016AE975E074
:106EE000C9010F947124B701C601800F911F0F943F
:106EF0005C2444ED50E260E070E0C6010E94D7EDF2
:106F000005E012E806C044ED50E260E070E0C70121
:106F1000F5CF1092FE141092FD140093F11410930B
:106F2000F4148092F5149092F614A092F714B09293
:106F3000F8140E9419EDBFEF8B1A9B0AAB0ABB0A2B
:106F4000E6EE8E16E0E29E06A104B10411F78E0172
:106F50000F5F1F4F84E1D8011D928A95E9F7809158
:106F6000B7198F938091B6198F938091AE148F9338
:106F70008091AD148F9384EA95E09F938F931F9334
:106F80000F930F948B244EED50E260E070E0C80147
:106F90000E94D7ED62E070E080E090E00E945CAE7D
:106FA0000FB6F894DEBF0FBECDBF31E2C32E32E183
:106FB000D32EE12CF12C43E1442E40E6542E612CDB
:106FC000712C88248394912CAA24AA94BA2C75E05D
:106FD000272EE2E83E2E0AE010E08091B61990914B
:106FE000B7198815990594F1B092FE14A092FD147A
:106FF0002092F1143092F4144092F5145092F61449
:107000006092F7147092F8140E9419ED1093FE1418
:107010000093FD142092F1143092F414C092F514F0
:10702000D092F614E092F714F092F8140E9419ED41
:10703000FFEF8F1A9F0A20E1420E511C611C711C48
:107040003FEFC31AD30AE30AF30AC7CF8091AD1406
:107050009091AE1424E0880F991F2A95E1F78D5F77
:107060009F49A0E0B0E020EF37E83093FE14209372
:10707000FD1405E00093F11412E81093F4148093CA
:10708000F5149093F614A093F714B093F8140E949B
:1070900019ED8091AD149091AE14805E9D4EA0E0EC
:1070A000B0E026E030E03093FE142093FD1400930E
:1070B000F1141093F4140C94EB2640E050E260E0DD
:1070C00070E0C80136CB8091AD149091AE14892B3D
:1070D00011F40C94F62991CBA7960FB6F894DEBF65
:1070E0000FBECDBFDF91CF911F910F91FF90EF9019
:1070F000DF90CF90BF90AF909F908F907F906F90D8
:107100005F904F903F902F9008952F923F924F9213
:107110005F926F927F928F929F92AF92BF92CF9227
:10712000DF92EF92FF920F931F93CF93DF93CDB730
:10713000DEB7C154D1090FB6F894DEBF0FBECDBF84
:1071400022968FAF22972091EE072CAF81E080939B
:10715000EE078091C6128D3409F4B4C3843511F45E
:107160000C942449873411F00C942B498091C4125B
:107170009091C5128B31910509F427C1B4F4843084
:10718000910534F482309105E4F597FF2EC096C343
:107190008531910511F40C942D498A31910509F43A
:1071A00010C1049709F08AC3CDC08A32910509F451
:1071B000ADC24CF48D319105B1F00CF420C14E9765
:1071C00009F45CC17BC38B35910509F41CC28C3575
:1071D000910509F41DC28A35910509F06FC310921B
:1071E000ED070C942D4914E036C180916F0288237D
:1071F00011F40C942D490E9435C20E949FCC0C942E
:107200002D4920916F02222311F40C942D4911E095
:10721000029709F010E00E9435C219821A821B827F
:107220001C821D821E821F82188682E50E94D6B8AB
:10723000882309F457C00E9456B86B017C0120E0F6
:1072400030E0A9010F94141A882309F461C08091D9
:107250003E1790913F17A0914017B091411788A712
:1072600099A7AAA7BBA78091421790914317A09115
:107270004417B09145178CA79DA7AEA7BFA78091D3
:10728000C8169091C916A091CA16B091CB1688ABBA
:1072900099ABAAABBBAB8091CC169091CD16A091C7
:1072A000CE16B091CF168CAB9DABAEABBFAB28A9C1
:1072B00039A94AA95BA968A579A58AA59BA50F94B8
:1072C000141A81110C9438492CA93DA94EA95FA923
:1072D0006CA57DA58EA59FA50F94141A8823C1F0D7
:1072E0000C94384989E40E94D6B8882331F00E9472
:1072F00056B869837A838B839C838AE40E94D6B8CC
:10730000882331F00E9456B86D837E838F839887DF
:1073100020E030E0A90169817A818B819C810F9402
:10732000141A81110C943D4A20E030E0A9016D81CE
:107330007E818F8198850F94141A81110C943D4A97
:107340000C94504A80E50E94D6B8882329F00E9408
:10735000ADF56B017C0103C0C12CD12C760183E516
:107360000E94D6B8882361F00E9456B820E030E031
:107370004AE754E40F947A1A0F9471226B017C014E
:107380000E94E2698091F216811105C060E085E8F3
:1073900097E00E949BFD0E947AFAC60ED71EE81E57
:1073A000F91E0E947AFADC01CB018C199D09AE0905
:1073B000BF09B7FD02C00C942D4980E00E9418530C
:1073C000F0CF0E940B6F0C942D490E94C99081113F
:1073D0000C942D498CE0EDEDF2E0DE011196019068
:1073E0000D928A95E1F760E070E080E50E94E4C4C8
:1073F000BE016F5F7F4F0E941EFC0C942D4980914F
:10740000520B8770873011F00C94574A60E08FE47C
:107410000E94F66E81110C942D490C94574A80916C
:10742000561781111DC00E94129E8823F9F0115039
:1074300011F40C94314C43EF57E06BEF77E085E0AB
:107440000E949DB961E086EE97E00E94E3B88EEC61
:1074500097E00E9454E60E94C990882301F306C079
:1074600060E08FE40E94F66E8823E9F20E9407B97B
:1074700089E998E00E9454E60C942D492091E61683
:107480003091E7164091E8165091E91660913E1749
:1074900070913F1780914017909141170F94FE20F3
:1074A000AB01BC0188E50E94A5AF69837A838B8319
:1074B0009C832091EA163091EB164091EC16509186
:1074C000ED16609142177091431780914417909187
:1074D00045170F94FE20AB01BC0189E50E94A5AFC2
:1074E0006D837E838F839887BE016B5F7F4FCE0154
:1074F00001960F94C607882311F40C942D4980E05F
:107500000E9460BF0E948DCF61E085E40E94F66E0C
:10751000182F21E0482FBE016B5F7F4FCE010196EF
:107520000E9452F66B017C019B01AC010F94F02389
:1075300081115FC089809A80AB80BC8020E030E000
:10754000A901C501B4010F94141A87FF05C027E1F2
:1075500037EB41E558EB04C027E137EB41E558E351
:10756000C501B4010F94FE20AB01BC018BEB98E088
:107570000E94E0528D809E80AF80B88420E030E091
:10758000A901C501B4010F94141A87FF05C027E1B2
:1075900037EB41E558EB04C027E137EB41E558E311
:1075A000C501B4010F94FE20AB01BC0186EB98E04D
:1075B0000E94E05220E030E0A901C701B6010F941B
:1075C000141A87FF05C067E177EB81E598EB04C0EB
:1075D00067E177EB81E598E3A70196010F94FE2020
:1075E000AB01BC0181EB98E00E94E0528AE00E946E
:1075F000A0500E9474CF113011F40E94F7650E94D0
:10760000F0D20C942D498FE08093ED070C942D4916
:10761000B9EE2B2EB2E03B2E1BE5E12E12E1F12E4E
:107620002EE337E13DA32CA30AEDC02E06E1D02EB8
:1076300000E010E0D1018D911D010E94D6B8882391
:1076400009F44BC00E9456B82B013C01133049F09D
:10765000F60120813181428153810F94FD202B015D
:107660003C01ACA1BDA12D913D914D915C91C30117
:10767000B2010F94FD204B015C012DEB37E346E88E
:1076800055EB0F945E2387FD0AC02DEB37E346E8E8
:1076900055E3C501B4010F94141A1816F4F413300D
:1076A00051F440924A1750924B1760924C177092C7
:1076B0004D1701E012C0A5019401F70160817181AD
:1076C000828193810F94FE20D7016D937D938D93DA
:1076D0009C931397812F0E94E2CB1F5FB4E0EB0EC7
:1076E000F11CECA1FDA13496FDA3ECA3F4E0CF0EB8
:1076F000D11C143009F09ECF002321F08AE497E1D9
:107700000E94F3690E94F0D20C942D4980916F027F
:10771000882311F40C942D4989E40E94D6B8082FCF
:10772000882321F00E9452B8E82E01C0E12C8AE49F
:107730000E94D6B8182F882321F00E9452B8F82E44
:1077400001C0F12C002319F024E02E1528F011239C
:1077500049F034E03F1530F483EC98E00E94B250D9
:107760000C942D4980E1EEE3F7E1A8ECB6E101903D
:107770000D928A95E1F70023F1F02091D01230911B
:10778000D1124E2D4203B001439F700D1124809100
:10779000741190917511680F791F072E000C880BDA
:1077A000990B0F941B1A6093C8167093C916809397
:1077B000CA169093CB161123F1F02091D21230917A
:1077C000D3124F2D4203B001439F700D11248091BD
:1077D000761190917711680F791F072E000C880B96
:1077E000990B0F941B1A6093CC167093CD1680934F
:1077F000CE169093CF1660E080E50E94F66E882347
:10780000C1F10023D1F02091E6163091E7164091A6
:10781000E8165091E9166091C8167091C9168091CA
:10782000CA169091CB160F94FD206093C8167093E2
:10783000C9168093CA169093CB161123D1F02091CC
:10784000EA163091EB164091EC165091ED166091CE
:10785000CC167091CD168091CE169091CF160F94C4
:10786000FD206093CC167093CD168093CE16909326
:10787000CF1640E050E0BA0186E40E94A5AF6B014C
:107880007C0120E030E0A9010F945E2318164CF42F
:1078900020E030E040E752E4C701B6010F94F82140
:1078A00003C060E070E0CB0169837A838B839C83A3
:1078B000CE0101960E94ACCF0C942D490E94AF904E
:1078C0000C942D498091C4129091C5128537910571
:1078D00011F40C946B440CF053C18934910509F4F4
:1078E000F2C40CF069C08A31910509F47DC39CF59E
:1078F0008431910509F4F7C27CF48131910509F4D2
:10790000D1C22CF4029708F44AC20C942149429740
:1079100009F40FC70C9421498731910509F408C374
:107920008CF48531910509F4FFC2469711F00C944F
:1079300021490E94A97B80917916877F80937916CF
:107940000C942D498831910509F40AC3499709F42B
:1079500040C30C9421498F31910509F470C47CF423
:107960008C31910509F4B5C30CF44CC38D319105EC
:1079700009F4B9C34E9709F4BDC30C9421498A3266
:10798000910509F47CC464F48032910509F411C4B2
:10799000819711F00C9421490E9417B60C942D493F
:1079A0008B32910509F48CC4C09711F00C942149D5
:1079B0000E94CF990C942D498836910509F425C56C
:1079C000ECF58135910509F49EC6C4F48C3491051B
:1079D00009F485C44CF48B34910511F00C942149C1
:1079E0000E94E3660C942D498D34910509F47AC404
:1079F0008E34910509F479C40C942149843591059C
:107A000009F497C68CF48235910509F48BC6833549
:107A1000910511F00C9421498091ED078F7E8062D1
:107A20008093ED070C942D498535910509F4ADC679
:107A30008C35910509F4C2C60C9421498E36910506
:107A400009F49CC5D4F48B36910509F48AC554F425
:107A50008936910509F44FC58A36910509F45FC549
:107A60000C9421498C36910511F40C942D498D36D6
:107A7000910509F4E9C40C9421498137910509F471
:107A8000D3C55CF48F36910509F489C5803791051B
:107A900011F40C942D490C9421498237910509F475
:107AA00017C78337910511F00C9421498DE79BE0AE
:107AB0000E94B25060E08DE69BE00E94D9E460E055
:107AC00088E59BE00E94D9E461E081E59BE00E94AB
:107AD000D9E461E086E49BE00E94D9E461E086E3BA
:107AE0009BE00E94D9E460E08DE29BE00E94D9E433
:107AF00061E083E29BE00E94D9E461E089E19BE0E0
:107B00000E94D9E461E081E19BE00E94D9E461E058
:107B100083E09BE00E94D9E461E085EF9AE00E9457
:107B2000D9E460E086EE9AE00E94D9E460E088ED56
:107B30009AE00E94D9E460E082EC9AE00E94D9E4E5
:107B400061E081EB9AE00E94D9E461E082EA9AE088
:107B50000E94D9E461E08DE89AE00E94D9E461E0F6
:107B60008AE79AE00E94D9E460E08DE69AE00E94FC
:107B7000D9E460E089E59AE00E94D9E40C942D49AB
:107B80008E32A1E09A0711F40C9442470CF070C0B9
:107B90008B3C910509F465C7ACF58D37910509F467
:107BA000AFC5BCF48737910509F4E0C60CF4A4C650
:107BB0008837910509F4DDC68937910511F00C94D9
:107BC00021491092B8081092B7080E948AE70C94D5
:107BD0002D498E3B910509F45BC554F48C38910511
:107BE00009F444C58B39910509F464C50C94214905
:107BF000883C910509F4C5C6893C910509F40EC776
:107C00000C9421498C3D910509F482C79CF48D3C6C
:107C1000910509F448C70CF443C78E3C910509F45B
:107C200055C7833D910511F00C9421490E94F7C47A
:107C30000C942D498232E1E09E0711F40C943746F2
:107C400054F48D3D910509F470C7823E910509F405
:107C5000C2C70C9421498C3221E0920711F40C9494
:107C60003A468D32914011F40C944F460C942149C0
:107C7000843F41E0940711F40C946F480CF043C02A
:107C80008239B1E09B0711F40C948C47DCF480330B
:107C9000F1E09F0711F40C94CF4614F40C9486473E
:107CA000803931E0930711F40C9489478139914070
:107CB00011F00C94214981E00E943F660E94F0D2AD
:107CC0000C942D49843AA1E09A0711F40C949F4733
:107CD0006CF48A39E1E09E0711F40C942D498C393B
:107CE000914011F40C9494470C942149853A21E079
:107CF000920711F40C94A2478C3A914011F40C9421
:107D000012480C942149883542E0940711F40C94F0
:107D100097481CF5873FB1E09B0711F40C94754818
:107D20007CF4853FF1E09F0711F40C947248863F84
:107D3000914011F00C9421490E94A4E70C942D4924
:107D4000883F31E0930711F40C947E488C309240C8
:107D500011F40C948F480C9421498C36A3E09A07B7
:107D600011F40C942D497CF48B35E2E09E0711F45C
:107D70000C949A488335934011F00C9421490E9449
:107D8000C1DD0C942D49803A23E0920709F447C2E3
:107D9000873E934011F40C9413490C9421490091AF
:107DA0000D1210910E1280E50E94D6B8882361F062
:107DB0000E94ADF56B017C01BB24B394672B682B4B
:107DC000692B31F4B12C04C0B12CC12CD12C76011B
:107DD00083E50E94D6B8882311F40C94434C0E948A
:107DE00056B820E030E04AE754E40F947A1A0F9432
:107DF00071226B017C01B1100BC0672B682B692BC2
:107E000039F40115110521F0D8018C91811102C0BE
:107E1000B12C02C0BB24B3940E94E269B11003C02C
:107E20008EE096E001C0C8010E947BAF1091EE0782
:107E300083E08093EE0781E080933C1744EF58E0A5
:107E40006DEF78E082E00E949DB982EE98E00E949A
:107E50007BAFC114D104E104F104B1F00E947AFABD
:107E6000C60ED71EE81EF91E0E947AFADC01CB016D
:107E70008C199D09AE09BF09B7FF0EC080913C1750
:107E800081110C94484C08C080913C17882321F044
:107E900080E00E941853F8CF10923C171093EE0721
:107EA0000C942D498091C71284FF02C00C944D4C54
:107EB0008091C91287FF02C00C944D4C8091CA1268
:107EC000837011F00C944D4C60E08FE099E00E94BB
:107ED0009BFD5F988A9880910801817080930601CC
:107EE00012980C942D4987E299E00E94B25081E4E7
:107EF00094E10E94AE938BE1E1E4F4E1DE0111969E
:107F000001900D928A95E1F760E070E0CE01019654
:107F10000E94A97DCE0101960E94E49488E199E037
:107F20000E94B2500C942D490E941A7C0C942D4949
:107F3000E0910D12F0910E128081882329F0803299
:107F400009F410823196F8CF40E061E080910D1283
:107F500090910E120E94067F10923D170C942D49AD
:107F60008091E40A8823E9F080E090E0A0EAB1E49F
:107F700088A399A3AAA3BBA31C8E1D8E1E8E1F8E41
:107F800019821A821B821C8220E0AE01405E5F4F84
:107F9000BE01645E7F4FCE0101960E945DBA0C94D3
:107FA0002D490E945050882321F00E94BA7B0E94E4
:107FB000E36661E088E698E30E94E3B848E359E0AD
:107FC00060E479E085E00E9456BA0E941FFE0C949E
:107FD0002D498091791682FF03C08B7F809379169B
:107FE0000E9421C40C942D498091791683FD02C012
:107FF0000C942D4983E50E94D6B881110C94694CEC
:108000000C942D4983E40E948DB88823C1F186E544
:1080100099E00E94B2508091EB13882339F1BE01A0
:108020006F5F7F4F88EE93E10E9475928E010F5F24
:108030001F4FF80181918F01882319F00E94A050F1
:10804000F8CFCE0101960E94D87E809166198823D0
:1080500089F080E20E94A05006E619E1D8018D91D6
:108060008D01882339F00E94A050F8CF8CE499E06C
:108070000E94B2508AE00E94A0500C942D4983E5E2
:108080000E94D6B8882309F10E943EB8182F90E0CC
:10809000CD970CF01CE31093E2070E947AFA6B0173
:1080A0007C01212F30E0A8EEB3E00F94BE20C60E75
:1080B000D71EE81EF91EC092DE07D092DF07E092BD
:1080C000E007F092E1070C942D490E94827B0C940A
:1080D0002D4940E060E080910D1290910E120E94B7
:1080E000067F0C942D49809179168E7F80937916A6
:1080F0000C942D498091791683FD02C00C942D4972
:108100000E9452F88091791683FD02C00C942D498B
:1081100060910D1270910E12CE014C960E948FEF5D
:108120008C01009711F40C942D496C8D7D8D198272
:108130001C8222E0AC01CE0101960E94DE988111E2
:1081400002C0F12C14C0CE0101960E94FDEE8823DE
:10815000C1F361E0CE0101960E945992009789F324
:1081600025EEFC0120831C820E946894F82ECE012B
:1081700001960E94E494B801FF2089F080E899E01C
:108180000E94C1508AE00E94A05010927516109271
:10819000761610927716109278160C942D4988E670
:1081A00099E00E94C15085E699E00E94B2500C947B
:1081B0002D498091791682FD0E94E269809179169D
:1081C00083FD02C00C942D4960E080E50E94F66EAC
:1081D000182F482F61E080910D1290910E120E948D
:1081E000067F83E50E94D6B8882381F00E942EB8CE
:1081F000AB01BC01409375165093761660937716C9
:108200007093781688EE93E10E946F910E94BA7B7A
:1082100011110C942D490E94E3660C942D49209174
:108220000D1230910E1290917916926090937916FA
:1082300040E060E0C9010E94067F0C942D490E9435
:1082400096FB6C8F7D8F8E8F9F8FBE016F5F7F4FF0
:10825000CE014C960E9438B560E0CE0101960E9496
:10826000F6FD0E94D850BE016F5F7F4F8EE899E007
:108270000E94C1508AE00E94A0500C942D4983E5D1
:108280000E94D6B8882311F40C942D490E943EB860
:10829000F82E6DE070E080E50F94FB088C0197FDEF
:1082A000DCC7E82E60E089E40E94F66E81110C9430
:1082B0007A4C802F0E940E508111AAC40C947A4CE3
:1082C0000E9421C6CAC780E50E948DB8882309F4A0
:1082D000C4C78091791682FDC0C70C94934C0E944C
:1082E000E5FBBBC70E949367B8C760E070E083E519
:1082F0000F94FB088E34910529F40E9445680E9472
:108300001FFEABC789EF99E00E94B2506091A708A9
:108310007091A80880EF99E00E94AE516091A90881
:108320007091AA0883EE99E00E94AE516091A7086F
:108330007091A8088091A9089091AA08681B790BF0
:108340008091AF0A815021E030E0823010F020E0CF
:1083500030E0621B730B88ED99E00E94AE518AE019
:108360000E94A05080ED99E00E94B2508091AB082D
:108370009091AC08A091AD08B091AE088C8F9D8F04
:10838000AE8FBF8FBE016F5F7F4FCE014C960E94B4
:1083900038B5BE016F5F7F4F83EC99E00E94C150FA
:1083A0008091AF089091B008A091B108B091B20847
:1083B0008C8F9D8FAE8FBF8FBE016F5F7F4FCE01C1
:1083C0004C960E9438B5BE016F5F7F4F83EB99E0FA
:1083D0000E94C15020E030E04AE754E46091B308C5
:1083E0007091B4088091B5089091B6080F94F82167
:1083F000AB01BC018BE999E00E94E0528DE60E943E
:10840000A0508AE00E94A05028C780911A1183FDD5
:1084100024C70E94FCC287FD20C783E50E94D6B80E
:10842000882379F00E9456B80F946A228B01CB0101
:108430000E94E4DB0635110524F40E9493670E9434
:108440001FFE0F949F1309C780911A1183FD05C762
:108450000E94FCC2F82E87FD00C783E50E94D6B8B3
:10846000082F811106C082E50E94D6B8182F8823F4
:10847000C1F10E9456B80F946A22CB010E94E4DB3E
:108480000E9456B820E030E04AEA52E40F94141AF1
:10849000181614F40C949E4C0E9493670E941FFEC1
:1084A0006091890B70918A0B072E000C880B990B39
:1084B0000F941B1A4B015C014090850B5090860B6A
:1084C0006090870B7090880BA30192010F945E233C
:1084D000181614F40C94BC4C002311F40C94A24C08
:1084E00011E00F949F13112309F4B7C6602F8F2D4D
:1084F0000E94E0D5B2C60E94FCC2182F87FD0AC0B8
:108500008CE19AE00E94B250812F0E94EBD38AE066
:108510000E94A050FCADF093EE070C94264E60E054
:1085200080E50F940A09182F823008F096C681E47E
:108530000E948DB8882321F060916E0B70E002C01C
:108540006FEF70E083E50E94E4C4E12FF0E0E259B0
:10855000F44F8F3F910519F010F08FEF90E080837A
:108560007CC660E080E50F940A09823008F075C689
:10857000E82FF0E0E259F44F10826FC68EE40E94BB
:10858000D6B8882309F469C60E942EB860930912F0
:1085900070930A1280930B1290930C125EC683E5BF
:1085A0000E948DB8882331F060E083E50F940A09BA
:1085B00080931A110E94D8508DE29AE00E94B25026
:1085C00080911A11882369F1A3E2EA2EAAE0FA2E1B
:1085D00000E010E020E080911A1190E0A0E0B0E00F
:1085E000002E04C0B695A795979587950A94D2F763
:1085F00080FF0EC0DD24D394D20E222319F08CE22A
:108600000E94A050F701859194910E94B2502D2DA7
:108610000F5F1F4F32E0E30EF11C05301105D9F654
:1086200029CD8FE19AE024CD83E50E94D6B8882336
:1086300071F00E943EB8282F30E02D3331051CF434
:10864000809300020AC68CE38093000206C60E9453
:10865000D8504091000250E060E070E084E39AE07E
:108660000E949D518AE00E94A050F7C580911A1186
:1086700083FDF3C583E50E94D6B8882309F4EDC5D0
:108680000E9456B80F946A22CB010E94D86EE5C5AD
:1086900080911A1183FDE1C583E50E94D6B8182F99
:1086A00081110C94BF4C82E50E94D6B881110C94C4
:1086B000BF4CD3C583E50E94D6B8882309F4CDC545
:1086C0000E943EB8182F90E0CD970CF01CE3109359
:1086D000E7070E947AFA6B017C01212F30E0A8EEB7
:1086E000B3E00F94BE20C60ED71EE81EF91EC0923E
:1086F000E307D092E407E092E507F092E607ADC504
:108700000E9421C4AAC50E94F5DB0E9493670E94C3
:10871000476B0E945E5068EE73E080E090E00E943C
:10872000E84F9BC58091ED078F7D80618093ED07B9
:1087300094C583E50E94D6B8882399F00E9456B864
:1087400020E030E04AE754E40F947A1A0F94712243
:1087500060930102709302028093030290930402DB
:108760007CC58091C71284FF02C00C94F44C8091A8
:10877000C91287FF02C00C94F44C8091CA12837016
:1087800011F00C94F44C0C94254D83E50E948DB8A7
:10879000882309F462C50E9456B820E030E04AE719
:1087A00054E40F947A1A0F9471226093E80770933F
:1087B000E9078093EA079093EB074FC50E94FCC23C
:1087C00087FD4BC59091C71294FD04C09091C912CA
:1087D00097FF0AC0E9EECE2EE2E0DE2EFBE1EF2E9F
:1087E000F1E1FF2E10E009C09091CA12937091F749
:1087F000682F81E00E94E6C530C5D6018D916D01DC
:108800000E94D6B8882309F459C0133009F04FC02C
:108810000E9456B84B015C0120E030E040EA51E490
:108820000F94141A87FF3AC0A501940160913B117F
:1088300070913C1180913D1190913E110F94F8215F
:108840002B013C019B01AC0160914B1170914C11CB
:1088500080914D1190914E110F947A1A60934B11A3
:1088600070934C1180934D1190934E116091660B53
:108870007091670B8091680B9091690B0F94191A96
:10888000A30192010F947A1A0F9471226093660BE0
:108890007093670B8093680B9093690B80923B11E8
:1088A00090923C11A0923D11B0923E1107C00E94DF
:1088B00056B8F701648B758B868B978B1F5FF4E03E
:1088C000EF0EF11C143009F098CF0E94BE69C5C4A8
:1088D0000E94F3E4C2C480910D1290910E12009791
:1088E00041F0DC012C91222321F060E00E94F6FD92
:1088F000B4C40E941FFEB1C400910D1210910E125B
:1089000094E0F12C40E0915021F1F8018081282F72
:108910002B7F213421F421812133D9F407C0803504
:10892000C1F4818180538A3048F013C0813421F032
:10893000853421F441E002C0FF24F39498012E5FB6
:108940003F4F89012F5F3F4FF80180818032C9F38B
:10895000DACF41110E94D850FF2021F088E69CE038
:108960000E94B250C8010E94F75277C40E9467E784
:1089700074C481E08093B8088093B7080E948AE7A6
:108980006CC40E94FCC2182F87FD67C484E40E9457
:108990008DB8882309F43FC00E9456B86B017C0152
:1089A00001E020E030E0A9010F94141A811101C008
:1089B00000E00093671220E030E0A901C701B60192
:1089C0000F94141A882339F10E9456B824E0120239
:1089D000F0011124E459FD4E6083718382839383F7
:1089E00020E030E0A90160916C1270916D128091CD
:1089F0006E1290916F120F94141A81110CC080E0C6
:108A000090E0A0EEBFE380936C1290936D12A09360
:108A10006E12B0936F120E9463C81FC40E94FCC202
:108A200087FD1BC479EEE72E72E0F72E0BE111E112
:108A3000D7018D917D010E948DB8882359F00E9445
:108A400056B80F947122F8016083718382839383F7
:108A50000E9477690C5F1F4FF1E10B321F0741F74E
:108A6000FCC30E94FCC287FDF8C369EEE62E62E0FB
:108A7000F62E0BE111E1D7018D917D010E948DB899
:108A8000882339F00E9456B8F80164A375A386A321
:108A900097A30C5F1F4FF1E10B321F0761F7DDC396
:108AA0000E9437F5DAC38091C71281FF02C00C948F
:108AB000284D8091C81281FF02C00C94284D8091EE
:108AC000C9128C7011F00C94284DC7C349EEC42E06
:108AD00042E0D42E5CEBE52E58E0F52E10E0D601F6
:108AE0008D916D010E948DB8882351F00E9456B877
:108AF000F7016083718382839383812F0E94E2CB8D
:108B00001F5FF4E0EF0EF11C133049F70C94823B29
:108B100083E50E94D6B8882309F49FC30E9452B807
:108B2000909355028093540298C30E94FCC2F82E81
:108B300087FD93C383E50E94D6B80F2D0F2C000C40
:108B4000110B882369F10E9452B8F801EE0FFF1F44
:108B5000E65AFD4F91838083000F111F000F111FF4
:108B60009801255D3D4F7901BC01990F880B990B48
:108B70000F941B1A2AE037ED43E25CE30F947A1A54
:108B8000F801E859FD4E20813181428153810F94D3
:108B90007A1AD7016D937D938D939C9313975DC340
:108BA0000E94D85085E40E94A05080E38F0D0E945F
:108BB000A050F801EE0FFF1FE65AFD4F6081718152
:108BC0008BE89CE00E94D75185E20E94A0508AE089
:108BD0000E94A05042C380E50E948DB8882309F40A
:108BE0003CC360E070E080E50F94FB08F82E6FEF67
:108BF0007FEF83E50F94FB088C010196039708F043
:108C00002CC3F7FC2AC38F2D0E940E50882339F005
:108C10000E94D45083E99CE00E94B2501EC30E947F
:108C2000E26960E08F2D0E941CF90F3FBFEF1B0728
:108C300031F00130110571F000E010E00DC08F2D12
:108C40000E94C4F831E020E0892B09F030E0032FC6
:108C5000122F02C001E010E08F2D0E94C4F880178F
:108C6000910709F4FAC280E00E941853F5CF0E94E0
:108C70006DE0F3C264E071E083E50E94E4C48C011E
:108C800068EE73E080E50E94E4C48938E3E19E0762
:108C900010F088E893E1B8010E943CFDDEC260E07C
:108CA00085E40F940A09811173C080E50E948DB894
:108CB000882351F00E9456B860938C0B70938D0BF3
:108CC00080938E0B90938F0B89E40E948DB888233C
:108CD00081F00E9456B82CEA35EC47E25EE30F942F
:108CE0007A1A6093900B7093910B8093920B9093F0
:108CF000930B84E40E948DB8882381F00E9456B8BB
:108D00002CEA35EC47E25EE30F94F8216093940B74
:108D10007093950B8093960B9093970B0E94D8506D
:108D200040918C0B50918D0B60918E0B70918F0B3D
:108D30008CEB9CE00E94E0522CEA35EC47E25EE3CB
:108D40006091900B7091910B8091920B9091930B8D
:108D50000F94F821AB01BC0188EB9CE00E94E0522B
:108D60002CEA35EC47E25EE36091940B7091950B31
:108D70008091960B9091970B0F947A1AAB01BC01DE
:108D800084EB9CE00E94E0528AE00E94A05065C201
:108D90000E94D45082EA9CE00E94B2505EC280E5FC
:108DA0000E948DB8882351F00E9456B860939708AE
:108DB000709398088093990890939A0889E40E9488
:108DC0008DB8882381F00E9456B82CEA35EC47E232
:108DD0005EE30F947A1A60939B0870939C088093CB
:108DE0009D0890939E0884E40E948DB8882381F0AA
:108DF0000E9456B82CEA35EC47E25EE30F94F82166
:108E000060939F087093A0088093A1089093A20894
:108E10000E94D85040919708509198086091990805
:108E200070919A0888EC9CE00E94E0522CEA35ECA4
:108E300047E25EE360919B0870919C0880919D08D9
:108E400090919E080F94F821AB01BC0184EC9CE04A
:108E50000E94E0522CEA35EC47E25EE360919F0805
:108E60007091A0088091A1089091A2080F947A1A9D
:108E7000AB01BC0180EC9CE00E94E0528AE00E94C1
:108E8000A050EBC183E50E948DB8182F882371F0A4
:108E90000E9456B80F946A227093300260932F029A
:108EA00021E0672B09F020E02093800B80E50E94F1
:108EB0008DB8882359F020912F0230913002232B56
:108EC00011F00E94E66E8093800BC7C11111C5C1DD
:108ED0000E94D85088EE9CE00E94B2508091800B96
:108EE000882319F080ED9CE002C08CEC9CE00E948D
:108EF000B25060912F027091300287ED9CE00E9489
:108F0000D75183ED9CE00E94B250A7C10E94BCAF34
:108F1000A4C10E94E269A1C180E00E943F660E9454
:108F2000F7650E94F0D299C18091C712887809F044
:108F3000E8C58091C912867009F0E3C512C60F9486
:108F400016098BC16FEF7FEF89E40F94FB08F82EB1
:108F50006FEF7FEF8AE40F94FB08E82E8AE50E940A
:108F60008DB8182F811105C081E50E948DB8B82EEB
:108F700001C0B12CF7FC06C0E7FC04C0111109C008
:108F8000B11007C00E94D45082E59DE00E94B2500B
:108F900064C1F4E0FF1510F0FE1538F40E94D450BF
:108FA00083E39DE00E94B25058C1CF2C0F2C000CDF
:108FB000DD080E2D0E2C000C110B0E9456B8BB20A4
:108FC00099F025E02C9DF0012D9DF00D1124E00F6E
:108FD000F11FEE0FFF1FEE0FFF1FE452FD4E208129
:108FE00031814281538103C020E030E0A9010F9418
:108FF000FE209B01AC0185E08C9DF0018D9DF00D64
:109000001124E00FF11FEE0FFF1FEE0FFF1FE452C0
:10901000FD4E20833183428353836E2D8F2D0E941A
:1090200077AE1BC10E94C990811117C10CEC1BE2E5
:109030002EE337E13DA32CA3CE0101961C0141E2B2
:10904000C42E4CE2D42E7C01F80165917591859176
:109050009491ACA1BDA18D909D90AD90BD90BDA30C
:10906000ACA3A50194010F94FD202B013C01F70155
:10907000608371838283938320E030E040EA51EC87
:109080000F945E2387FD0AC020E030E040EA51E4FF
:10909000C301B2010F94141A18162CF4F60184912E
:1090A00018160CF482C5D7018D909D90AD90BD909F
:1090B0007D0120E030E040EA51ECC501B4010F949D
:1090C0005E2387FD7CC520E030E040EA51E4C50125
:1090D000B4010F94141A18160CF083C570C50E94C1
:1090E00077A9BBC00E9407ECB8C061E083E50E948D
:1090F000F66E91E089270E9411E9AFC081E080936C
:10910000CB120E947EA31092CB12882309F4A5C033
:109110000E94D8508EEA9DE00E94B2509EC080917D
:10912000791682FF9AC080648093791696C00E9457
:1091300025C393C00E94FCC2082F87FD8EC085E521
:109140000E948DB88823B1F1E02E002E000CFF089C
:109150000E9456B84B015C0120E030E0A9010F9459
:109160005E2387FF04C0B7FAB094B7F8B094C70184
:1091700023E0880F991F2A95E1F79C012C523D4E60
:109180007901D9018D929D92AD92BC92139720E006
:1091900030E04AEF53E4C501B4010F945E23181682
:1091A0004CF480E090E0AAEFB3E4F7018083918370
:1091B000A283B3838CE40E948DB8882309F44DC048
:1091C000002E000C110B0E9456B86B017C0120E0B0
:1091D00030E0A9010F945E2387FF04C0F7FAF094F2
:1091E000F7F8F09420E030E04AEF53E4C701B6010D
:1091F0000F945E23980193E0220F331F9A95E1F7B5
:10920000F901EC52FD4E18162CF0C482D582E6828C
:10921000F78223C080E090E0AAEFB3E484839583D3
:10922000A683B7831AC081E080936F021092321731
:1092300060E083E50E94F66E81110FC00E943CB78A
:109240000CC00E94AF9009C08091C412882329F0FD
:109250000E94D6D302C00E94AF902296FFAD229703
:10926000F11102C00E94E7B62CAD2093EE07EEC4C8
:1092700020E030E0A901C701B6010F94141A881F3D
:109280008827881F181709F4F3C080E090E0A0E851
:10929000BFEB88AF99AFAAAFBBAF28A539A54AA548
:1092A0005BA568A979A98AA99BA90F94FD202B0128
:1092B0003C012CA53DA54EA55FA56CA97DA98EA955
:1092C0009FA90F94FD206CA37DA38EA39FA3A30150
:1092D0009201C301B2010F947A1A4B015C012CA1D7
:1092E0003DA14EA15FA1CA01B9010F947A1A9B0159
:1092F000AC01C501B4010F94FE200F94AC234B01C7
:109300005C0120E030E040E05FE30F947A1A2196A0
:109310006CAF7DAF8EAF9FAF2197A7019601C701BC
:10932000B6010F947A1A6B017C0121962CAD3DADEC
:109330004EAD5FAD2197CA01B9010F947A1A9B0116
:10934000AC01C701B6010F94FD200F94AC236B0153
:109350007C018CA19DA1AEA1BFA1B0588CA39DA3FF
:10936000AEA3BFA32DEB37E346E855EBC501B4012F
:109370000F945E2387FD0AC02DEB37E346E855E3E3
:10938000C501B4010F94141A18165CF4A5019401D8
:1093900060E070E080E89FE30F94F8214B015C01EE
:1093A00003C0812C912C5401A5019401C301B20189
:1093B0000F947A1A28AD39AD4AAD5BAD0F947A1A85
:1093C000A70196010F947A1A2B013C0128A939A90B
:1093D0004AA95BA968A579A58AA59BA50F94FE203B
:1093E00020E030E040E05FE30F947A1A9B01AC018B
:1093F000C301B2010F94FE2028A539A54AA55BA59B
:109400000F94FD2069837A838B839C83A50194014B
:109410006CA17DA18EA19FA10F947A1A28AD39ADC0
:109420004AAD5BAD0F947A1AA70196010F947A1A90
:109430006B017C012CA93DA94EA95FA96CA57DA556
:109440008EA59FA50F94FE2020E030E040E05FE372
:109450000F947A1A9B01AC01C701B6010F94FE204C
:109460002CA53DA54EA55FA50F94FD200C94843935
:1094700080E090E0A0E8BFE30CCF412FBE016F5F1A
:109480007F4F88EC96E10E9413E10E947AFA609384
:109490004113709342138093431390934413DDCE92
:1094A0000E94D4508FE697E00E94B250D6CE0E9420
:1094B000E269909156179CAB80E00E9460BF0E94C9
:1094C0008DCF81E08093B8080E948AE788E50E94EA
:1094D0008DB8182F89E50E948DB8082F8AE50E9463
:1094E0008DB81013BCC1181711F0012FB8C101E0DD
:1094F00011E091E09CA780E1EEE3F7E1A8ECB6E192
:1095000001900D928A95E1F782E50E94D6B88823F2
:1095100061F00E9456B86B017C0120E030E0A901A7
:109520000F94141A882369F106C0C12CD12C80E84D
:10953000E82E80E4F82E111103C0002309F4FCC0CA
:10954000C092D016D092D116E092D216F092D316D5
:10955000A7019601609146177091471780914817AF
:10956000909149170F94141A87FF0BC019821A8221
:109570001B821C82BE016F5F7F4F80ED96E10E94CF
:1095800011D1112309F4D3C0002309F4CDC01092E6
:109590003E1710923F1710924017109241171092E9
:1095A00042171092431710924417109245170E94C9
:1095B000C4D1E1E2FCE2A491A8AFE5E1FCE2C590F0
:1095C000D590E590F490E9E1FCE285909590A59026
:1095D000B490A5019401C701B6010F945E2318163B
:1095E0002CF4A7019601C501B40104C0A5019401A2
:1095F000C701B6010F94F8212B013C01ECEDFBE211
:1096000085919591A591B4918CA39DA3AEA3BFA381
:10961000E8EDFBE285919591A591B49188A799A772
:10962000AAA7BBA79C01AD016CA17DA18EA19FA1A2
:109630000F945E23181634F428A439A49AA598AB85
:109640001BA505C02CA03DA0AEA1A8AB1FA1A301E6
:109650009201C301B2010F947A1A20E030E040E891
:109660005FE30F94FE200F94AC23910148A9512F82
:109670000F947A1A68A379A38AA39BA3E2E2FCE27F
:10968000149120E030E040EC5FE3C501B4010F9499
:109690007A1A4B015C01612F110F770B880B990B24
:1096A0000F941B1A9B01AC01C501B4010F947A1AE7
:1096B00069837A838B839C8320E030E040EC5FE316
:1096C000C701B6010F947A1A6B017C01B8AD6B2FFC
:1096D000BB0F770B880B990B0F941B1A9B01AC01E6
:1096E000C701B6010F947A1A6C8F7D8F8E8F9F8F72
:1096F000AE01405E5F4FBE016F5F7F4FCE014C9663
:109700000E94EFD00E9499E710923E1710923F17E7
:10971000109240171092411710924217109243175F
:10972000109244171092451780E00E94C6D1002382
:1097300019F081E00E94C6D1ECA5EE2309F481C0A6
:10974000809149138370833051F060E080EC97E0A2
:109750000E949BFD0E94D85081EB97E06EC00E9452
:10976000C4D18090461790904717A0904817B090AA
:1097700049172091E6163091E7164091E81650916E
:10978000E91660E070E088E492E40F94FD206093B5
:10979000C8167093C9168093CA169093CB16209161
:1097A000EA163091EB164091EC165091ED1660E000
:1097B00070E088E492E40F94FD206B017C016093DB
:1097C000CC167093CD168093CE169093CF16209121
:1097D000EE163091EF164091F0165091F116C5013A
:1097E000B4010F94FD206093D0167093D11680932E
:1097F000D2169093D316B701A60188EC96E10F9488
:10980000E20A882389F019821A821B821C82AE0127
:109810004F5F5F4F6CEC76E188EC96E10E94EFD0F1
:1098200082E00E94C6D10BC060E080EA97E00E940F
:109830009BFD0E94D8508EE897E00E94B2500E9493
:10984000F7650E94C4D18091B7088093B8088CA9AD
:109850000E9460BF0E9474CF0E94F0D2FECC8CA701
:109860004ACE61E08CE898E00E94E3B887E198E096
:109870000E9454E661E080E498E30E94E3B888E047
:1098800098E00E9428EEB1100C94083F0C94013F20
:1098900080E00E9418530C94343F88E50E948DB8F4
:1098A00081115F9889E50E948DB881118A988AE5B7
:1098B0000E948DB8882329F08091080181708093DF
:1098C000060185E40E948DB8882309F4C6CC12985D
:1098D000C4CC0E942EB8AB01BC01409375165093C6
:1098E0007616609377167093781688EE93E10E944F
:1098F0006F91B3CC61E0802F0E941CF96F2D802FF7
:109900000E94EDF86F2D70E0802F0E9458F9A7E0BB
:10991000EA1203C0F0926F0BA0CCB9E0EB129DCC21
:10992000F0926E0B9ACC0E943EB890E0853691057D
:1099300014F084E690E080933D178FCC0E94E3669C
:109940000C945042A3019201C501B4010F945E230F
:10995000181694F081E09AE09F938F9387E19AE044
:109960009F938F931F920E9438F60F900F900F9045
:109970000F900F900C9470428CE09AE0EDCF0E9413
:1099800056B80F946A22CB010E94D86E0E9456B836
:1099900020E030E040EA50E40F945E23181614F4FF
:1099A0000E94E3666091940870919508072E000C60
:1099B000880B990B0F941B1A2091900830919108F5
:1099C00040919208509193080F945E2318161CF44E
:1099D0008AE49AE002C08BE39AE060E00E949BFD7B
:1099E000812F0E9462D439CC0E94E26988E50E94EE
:1099F0008DB8882331F05F9A809149138E7F8093D0
:109A0000491389E50E948DB8882331F08A9A8091A4
:109A100049138D7F809349138AE50E948DB888236E
:109A200059F08091080180958170809306018091A2
:109A300049138B7F8093491385E40E948DB8882356
:109A400009F40BCC0E940C5008CC0E94476B05CC4B
:109A500082E40E948DB8882351F00E94ADF5609396
:109A60002B1170932C1180932D1190932E1183E55F
:109A70000E948DB8882351F00E9456B860935B1104
:109A800070935C1180935D1190935E1184E50E9448
:109A90008DB8882351F00E9456B860935F1170937F
:109AA000601180936111909362118AE40E948DB8D5
:109AB000882309F4D2CB0E9456B86B017C012AE0BE
:109AC00037ED43E25CE30F945E2387FD13C02AE980
:109AD00039E949E95EE3C701B6010F94141A181673
:109AE0004CF0C092560BD092570BE092580BF0926C
:109AF000590BB3CB0E94D4508CE69CE00E94B2502C
:109B0000ACCB88E40E948DB8882321F00E94E66ED9
:109B10008093EC0782E50E948DB8082F83E50E94B0
:109B20008DB8182F011102C0882351F010928A08B5
:109B30000E943350112321F00E94E66E809315029B
:109B400084E40E948DB8882309F487CB0E9456B81C
:109B5000609363027093640280936502909366023F
:109B60007CCB0E94D85082E29DE00E94B25080914E
:109B70001502811117C08BEF9CE00E94B2508AE061
:109B80000E94A0504091630250916402609165026E
:109B90007091660282E09DE00E94E0528AE00E949D
:109BA000A0505BCB8FEF9CE0E8CFB7FAB094B7F84A
:109BB000B094F70180829182A282B38274CA0E941B
:109BC000D45080E99DE00E94B25061E082E89DE0BF
:109BD0000E949BFD68E270E088EC90E00E943CFDF2
:109BE0003CCB0C5F1F4FFFEFCF1ADF0A2BE2083D83
:109BF000120709F029CA3CEBE32E38E0F32E10E0FF
:109C0000F10181919191A191B1911F01F70181938E
:109C10009193A193B1937F01812F0E94E2CB1F5FAB
:109C2000133071F70E94F0D260E082E79DE00E945D
:109C30009BFD63E972E084E690E00E943CFD6AEBE4
:109C400072E084E690E00E943CFD07CBCF5BDF4FE3
:109C50000FB6F894DEBF0FBECDBFDF91CF911F913D
:109C60000F91FF90EF90DF90CF90BF90AF909F90BB
:109C70008F907F906F905F904F903F902F900895BE
:109C80002F923F924F925F926F927F928F929F920C
:109C9000AF92BF92CF92DF92EF92FF920F931F93FA
:109CA000CF93DF93CDB7DEB760970FB6F894DEBFE2
:109CB0000FBECDBF8A876B87942EA22E282F30E04F
:109CC0003D872C8770E07987688715E0129FC00177
:109CD000139F900D11249F878E87FB01E80FF91FBA
:109CE000EE0FFF1FEE0FFF1FE452FD4E60817181EA
:109CF000828193819B01AC010F94F023882309F4A6
:109D00004EC14A85490D2B852A0D149FB00111249F
:109D1000E885F985E60FF71FEE0FFF1FEE0FFF1F17
:109D2000E452FD4ED080E180F2800381490D149F02
:109D3000A0011124E885F985E40FF51FEE0FFF1F40
:109D4000EE0FFF1FE452FD4E1081918082807380E0
:109D5000822F90E0EE85FF85E80FF91FEE0FFF1FC1
:109D6000EE0FFF1FE452FD4E608051803280338140
:109D700039832A0D30E0EE85FF85E20FF31FEE0FE9
:109D8000FF1FEE0FFF1FE452FD4EFF87EE87F081AD
:109D9000FA83EE85FF85F181FB83EE85FF85F281F5
:109DA000FC83EE85FF85F381FD83FB01E80FF91F3E
:109DB000EE0FFF1FEE0FFF1FE452FD4E60816E831A
:109DC000B18072817F8383818E87FA01E20FF31F56
:109DD000EE0FFF1FEE0FFF1FE452FD4E4080A180EB
:109DE0009281988B2380212F392D482D572D612F5B
:109DF000792D882D972D0F94F023882321F010E0E2
:109E0000912C812C712C2D2D3E2D4F2D502F6D2DF1
:109E10007E2D8F2D902F0F94F023882321F0D12EAB
:109E2000E92CF82C072D2A813B814C815D816A81C8
:109E30007B818C819D810F94F023882321F01A82ED
:109E40001B821C821D82262D352D432D5981662DA6
:109E5000752D832D99810F94F023882329F06A8032
:109E60005B803C80ED81E983242D3A2D4889522D79
:109E7000642D7A2D8889922D0F94F023882321F068
:109E8000412CA12C188A212C2E813B2D4F815E85DF
:109E90006E817B2D8F819E850F94F023882329F07E
:109EA0004E82BA2CF889FF832E862D2D3E2D4F2D04
:109EB000502F6D2D7E2D8F2D902F0F94FE20212F52
:109EC000392D482D572D0F94FD206B017C01262D37
:109ED000352D432D5981662D752D832D99810F9434
:109EE000FE202A813B814C815D810F94FD209B01E6
:109EF000AC01C701B6010F94FE203B014C012E813D
:109F00003B2D4F815E856E817B2D8F819E850F94C9
:109F1000FE20242D3A2D4889522D0F94FD209B01BF
:109F2000AC01C401B3010F94FE2020E030E040E416
:109F300050E40F94F8219B01AC0185E06C857D8590
:109F4000869FF001879FF00D112488859985E80F81
:109F5000F91FEE0FFF1FEE0FFF1FE452FD4E20838F
:109F60003183428353836B858A8560960FB6F8945C
:109F7000DEBF0FBECDBFDF91CF911F910F91FF903C
:109F8000EF90DF90CF90BF90AF909F908F907F9099
:109F90006F905F904F903F902F900C9477AE6096AB
:109FA0000FB6F894DEBF0FBECDBFDF91CF911F91EA
:109FB0000F91FF90EF90DF90CF90BF90AF909F9068
:109FC0008F907F906F905F904F903F902F9008956B
:109FD000CF92DF92EF92FF926B017C0183E3C81670
:109FE000D104E104F10470F082E3C81AD108E10859
:109FF000F10862E370E080E090E00E9440FA0F9484
:10A000005303ECCFC701B6010E9440FAFF90EF90D6
:10A01000DF90CF900D945303129A0895FF920F93FF
:10A020001F93CF93DF931F92CDB7DEB7F82E03EDCA
:10A030001DE041E050E0B801CE0101960F944E19A9
:10A0400089818F1102C081E007C00F5F1F4F8DE033
:10A050000C3E180771F780E00F90DF91CF911F91B0
:10A060000F91FF9008958091630290916402A091F6
:10A070006502B09166028093520A9093530AA093AE
:10A08000540AB093550A089580910108811107C0C0
:10A090000E9407EC882319F081E08093010808955D
:10A0A0009091791693FB882780F993FF06C081E091
:10A0B0009091EB13911101C080E00895EEE6FBE072
:10A0C0001082118208958F929F92AF92BF92CF9289
:10A0D000DF92EF92FF920F93CF93DF931F92CDB752
:10A0E000DEB75C016B017A014901F5018081918144
:10A0F0000F9444208983002311F0F6018083BE0170
:10A100006F5F7F4FC4010E94BFEDF5018081918197
:10A11000019691838083FFEFCF1ADF0A81E0E81A6E
:10A12000F10819F780E00F90DF91CF910F91FF9028
:10A13000EF90DF90CF90BF90AF909F908F90089559
:10A140009091C00095FFFCCF8093C6000895CF93F7
:10A15000C82FCC2329F080E20E94A050C150F9CF33
:10A16000CF910895CF93DF93FC018491EF01219665
:10A17000882321F00E94A050FE01F7CFDF91CF91FC
:10A1800008950F931F93CF93DF938B010E94B250DA
:10A19000E8018991882319F00E94A050FACFDF913D
:10A1A000CF911F910F9108958BE090E10C94B250E4
:10A1B00085E090E10C94B2507F928F929F92AF9283
:10A1C000BF92CF92DF92EF92FF920F931F93CF93A4
:10A1D000DF931F92CDB7DEB77C0159018B016B0174
:10A1E000C40ED51E0C151D0559F1F7018080918014
:10A1F000F80171908F017982C4010F944420781680
:10A2000091F0672DC4010F944C20C4010F94442099
:10A210009981891741F00E94D85089EB9DE00E94F6
:10A22000B25081E00EC0BE016F5F7F4FC5010E943A
:10A23000BFEDF70180819181019691838083D2CF18
:10A2400080E00F90DF91CF911F910F91FF90EF90E1
:10A25000DF90CF90BF90AF909F908F907F900895A8
:10A260008F929F92AF92BF92EF92FF920F931F93A4
:10A27000CF93DF93CDB7DEB7A0970FB6F894DEBFCC
:10A280000FBECDBF611571058105910591F100E00B
:10A29000842E912CA12CB12C102FEE24E394F12CC0
:10A2A000EC0EFD1EE00EF11C07FDFA94A5019401D1
:10A2B0000F946A20F7016083B901CA010F5F61152D
:10A2C00071058105910541F71F3F31F1E1E0F0E0B3
:10A2D000EC0FFD1FE10FF11D17FDFA9580818A300B
:10A2E00010F097E301C090E3890F0E94A050115035
:10A2F000EBCF80E3A0960FB6F894DEBF0FBECDBFC4
:10A30000DF91CF911F910F91FF90EF90BF90AF9091
:10A310009F908F900C94A050A0960FB6F894DEBF3B
:10A320000FBECDBFDF91CF911F910F91FF90EF90A6
:10A33000BF90AF909F908F900895CF92DF92EF9251
:10A34000FF926A017B010E94B2504AE0C701B60148
:10A35000FF90EF90DF90CF900C943051CF93DF932C
:10A36000EB010E94B250BE0180E090E04AE0DF9134
:10A37000CF910C943051CF92DF92EF92FF926B010C
:10A380007C0197FF0BC08DE20E94A050F094E094F6
:10A39000D094C094C11CD11CE11CF11C4AE0C7013F
:10A3A000B601FF90EF90DF90CF900C943051CF9397
:10A3B000DF93EB010E94B250BE01DD0F880B990BB9
:10A3C000DF91CF910C94BB518F929F92AF92BF922D
:10A3D000CF92DF92EF92FF92CF936B017C01B42E6C
:10A3E00020E030E0A9010F94141A87FF07C08DE226
:10A3F0000E94A050F7FAF094F7F8F094C0E060E003
:10A4000070E080E09FE3CB1541F02DEC3CEC4CEC90
:10A410005DE30F947A1ACF5FF6CF9B01AC01C701C1
:10A42000B6010F94FE206B017C010F9471224B0149
:10A430005C014AE00E943051CC2389F1C501B4018E
:10A440000F94191A9B01AC01C701B6010F94FD20AE
:10A450006B017C018EE20E94A05020E030E040E2DF
:10A4600051E4C701B6010F947A1A4B015C010F94B5
:10A470006A226B01770FEE08FF08C701B6010E9440
:10A48000BB51C701B6010F941B1A9B01AC01C5015A
:10A49000B4010F94FD206B017C01C150F1F6CF9106
:10A4A000FF90EF90DF90CF90BF90AF909F908F90F4
:10A4B00008958F929F92AF92BF92CF92DF92EF92C8
:10A4C000FF920F931F93CF93DF9382E190E10E945D
:10A4D000B250C12CD12C760186E00E94A750C70152
:10A4E000B6010E94BB518FEFC81AD80AE80AF80AD1
:10A4F00095E0C916D104E104F10471F78AE00E94E5
:10A50000A0500CED12E1C12CD12C760180E20E940A
:10A51000A050C701B6010E94BB51C0E0D0E080E26C
:10A520000E94A050F801EC0FFD1F80809180A28056
:10A53000B380A5019401C501B4010F94F0238111EA
:10A5400012C020E030E0A901C501B4010F945E23E0
:10A5500087FD03C08BE20E94A05043E0C501B40117
:10A560000E94E45109C0B12C80E20E94A050B39433
:10A570008DE396E0B912F9CF6496C436D10579F629
:10A580008AE00E94A0508FEFC81AD80AE80AF80A99
:10A590000C5F1F4F95E0C916D104E104F10409F0E6
:10A5A000B5CF8AE0DF91CF911F910F91FF90EF908F
:10A5B000DF90CF90BF90AF909F908F900C94A05061
:10A5C000CF92DF92EF92FF926A017B010E94B2501C
:10A5D00042E0C701B601FF90EF90DF90CF900C945E
:10A5E000E4518DE00E94A0508AE00C94A050CF93DB
:10A5F000DF93EC018991882319F00E94A050FACFD3
:10A60000DF91CF910C94F152809185119091861138
:10A61000981759F0E92FF0E0EB57FE4E82819F5FCB
:10A620009F779093861190E008958FEF9FEF0895A4
:10A630002F923F924F925F926F927F928F929F9252
:10A64000AF92BF92CF92DF92EF92FF920F931F9340
:10A65000CF93DF93CDB7DEB728970FB6F894DEBF60
:10A660000FBECDBFE82E0E94F81C0E947AFA4B0163
:10A670005C0180910002882359F18091EE078823C4
:10A6800039F14091020850910308609104087091DB
:10A69000050895018401041B150B260B370B37FDAC
:10A6A0002AC0833079F03CF4813094F00E94D85075
:10A6B0008BE19EE00BC0843059F40E94D8508CEEA0
:10A6C0009DE004C00E94D85084E09EE00E94B250F9
:10A6D0002091000230E0A8EEB3E00F94BE20860E79
:10A6E000971EA81EB91E8092020890920308A0929D
:10A6F0000408B092050880911502882309F48EC0E1
:10A7000080918A0881118AC08091AF0A813021F03E
:10A710008091791682FF0CC6F89464990EC66091F8
:10A72000520A7091530A8091540A9091550A789474
:10A7300020E030E0A9010F94141A87FF6FC011E0E8
:10A7400010938A088091E40A811166C081E296E044
:10A750000E94F75284E08093A90A82E08093BE07AA
:10A7600081E09AE59093FE148093FD148EE490E0CE
:10A77000909300158093FF1487E08093F11482E892
:10A780008093F41484E890E0A0E0B0E08093F514A6
:10A790009093F614A093F714B093F8140E9419ED57
:10A7A00010930F120E9407B940E06CE57EE086E04E
:10A7B00096E20E9413B980E30E94A0508AE00E94B2
:10A7C000A0500E94FBB88091EC0760E0182719F0B8
:10A7D0008EED94E20DC08AE49EE00E94E3B880E32F
:10A7E0000E94A0508AE00E94A05060E08DE29EE0AE
:10A7F0000E94E3B888E39EE00E94B25080E30E948A
:10A80000A0508AE00E94A050112331F083E39EE023
:10A810009093CA088093C9080E94E26980914C0A0B
:10A82000843008F07FC20E947AFA4B015C0180916B
:10A830004C0A81111DC08091851190918611891B50
:10A840008F77B1F480916B0890916C08A0916D089E
:10A85000B0916E08A5019401281B390B4A0B5B0BC4
:10A86000DA01C901885E9340A109B109B7FF76C535
:10A8700060E6F62E80914C0A843008F036C1809153
:10A88000851190918611891B8F7709F42EC10E9442
:10A890000453AC0197FDEECF2091071230910812BE
:10A8A0008A3019F08D3009F0E8C010926A0821153D
:10A8B000310519F40F945303DDCFF901E65FF74F2B
:10A8C000108210920812109207120AE018E0F801A4
:10A8D0008191803211F48F01FACF8E3409F07AC061
:10A8E0000115110509F476C064E97FE0C8010F94F1
:10A8F00092196C01892B41F06EE470E0C801049656
:10A900000F945124009709F4C8014AE050E060E038
:10A9100070E001960F940A17609306087093070879
:10A9200080930808909309084090091250900A12E9
:10A9300060900B1270900C123FEF431A530A630A97
:10A94000730A641575058605970531F0CD2821F445
:10A9500060E081E69FE0C7C06AE270E0C8010F9442
:10A9600080249C01009709F1982F901BD12C9923EA
:10A9700039F09150F801E90FF11D8081D826F7CF09
:10A980004AE050E060E070E0C90101960F940A17B8
:10A990004D2C512C612C712C64157505860597057D
:10A9A00041F060E082E49FE09EC060E088E19FE0CB
:10A9B0009AC08091060890910708A0910808B0916C
:10A9C00009088093091290930A12A0930B12B09376
:10A9D0000C1212C08091791680FF0EC064E371E101
:10A9E000C8010F949219009709F47AC0FC01838181
:10A9F00080538A3008F474C080916F0281111CC0AA
:10AA000067E470E0C8010F9451240097A9F04AE070
:10AA100050E060E070E001960F940A176430710511
:10AA20008105910548F487E79EE00E94B25060E0FE
:10AA30008DE69EE00E949BFD80926B0890926C08D0
:10AA4000A0926D08B0926E0880910A088B3309F4C9
:10AA500011CF80914C0A843008F00CCF8091C80847
:10AA6000F89EC00111246AE078E08553974F0F9457
:10AA70005C2481E00E947ADDFDCE2F3531050CF09B
:10AA8000F9CE8C35C1F40E94045397FDF3CE20918A
:10AA90006A082111EFCE2091071230910812A90106
:10AAA0004F5F5F4F5093081240930712F901E65F22
:10AAB000F74F8083DFCE8B3321F481E080936A08E7
:10AAC000D9CE80916A088111D5CEC90101969093A3
:10AAD000081280930712F901E65FF74F4083CACE50
:10AAE00060E08EEE9EE00E9458B78091791682FF5A
:10AAF00019C180914C0A811102C010927008DD24A6
:10AB0000D394409175165091761660917716709196
:10AB100078168091711690917216A0917316B0916B
:10AB20007416481759076A077B0708F4D12C00E010
:10AB300010E0CC24C39430E6B32E44E6A42E59E6AC
:10AB4000952E80914C0A843008F0ECC0D110EAC0F8
:10AB5000809170088111E6C08091F0139091F113FB
:10AB6000A091F213B091F31380937516909376161B
:10AB7000A0937716B093781641E050E0BE016F5F66
:10AB80007F4F88EE93E10E945495019719F48981D3
:10AB900090E002C08FEF9FEFF82E40907516509016
:10ABA00076166090771670907816409171165091D5
:10ABB00072166091731670917416DD24D394441646
:10ABC00055066606770608F4D12C44165506660627
:10ABD0007706B0F4019609F461C02AE0F21609F490
:10ABE0006EC03DE0F31609F46AC043E2F41619F0B2
:10ABF0005AE3F5127CC080916F08811178C054C06F
:10AC00000E94E26988EE93E10E94DB9480917016C5
:10AC1000882339F1815080937016989EC0011124C9
:10AC200041E061E08751954F0E94067FE0917016E8
:10AC300064E0E69FF0011124EB51F54F4081518112
:10AC400062817381409375165093761660937716E0
:10AC50007093781688EE93E10E946F910E94BA7B00
:10AC600016C00E94A97B0E94476B0E9493670E94B6
:10AC700096FB6D3371058105910518F48FE99FE00E
:10AC800002C084EA9FE00E9481B7A0923D178091A4
:10AC9000791682FD0DC087EB9FE004C00E94D4505E
:10ACA00088EA9FE00E94B25073E2F71208C005C024
:10ACB00053E2F51260C300E010E0C09270081092F9
:10ACC0006F080115110519F40F9453030DC08091FD
:10ACD000C808B89E000D111D1124F801E553F74F67
:10ACE000108280E00E947ADD00E010E02ACF0F356C
:10ACF000110508F026CF8BE3F81203C0C0926F084D
:10AD000020CF80916F0881111CCF8091C808F80175
:10AD1000B89EE00DF11D1124E553F74FF0820F5F4F
:10AD20001F4F0FCF0E947AFA4B015C014091E80758
:10AD30005091E9076091EA077091EB0741155105C1
:10AD40006105710529F18091411390914213A09101
:10AD50004313B0914413840F951FA61FB71F95018D
:10AD60008401081B190B2A0B3B0B37FD11C00E94F5
:10AD7000D4506091540B7091550B8BEC9FE00E9466
:10AD8000C1508AE00E94A05080E090E00E9428EE2E
:10AD900040910102509102026091030270910402FD
:10ADA000411551056105710509F44EC090915F147C
:10ADB00080916014981759F00E947AFA60934113B9
:10ADC0007093421380934313909344133DC080913A
:10ADD000E40A811137C0E11035C080914113909190
:10ADE0004213A0914313B0914413840F951FA61FE3
:10ADF000B71FA5019401281B390B4A0B5B0B57FDAC
:10AE000021C08091810881111FC081E08093810859
:10AE10005F9A809149138E7F809349138A9A80911B
:10AE200049138D7F8093491380910801809581702B
:10AE300080930601809149138B7F809349130E9470
:10AE40000C5002C01092810880917D0890917E087C
:10AE5000A0917F08B0918008B501A401481B590B4F
:10AE60006A0B7B0B77FDAAC190915F1480916014EF
:10AE700020915C0210915D0298130EC060916E0BE0
:10AE8000269FB0011124660F672F661F770B7195FF
:10AE9000062F80916F0B17C08091601458E5859F35
:10AEA000C00111248856944FFC01EA5AFF4F0081DB
:10AEB000029FB0011124660F672F661F770B7195F3
:10AEC000062F31968081819FB0011124660F672F74
:10AED000661F770B7195162F002331F10E947AFAC5
:10AEE000C0907508D0907608E0907708F0907808C8
:10AEF000DC01CB01C114D104E104F10469F48C59E3
:10AF00009F4FAF4FBF4F8093750890937608A093E3
:10AF10007708B093780806C08C199D09AE09BF095F
:10AF2000B7FF0AC00FEF08C010927508109276089C
:10AF30001092770810927808602F70E089E00E94E4
:10AF400058F9112331F10E947AFAC0907908D09013
:10AF50007A08E0907B08F0907C08DC01CB01C114FA
:10AF6000D104E104F10469F48C599F4FAF4FBF4FF6
:10AF70008093790890937A08A0937B08B0937C081B
:10AF800006C08C199D09AE09BF09B7FF0AC01FEFA3
:10AF900008C01092790810927A0810927B081092DB
:10AFA0007C08612F70E087E00E9458F98091981228
:10AFB000882309F4F6C0E0901E02F0901F02009171
:10AFC0002002109121026091890B70918A0B6E5FB3
:10AFD0007F4F072E000C880B990B0F941B1A9701BB
:10AFE000A8010F94141A87FDDCC030906014212C46
:10AFF0001A821B821C8280915F14831509F467C03A
:10B00000832D90E068E5689FF001699FF00D1124A1
:10B01000E856F44F458956896789708D452B462B34
:10B02000472B89F4418D528D638D748D452B462BB2
:10B03000472B49F4458D568D678D70A1452B462BC6
:10B04000472B09F43FC078E5789F9001799F300D38
:10B050001124C9018856944F6C01FC0161817281F1
:10B06000838194810F94AC232B013C01F60161A1F3
:10B0700072A183A194A10F94191A6D837E838F838B
:10B080009887F60165A176A187A190A50F94191A5A
:10B090009B01AC016D817E818F8198850F94F82191
:10B0A000A30192010F947A1A3B016C01222D3A817F
:10B0B0004B815C810F945E23181624F4262C7A822F
:10B0C000CB82DC8281E0830D8F70382E94CF20916B
:10B0D0002202309123024091240250912502622DD8
:10B0E0007A818B819C810F947A1A9701A8010F9421
:10B0F000FE203B016C0120901A0230901B02409010
:10B100001C0250901D029B01AC01B701C8010F94B5
:10B110005E2318166CF09101A201B301C6010F94D1
:10B120005E2318161CF47101820102C073018601AE
:10B130004090710850907208609073087090740885
:10B140009701A801C301B2010F945E231816C4F43D
:10B1500020E037ED43EA5CE3B701C8010F947A1AA7
:10B160006B017C0128E431EE4AE75FE3C301B201E1
:10B170000F947A1AA70196010F94FE207B018C018F
:10B18000C701D8018093710890937208A093730847
:10B19000B0937408B701C8010F946A22CB010E94D2
:10B1A000E4DBF4E68F0E911CA11CB11C80927D089B
:10B1B00090927E08A0927F08B09280080F9453036B
:10B1C0008091AF0A813009F06EC00E947AFA6B015B
:10B1D0007C018091860890918708A0918808B091A1
:10B1E000890897018601081B190B2A0B3B0B37FDB9
:10B1F0003AC08090B00A9090B10AA090B20AB09084
:10B20000B30A0E9496FB6093B00A7093B10A8093D0
:10B21000B20A9093B30A0091AB081091AC08209148
:10B22000AD083091AE08081919092A093B09DC015B
:10B23000CB01800F911FA21FB31F8093AB08909387
:10B24000AC08A093AD08B093AE08D701C601805FEB
:10B25000984DAF4FBF4F8093860890938708A09377
:10B260008808B09389088091820890918308A09102
:10B270008408B0918508A7019601281B390B4A0B59
:10B280005B0B57FD10C030E8C30E3EEED31EE11C31
:10B29000F11CC0928208D0928308E0928408F09258
:10B2A00085080E946D670E94B4FC8091E70788239F
:10B2B00091F00E947AFA0091E3071091E40720913F
:10B2C000E5073091E607DC01CB01801B910BA20B57
:10B2D000B30BB7FF53C00E947AFA6B017C01209137
:10B2E000E207222309F468C08091DE079091DF070E
:10B2F000A091E007B091E107B701A601481B590BE7
:10B300006A0B7B0B77FD58C030E0A8EEB3E00F94DA
:10B31000BE20C60ED71EE81EF91EC092DE07D092D0
:10B32000DF07E092E007F092E1070E94827B44C0D1
:10B330008091E40A8111F0C971CA809163029091F1
:10B340006402A0916502B09166028093520A9093C4
:10B35000530AA093540AB093550AE1C989E99FE0C2
:10B360000E94B25080926B0890926C08A0926D0877
:10B37000B0926E087DCA10926F08A6CC0E947AFA2D
:10B380006B017C012091E70730E0A8EEB3E00F9459
:10B39000BE20C60ED71EE81EF91EC092E307D0924B
:10B3A000E407E092E507F092E60780E00E94EBD325
:10B3B0008AE00E94A0508FCF28960FB6F894DEBF87
:10B3C0000FBECDBFDF91CF911F910F91FF90EF90F6
:10B3D000DF90CF90BF90AF909F908F907F906F90B5
:10B3E0005F904F903F902F9008951F920F920FB64D
:10B3F0000F9211240F900FBE0F901F9018951F925F
:10B400000F920FB60F9211240BB60F920F931F934A
:10B410002F933F934F935F936F937F938F939F935C
:10B42000AF93BF93CF93DF93EF93FF930091861178
:10B43000D091851111E01D0F1F77C091C60090912A
:10B440000008492F092E000C550B660B770B413174
:10B45000510508F064C0FA018827E256FF4F8F4F6C
:10B460000D94F520CD3449F0CE34B9F481E006C016
:10B47000CA3338F0CD3409F043C082E0809300082D
:10B4800076C0C03308F073C0C03209F470C0CD324A
:10B49000B9F56DC0C13351F018F4C03289F567C0F9
:10B4A000C43331F0C83361F58BE0E8CF83E0E6CFF9
:10B4B00088E0E4CFC03321F0C13311F586E0DECF60
:10B4C00084E0DCCFC833E1F485E0D8CFC233C1F4E7
:10B4D00087E0D4CFC133A1F489E0D0CFC03381F469
:10B4E0008AE0CCCFC73361F48CE0C8CFC63341F4D7
:10B4F0008DE0C4CFC032D9F1C33511F48EE0BECF98
:10B5000080E1BCCF80ED8C0F8A3088F59FE090936E
:10B5100000088093FF072BC0CA3049F526C0CA3007
:10B5200031F580915F15882301F1973089F03CF463
:10B530009530D9F41092140210923C1716C09A302C
:10B5400059F09F3091F48091FF070E943FB90DC0E0
:10B5500081E08093F71C09C00E949D6B0E94E26904
:10B560008EEF0E9456D10E94C4D11092000801179C
:10B5700031F0ED2FF0E0EB57FE4EC283D12FD09388
:10B580008511FF91EF91DF91CF91BF91AF919F9185
:10B590008F917F916F915F914F913F912F911F916B
:10B5A0000F910F900BBE0F900FBE0F901F9018952C
:10B5B0008EBD0DB407FEFDCF08958FEF8EBD0DB487
:10B5C00007FEFDCF8EB50895909164009B7F909308
:10B5D0006400982F906A96959CBD80FD03C091E011
:10B5E000863009F490E09DBD08952F923F924F92CE
:10B5F0005F926F927F928F929F92AF92BF92CF9203
:10B60000DF92EF92FF920F931F93CF93DF93CDB70B
:10B61000DEB72F970FB6F894DEBF0FBECDBF8FEF0A
:10B620009FEF90938900809388001AE0D12E1F86A7
:10B630001E8678948091990A90919A0AA0919B0A0B
:10B64000B0919C0A892B8A2B8B2B09F0D5C1809154
:10B65000DA1C8823D1F01092DA1C8091D81C9091CA
:10B66000D91C892B91F010925A0A1092D91C109271
:10B67000D81C90915F1480916014981731F08091DC
:10B6800060148F5F8F70809360148091D81C9091AC
:10B69000D91C892B09F4B0C10091950A1091960A22
:10B6A0002091970A3091980A8091910A9091920A7C
:10B6B000A091930AB091940A4091880A50E060E00A
:10B6C00070E0801B910BA20BB30B481759076A0758
:10B6D0007B0710F4DB01CA01482F800F911FA21FC6
:10B6E000B31F8093950A9093960AA093970AB093FC
:10B6F000980A80918400909185004E9680905F0A10
:10B700009090600AA090610AB090620A00916F0A5E
:10B710001091700A2091710A3091720A080D191D5A
:10B720002A1D3B1D00936F0A1093700A2093710A23
:10B730003093720A37FD1CC0889A00914E0A002E81
:10B74000000C110B220B330B8090E71C9090E81C2F
:10B75000A090E91CB090EA1C080D191D2A1D3B1D84
:10B760000093E71C1093E81C2093E91C3093EA1C1B
:10B770008090630A9090640AA090650AB090660A6F
:10B780000091730A1091740A2091750A3091760A1B
:10B79000080D191D2A1D3B1D0093730A1093740A8E
:10B7A0002093750A3093760A37FD1CC08E9A00915B
:10B7B0004F0A002E000C110B220B330B8090EB1C58
:10B7C0009090EC1CA090ED1CB090EE1C080D191D83
:10B7D0002A1D3B1D0093EB1C1093EC1C2093ED1CC9
:10B7E0003093EE1C8090670A9090680AA090690AD6
:10B7F000B0906A0A0091770A1091780A2091790A2C
:10B8000030917A0A080D191D2A1D3B1D0093770AF5
:10B810001093780A2093790A30937A0A37FD21C071
:10B8200020910B0120952870209309010091500A66
:10B83000002E000C110B220B330B8090EF1C90900C
:10B84000F01CA090F11CB090F21C080D191D2A1DCF
:10B850003B1D0093EF1C1093F01C2093F11C3093C0
:10B86000F21C80906B0A90906C0AA0906D0AB090C8
:10B870006E0A00917B0A10917C0A20917D0A30911A
:10B880007E0A080D191D2A1D3B1D00937B0A10938B
:10B890007C0A20937D0A30937E0A37FD1CC0149ADF
:10B8A0000091510A002E000C110B220B330B8090DB
:10B8B000F31C9090F41CA090F51CB090F61C080DA1
:10B8C000191D2A1D3B1D0093F31C1093F41C20939B
:10B8D000F51C3093F61C20918400309185002817C8
:10B8E0003907C8F300916F0A1091700A2091710A0C
:10B8F0003091720A37FD15C080905B0A90905C0A07
:10B90000A0905D0AB0905E0A081919092A093B093E
:10B9100000936F0A1093700A2093710A3093720A91
:10B9200088980091730A1091740A2091750A3091D9
:10B93000760A37FD15C080905B0A90905C0AA09053
:10B940005D0AB0905E0A081919092A093B0900939B
:10B95000730A1093740A2093750A3093760A8E98AE
:10B960000091770A1091780A2091790A30917A0A29
:10B9700037FD19C080905B0A90905C0AA0905D0A28
:10B98000B0905E0A081919092A093B090093770A41
:10B990001093780A2093790A30937A0A20910B0148
:10B9A00028702093090100917B0A10917C0A209154
:10B9B0007D0A30917E0A37FD15C080905B0A909019
:10B9C0005C0AA0905D0AB0905E0A081919092A095C
:10B9D0003B0900937B0A10937C0A20937D0A3093E5
:10B9E0007E0A1498415041F02091840030918500E6
:10B9F00028173907C8F381CE8091990A90919A0A45
:10BA0000A0919B0AB0919C0A892B8A2B8B2B11F059
:10BA10000C942363E091D81CF091D91C309711F459
:10BA20000C94AA648091950A9091960AA091970A25
:10BA3000B091980A4091910A5091920A6091930AAC
:10BA40007091940A84179507A607B70708F46EC08B
:10BA500080911502882309F44EC085899689A789AB
:10BA6000B08D892B8A2B8B2BA1F4818D928DA38D88
:10BA7000B48D892B8A2B8B2B61F4858D968DA78DA8
:10BA8000B0A1892B8A2B8B2B21F48091E40A882387
:10BA900091F161A172A183A194A18090520A90902A
:10BAA000530AA090540AB090550AEB5BFF4F2081D7
:10BAB00023FF07C090958095709561957F4F8F4FBC
:10BAC0009F4F0F941B1A20917C0B30917D0B40915E
:10BAD0007E0B50917F0B0F947A1A9B01AC01C5012C
:10BAE000B4010F94FD206093520A7093530A80931F
:10BAF000540A9093550A10925A0A1092D91C109227
:10BB0000D81C90915F1480916014981711F40C94D4
:10BB1000AA64809160148F5F8F7080936014B0ED81
:10BB20004B2EB7E05B2E612C712CE7C340918D0A40
:10BB300050918E0A60918F0A7091900A48175907A8
:10BB40006A077B0708F4A5C18090890A90908A0A49
:10BB5000A0908B0AB0908C0A85A996A9A7A9B0AD30
:10BB600088169906AA06BB0608F077C181149104CD
:10BB7000A104B10449F48091560A9091570AA0910A
:10BB8000580AB091590A65C1B0E0AC2D882D392D05
:10BB90002A2DF981EA817B816C815D814E819F81B3
:10BBA0005091B40A589F712D66274091B50A489F5D
:10BBB000700D611D1090B60A189E600D539F700D98
:10BBC000611D439F600D529F600DF72FE62FF79F79
:10BBD000512D44279927F69F500D411D9B1FE79F2C
:10BBE000500D411D9B1FE69F400D911DF42FE92F25
:10BBF000F79FA12D44279927F69FA00D411D9B1F5C
:10BC0000E79FA00D411D9B1FE69F400D911DF42F46
:10BC1000E92F55278091560A3091570A2091580AEA
:10BC20000090FB070B2A09F484C04091F7074F9F4F
:10BC300051198B0B3B0B2B0B9091F8079F9F5019C1
:10BC400081093B0B2B0BA091F907AF9F801931099C
:10BC50002B0B4E9F501981093B0B2B0B9E9F80197C
:10BC600031092B0BAE9F30192109F79FA12D4427D5
:10BC70009927F69FA00D411D9B1FE79FA00D411D19
:10BC80009B1FE69F400D911DF42FE92F4091F30774
:10BC90004F9F510D8B1F3B1F2B1F9091F4079F9FB0
:10BCA000500D811D3B1F2B1FA091F507AF9F800DED
:10BCB000311D2B1F4E9F500D811D3B1F2B1F9E9F23
:10BCC000800D311D2B1FAE9F300D211DF79FA12D23
:10BCD00044279927F69FA00D411D9B1FE79FA00DAC
:10BCE000411D9B1FE69F400D911DF42FE92F4091B0
:10BCF000EF074F9F51198B0B3B0B2B0B9091F007CC
:10BD00009F9F501981093B0B2B0BA091F107AF9F0F
:10BD1000801931092B0B4E9F501981093B0B2B0BBE
:10BD20009E9F801931092B0BAE9F301921090C946D
:10BD30001B5F4091F7074F9F510D8B1F3B1F2B1F20
:10BD40009091F8079F9F500D811D3B1F2B1FA091C5
:10BD5000F907AF9F800D311D2B1F4E9F500D811D88
:10BD60003B1F2B1F9E9F800D311D2B1FAE9F300D43
:10BD7000211DF79FA12D44279927F69FA00D411D56
:10BD80009B1FE79FA00D411D9B1FE69F400D911D2E
:10BD9000F42FE92F4091F3074F9F51198B0B3B0B69
:10BDA0002B0B9091F4079F9F501981093B0B2B0B94
:10BDB000A091F507AF9F801931092B0B4E9F5019A9
:10BDC00081093B0B2B0B9E9F801931092B0BAE9FDA
:10BDD00030192109F79FA12D44279927F69FA00D1F
:10BDE000411D9B1FE79FA00D411D9B1FE69F400D1E
:10BDF000911DF42FE92F4091EF074F9F510D8B1F9D
:10BE00003B1F2B1F9091F0079F9F500D811D3B1FE3
:10BE10002B1FA091F107AF9F800D311D2B1F4E9F4F
:10BE2000500D811D3B1F2B1F9E9F800D311D2B1F11
:10BE3000AE9F300D211D1124CA2EF983EA837B8326
:10BE40006C835D834E839F8390E0932BA0E0B0E0F2
:10BE5000A22B29E539E111E011C081A992A9A3A97A
:10BE6000B4A9F7CFB695A79597958795110F2C5F35
:10BE70003F4F49E12537340709F43BC4F9014591A7
:10BE8000559165917491481759076A077B0750F3DC
:10BE900030C44091840A5091850A6091860A70915D
:10BEA000870A481759076A077B0708F0B9C18091CC
:10BEB000830A81111FC0DF01AF5BBF4FED90FD9082
:10BEC0000D911C9113971D962D913D914D915C9173
:10BED00061A972A983A994A90E942E6551E050938B
:10BEE000830AE091D81CF091D91C81A892A8A3A83C
:10BEF000B4A887C180917F0A9091800AA091810A9D
:10BF0000B091820A41AD52AD63AD74AD841795070F
:10BF1000A607B70708F06FC10097A105B10549F45E
:10BF20008090560A9090570AA090580AB090590AEB
:10BF300068C130E04885882E292F8A2FE9857A85C7
:10BF40006B855C859D859091B40A989D612D5527E0
:10BF50002090B50A289C600D511D1090B60A189CBF
:10BF6000500D929F600D511D229E500D989F500DB7
:10BF7000E62F752FE69F912D22243324E59F900D07
:10BF8000211C331E769F900D211C331E759F200CA3
:10BF9000311CE22D732DE69F412D22243324E59F91
:10BFA000400D211C331E769F400D211C331E759FB2
:10BFB000200C311CE22D732D99278090560A209178
:10BFC000570A8091580A0090FB07032A09F484C09D
:10BFD0002090F7072E9E9119830A230B830B309034
:10BFE000F8073E9E90198108230B830B4091F907B7
:10BFF0004E9F80182109830B279E90198108230BDF
:10C00000830B379E80182109830B479F20198109D4
:10C01000E69F412D22243324E59F400D211C331E31
:10C02000769F400D211C331E759F200C311CE22D84
:10C03000732D2090F3072E9E910D831E231F831FC7
:10C040003090F4073E9E900D811C231F831F40916A
:10C05000F5074E9F800C211D831F279E900D811C8C
:10C06000231F831F379E800C211D831F479F200D98
:10C07000811DE69F412D22243324E59F400D211C84
:10C08000331E769F400D211C331E759F200C311CE2
:10C09000E22D732D2090EF072E9E9119830A230B1A
:10C0A000830B3090F0073E9E90198108230B830B81
:10C0B0004091F1074E9F80182109830B279E90190C
:10C0C0008108230B830B379E80182109830B479F20
:10C0D000201981090C94EE602090F7072E9E910D97
:10C0E000831E231F831F3090F8073E9E900D811CF6
:10C0F000231F831F4091F9074E9F800C211D831F32
:10C10000279E900D811C231F831F379E800C211DAD
:10C11000831F479F200D811DE69F412D222433243C
:10C12000E59F400D211C331E769F400D211C331EC0
:10C13000759F200C311CE22D732D2090F3072E9E4D
:10C140009119830A230B830B3090F4073E9E9019BC
:10C150008108230B830B4091F5074E9F801821091E
:10C16000830B279E90198108230B830B379E801821
:10C170002109830B479F20198109E69F412D222425
:10C180003324E59F400D211C331E769F400D211C5A
:10C19000331E759F200C311CE22D732D2090EF076C
:10C1A0002E9E910D831E231F831F3090F0073E9E0D
:10C1B000900D811C231F831F4091F1074E9F800C1F
:10C1C000211D831F279E900D811C231F831F379ED7
:10C1D000800C211D831F479F200D811D112448873E
:10C1E000E9877A876B875C879D87912C922AA12C9F
:10C1F000B12CA82A06C0E25BFF4F80809180A2800C
:10C20000B38089E599E121E0FC0145915591659163
:10C210007491481559056A057B0508F4CDC2D7C24B
:10C220008091160290911702A0911802B091190204
:10C23000B7FF5BC0EA5BFF4F80809180A280B38034
:10C2400089E599E121E0FC01459155916591749151
:10C25000481559056A057B0550F4B694A794979440
:10C260008794220F0496A9E185379A0761F72093F6
:10C27000880AB0E28B169104A104B10408F43BC310
:10C2800020E2821A9108A108B108811438E09306CF
:10C29000A104B10408F40BC344E0949EC00111242E
:10C2A000875A9A4EFC01329625913491782D662753
:10C2B000739FA001729F410D561F0694461F561F83
:10C2C000112460E070E0FC0125913491C901A0E0E7
:10C2D000B0E0841B950BA60BB70B809316029093CE
:10C2E0001702A0931802B0931902409016025090C2
:10C2F000170260901802709019028091D81C9091DA
:10C30000D91C892B09F097C10E94C2659093D91C52
:10C310008093D81C892B09F48EC1E091D81CF09130
:10C32000D91C808183FF3EC0858D968DA78DB0A1DD
:10C33000418D528D638D748D058916892789308DC5
:10C340000093E71C1093E81C2093E91C3093EA1C2F
:10C350004093EB1C5093EC1C6093ED1C7093EE1C0F
:10C360008093EF1C9093F01CA093F11CB093F21CEF
:10C3700081A192A1A3A1B4A18093F31C9093F41C7A
:10C38000A093F51CB093F61C90915F1480916014FB
:10C39000981709F4B9CF809160148F5F8F708093E4
:10C3A0006014B2CF058916892789308D81E0011587
:10C3B00011052105310509F480E0818C928CA38C54
:10C3C000B48C81149104A104B10409F08260458DFC
:10C3D000568D678D70A1411551056105710509F0F4
:10C3E000846080935A0A10927F0A1092800A1092F9
:10C3F000810A1092820A1092890A10928A0A109277
:10C400008B0A10928C0A85A196A1A7A1B0A5809352
:10C41000910A9093920AA093930AB093940A4424A9
:10C4200055243201481A590A6A0A7B0A40926F0A57
:10C430005092700A6092710A7092720A4092730A66
:10C440005092740A6092750A7092760A4092770A46
:10C450005092780A6092790A70927A0A40927B0A26
:10C4600050927C0A60927D0A70927E0A41A052A08E
:10C4700063A074A0440C551C661C771C000F111F90
:10C48000221F331F00935F0A1093600A2093610AF2
:10C490003093620A880C991CAA1CBB1C8092630A08
:10C4A0009092640AA092650AB092660A440F551FE2
:10C4B000661F771F4093670A5093680A6093690A62
:10C4C00070936A0A40926B0A50926C0A60926D0AED
:10C4D00070926E0A880F991FAA1FBB1F80935B0A78
:10C4E00090935C0AA0935D0AB0935E0A1092950A3D
:10C4F0001092960A1092970A1092980A81A592A516
:10C50000A3A5B4A580938D0A90938E0AA0938F0A59
:10C51000B093900A85A596A5A7A5B0A98093840A93
:10C520009093850AA093860AB093870AEB5BFF4F2E
:10C5300080819091B908891721F08093B9080E94F1
:10C5400080650E94FAE68FEF9FEFDC018093160270
:10C5500090931702A0931802B0931902E091D81C8F
:10C56000F091D91CDF01DD96ED90FD900D911C91AD
:10C5700021A932A943A954A9E65BFF4F60817181CB
:10C58000828193810E942E651092830AE091D81CCB
:10C59000F091D91CE65BFF4F80809180A280B38030
:10C5A00089E599E121E0FC014591559165917491EE
:10C5B000481559056A057B0558F4B694A7949794D5
:10C5C0008794220F049645E759E14817590759F710
:10C5D0002093880A50E285169104A104B10408F45E
:10C5E000B3C190E2891A9108A108B1088114A8E0AA
:10C5F0009A06A104B10408F484C1B4E09B9EC00172
:10C600001124875A9A4EFC01329625913491782D47
:10C610006627739FA001729F410D561F0694461F07
:10C62000561F1124FC0145905490612C712C441A22
:10C63000550A610871084092990A50929A0A6092CC
:10C640009B0A70929C0A8091990A90919A0AA091F3
:10C650009B0AB0919C0AAC01BD01009721E0A207A2
:10C66000B10520F04FEF5FEF60E070E0841B950BA9
:10C67000A60BB70B8093990A90939A0AA0939B0AF2
:10C68000B0939C0AF8948091840090918500409624
:10C69000DA94DD2061F0AE85BF85A40FB51FBF879A
:10C6A000AE87A817B90710F40C94195B02C09F87D6
:10C6B0008E872E853F85309389002093880078945B
:10C6C0002F960FB6F894DEBF0FBECDBFDF91CF918E
:10C6D0001F910F91FF90EF90DF90CF90BF90AF90A0
:10C6E0009F908F907F906F905F904F903F902F9092
:10C6F00008951093880A80329105A105B10508F4C8
:10C7000056C08097A109B109811528E09207A105BB
:10C71000B105F0F044E0949F90011124275A3A4E5D
:10C72000F901329645915491EE27859FB001849F7F
:10C73000610D7E1F06946E1F7E1F1124F901459026
:10C740005490612C712C461A570A6108710822C056
:10C75000AC01BD017695679557954795FA01EC7F39
:10C76000AF01475A5E4EFA0125913491FA01329693
:10C77000659174918770869FA001879F500D112449
:10C78000A3E056954795AA95E1F72901441A550A61
:10C79000612C712C840C951CA61CB71C8092890AF4
:10C7A00090928A0AA0928B0AB0928C0AA6CD80E25F
:10C7B00090E0A0E0B0E0A5CFB694A79497948794BA
:10C7C000220F049659E18537950709F01DCD209376
:10C7D000880A70E287169104A104B10408F461C0CC
:10C7E00070E2871A9108A108B108811488E09806C0
:10C7F000A104B104F8F0A4E09A9EC0011124875A64
:10C800009A4EFC01329625913491B82D6627B39F3C
:10C81000A001B29F410D561F0694461F561F1124BA
:10C82000FC0145905490612C712C441A550A610802
:10C83000710822C0D501C401B695A7959795879533
:10C84000FC01EC7FCF01875A9E4EFC01459054902D
:10C85000FC01329625913491482D4770429FC001CA
:10C86000439F900D1124E3E096958795EA95E1F7B3
:10C87000481A590A612C712C80917F0A9091800A84
:10C88000A091810AB091820A840D951DA61DB71D45
:10C8900080937F0A9093800AA093810AB093820AC2
:10C8A0002CCD60E2862E912CA12CB12C99CFD501F4
:10C8B000C401B695A79597958795FC01EC7FCF01AC
:10C8C000875A9E4EFC0125913491FC013296459188
:10C8D0005491682D6770649FC001659F900D11246D
:10C8E00063E0969587956A95E1F7281B390BC90196
:10C8F000A0E0B0E0F2CC40E2842E912CA12CB12C2F
:10C90000BFCCD501C401B695A79597958795FC0135
:10C91000EC7FCF01875A9E4EFC0145905490FC015C
:10C92000329625913491482D4770429FC001439F14
:10C93000900D1124A3E096958795AA95E1F7481AE2
:10C94000590A612C712C77CE90E2892E912CA12C62
:10C95000B12C47CE80ED482E87E0582E612C712CEB
:10C96000D3CCCF93DF9380915F1490916014891B97
:10C970008F708F3021F480E00E941853F4CF8091A3
:10C980005F148F5F8F70A0915F1498E59A9FD0011C
:10C990001124FD01E856F44FEF0119929A95E9F739
:10C9A00098E09083A355B44F90E1E5E7F4E101905E
:10C9B0000D929A95E1F720915F14909160142913DC
:10C9C00003C094E690935C1480935F1480916F0091
:10C9D000826080936F00DF91CF9108950F930FB71E
:10C9E0000F9300916E000F930B7F00936E000091E8
:10C9F0006F000D7F00936F000F930BB70F930CB771
:10CA00000F921F922F933F934F935F936F937F9358
:10CA10008F939F93AF93BF93EF93FF9311240E9443
:10CA2000F55AFF91EF91BF91AF919F918F917F91B7
:10CA30006F915F914F913F912F911F900F900CBF7D
:10CA40000F910BBF0F910260F89400936F000F914C
:10CA500000936E000F910FBF0F911895EF92FF9208
:10CA60000F931F93E092B40AF092B50A0093B60AAE
:10CA70001093B70A6093560A7093570A8093580A26
:10CA80009FEFFF27621B730B840B30F4809570952A
:10CA90006195790B890B99279093FB07A6E06A9F14
:10CAA0000092EF07512DEE277A9F500DE11D8A9FCE
:10CAB000E00D5093F007E093F107AFE06A9F00921A
:10CAC000F307512DEE277A9F500DE11D8A9FE00D4F
:10CAD0005093F407E093F507AAE06A9F0092F707E6
:10CAE000512DEE277A9F500DE11D8A9FE00D509346
:10CAF000F807E093F9071F910F91FF90EF900895C9
:10CB00000000000000008091B90880FF03C08998F0
:10CB10008FEF02C0899A81E080934E0A8091B90814
:10CB2000869580FF03C08F9A8FEF02C08F9881E0B7
:10CB300080934F0A8091B9088695869580FF08C03A
:10CB400080910B0180958270809309018FEF06C060
:10CB500080910B0182708093090181E08093500ADB
:10CB60008091B90886958695869580FF03C01698B2
:10CB70008FEF02C0169A81E08093510A00000000F6
:10CB80000000089580915F1490916014891B8F704C
:10CB900019F480E090E0089590915C14992351F08D
:10CBA000833030F48FEF890F19F080935C14F1CF4C
:10CBB00010925C14E091601488E5E89FF001112464
:10CBC000E856F44F808180FDE4CF809160148F5F40
:10CBD0008F7080935D149091601480915E1498130F
:10CBE00004C080915D1480935E14CF010895CF92AC
:10CBF000DF92EF92FF92CF93DF93CDB7DEB7289706
:10CC00000FB6F894DEBF0FBECDBF20E030E040EAA3
:10CC100050E46091461770914717809148179091A2
:10CC200049170F94141A8823E9F01D821E821F826F
:10CC30001886C12CD12C80EAE82E80E4F82EC98217
:10CC4000DA82EB82FC82BE016B5F7F4FCE010196E0
:10CC50000E9411D1C0924617D0924717E092481710
:10CC6000F092491728960FB6F894DEBF0FBECDBFDD
:10CC7000DF91CF91FF90EF90DF90CF900895BF921A
:10CC8000CF92DF92EF92FF920F931F93CF93DF9398
:10CC9000CDB7DEB728970FB6F894DEBF0FBECDBF75
:10CCA0009091BA08981709F47DC0B82E882309F42A
:10CCB00054C080E090E0A0E2B1E48D839E83AF8316
:10CCC000B887C090EE16D090EF16E090F016F09076
:10CCD000F11620E030E0A901C701B6010F94141A43
:10CCE00087FF0CC0A701960160E070E080E291E44C
:10CCF0000F94FD206D837E838F83988720E030E042
:10CD000048EC53E46D817E818F8198850F945E237A
:10CD1000181644F480E090E0A8ECB3E48D839E8381
:10CD2000AF83B8872D813E814F815885609146172A
:10CD30007091471780914817909149170F94141AD2
:10CD400087FF0BC019821A821B821C82BE016F5F93
:10CD50007F4FCE0105960E9411D160913E177091D0
:10CD60003F178091401790914117209142173091C1
:10CD70004317409144175091451719821A821B821C
:10CD80001C82E0904617F0904717009148171091C9
:10CD90004917FE0131966F010E942ED0B092BA0859
:10CDA0000E948AE780E028960FB6F894DEBF0FBE97
:10CDB000CDBFDF91CF911F910F91FF90EF90DF904A
:10CDC000CF90BF900895CF93DF93C091AF0A8BE7C8
:10CDD00096E00E94F7528091AA0A873009F445C074
:10CDE00083E08093A90A81E08093260280E190E0AD
:10CDF0009093FE148093FD1485E08093F114D2E8A3
:10CE0000D093F41484E190E1A0E0B0E08093F514B5
:10CE10009093F614A093F714B093F8140E9419EDB0
:10CE200061E070E080E090E00E945CAE81E09AE515
:10CE30009093FE148093FD1485E390E09093001589
:10CE40008093FF1487E08093F114D093F41484E866
:10CE500090E0A0E0B0E08093F5149093F614A093D6
:10CE6000F714B093F8140E9419EDC13081F1C2306B
:10CE700059F40E9496FB6093A10A7093A20A8093D2
:10CE8000A30A9093A40A02C00E94CAFB81E0809387
:10CE9000AF0A0E947AFA60939D0A70939E0A80936B
:10CEA0009F0A9093A00AC230A1F08091A7089091A8
:10CEB000A80801969093A8088093A7081092B00A3A
:10CEC0001092B10A1092B20A1092B30A02C080E026
:10CED00001C081E0DF91CF910895CF93DF9300D01F
:10CEE0001F92CDB7DEB78091A6088823A9F083E30F
:10CEF00090E09C838B831A8219829E012F5F3F4FA3
:10CF000040E150E067EA78E0CE0103960E94DC50F1
:10CF100083E996E00E94F7520F900F900F900F90C8
:10CF2000DF91CF910895CF92DF92EF92FF920F930E
:10CF30001F938091AF0A8150823010F080E09EC034
:10CF400083EB96E00E94F7528091AA0A8330C9F1E0
:10CF500040E060E070E0CB010E9449FE41E060E00B
:10CF600070E0CB010E9449FE81E08093050210929F
:10CF7000A80A21E030E03093A70A2093A60A809304
:10CF8000260281E09AE59093FE148093FD148DE2D1
:10CF900090E0909300158093FF1487E08093F11444
:10CFA00082E88093F41484E890E0A0E0B0E08093FD
:10CFB000F5149093F614A093F714B093F8140E940C
:10CFC00019ED1092AF0A0E947AFA6093AB0A70933F
:10CFD000AC0A8093AD0A9093AE0A8091A908909113
:10CFE000AA0801969093AA088093A908C090B00A55
:10CFF000D090B10AE090B20AF090B30A0E9496FB7A
:10D000006093B00A7093B10A8093B20A9093B30A06
:10D010000091AB081091AC082091AD083091AE089A
:10D020000C191D092E093F09DC01CB01800F911F4E
:10D03000A21FB31F8093AB089093AC08A093AD08D8
:10D04000B093AE080E9496FB0091AF081091B00813
:10D050002091B1083091B208061717072807390741
:10D0600050F40E9496FB6093AF087093B0088093D1
:10D07000B1089093B2080E946D6781E01F910F91F3
:10D08000FF90EF90DF90CF900895CF93DF9300D083
:10D090001F921F92CDB7DEB781E08093A608E7EA22
:10D0A000F8E080E1DF011D928A95E9F70E946D6743
:10D0B00086E18D8382E390E09C838B831A821982C0
:10D0C0009E012F5F3F4F41E050E0BE016B5F7F4FFD
:10D0D000CE0103960E94DC500F900F900F900F909E
:10D0E0000F90DF91CF9108959F92AF92BF92CF9210
:10D0F000DF92EF92FF920F931F93CF93DF9300D0B5
:10D100001F921F92CDB7DEB7E9E7F9E10027BB27F1
:10D11000462F572FA82FAA2341F4A52F542FB85FCD
:10D12000AA2319F4A52F5527B85FA03138F45295DA
:10D13000A295452F4F70507FA42BBC5FA03428F4DC
:10D14000550FAA1F550FAA1FBE5FA03818F4550F20
:10D15000AA1FB395550FAA1FEA0FF01F449151E083
:10D16000AA27B85081F1C8F0B0FF02C0440F551F84
:10D17000B1FF04C0440F551F440F551FB2FF06C036
:10D1800052954295142F1F70407F512BB3FF1BC047
:10D19000A52F542F44270C94E368B195B0FF02C02B
:10D1A00055954795B1FF04C05595479555954795B9
:10D1B000B2FF05C05295407F4295452B5F70B3FF8B
:10D1C00002C0452F5527DD24CC24BB24B2E0649F48
:10D1D000D018C108B00AB00B749FC018B108B00BCA
:10D1E000849FB018B109659FC018B108B00B759F36
:10D1F000B018B109859FB0196A9FB018B1097A9F1C
:10D20000B0194D9DA12C99249927332722275D9D84
:10D21000A00C911C901F301F201FAD9D900C911DE4
:10D22000301F201F4C9DA00C911C901F301F201FF1
:10D230005C9D900C911D301F201FAC9D900D311DE9
:10D24000201F4B9D900C911D301F201F5B9D900D4A
:10D25000311D201FAB9D300D211D4B9F900D311DA9
:10D26000201F5B9F300D211DAB9F200DB1E0BB2423
:10D27000CC24DD24699FD018C108B00AB00B799F77
:10D28000C018B108B00B899FB018B109639FC018CE
:10D29000B108B00B739FB018B109839FB019629F9A
:10D2A000B018B109729FB019D61AC70AB80A20F08F
:10D2B000B1E09B0F301F201F1124692F70E0732BEA
:10D2C000CB01A0E0B0E0BC01CD01822B0F900F900C
:10D2D0000F900F900F90DF91CF911F910F91FF90C2
:10D2E000EF90DF90CF90BF90AF909F900895CF9236
:10D2F000DF92EF92FF920F931F93CF93DF93CBE1D7
:10D30000D1E10AE51BE0C12CD12C7601C3946991CF
:10D310007991899199910F94191A288939894A89A3
:10D320005B890F947A1A0F947122F80161937193BB
:10D33000819391938F01C616D706E806F90610F47B
:10D340006B017C01F1E1CB32DF0709F76FEF7FEF73
:10D35000CB01A70196010F946A2020936A0B3093AA
:10D360006B0B40936C0B50936D0BDF91CF911F9122
:10D370000F91FF90EF90DF90CF9008950F931F9340
:10D38000CF93DF930FE211E1C0E7DBE0F8012191D9
:10D390003191419151918F0160E070E080E89FE30D
:10D3A0000F94F8216993799389939993FBE0C0389E
:10D3B000DF0761F70E946990DF91CF911F910F9174
:10D3C0000C94776990915F1480916014981306C053
:10D3D0008091181190911911892B21F080E00E9401
:10D3E0001853F0CF089520913B1130913C1140919A
:10D3F0003D1150913E11FC016081718182819381C8
:10D400000F947A1A0F946B23609381147093821493
:10D41000809383149093841490915F14809160148E
:10D4200098130C94B1640E94E26980916F00982F68
:10D43000927081FF05C080916F008D7F80936F0097
:10D4400040918114509182146091831470918414DE
:10D450004093F31C5093F41C6093F51C7093F61CDE
:10D46000992329F080916F00826080936F00089566
:10D470004F925F926F927F928F929F92AF92BF92E4
:10D48000CF92DF92EF92FF920F931F93CF93DF9390
:10D49000EC018B015A01F90120913B1130913C11B3
:10D4A00040913D1150913E11608171818281938143
:10D4B0000F947A1A0F946B236B017C012091371122
:10D4C000309138114091391150913A11F501608134
:10D4D0007181828193810F947A1A0F946B234B018F
:10D4E0005C012091331130913411409135115091EC
:10D4F0003611F80160817181828193810F947A1ACB
:10D500000F946B232B013C0120912F11309130118E
:10D510004091311150913211688179818A819B81CA
:10D520000F947A1A0F946B2360937514709376148A
:10D5300080937714909378144092791450927A14CF
:10D5400060927B1470927C1480927D1490927E1471
:10D55000A0927F14B0928014C0928114D092821451
:10D56000E0928314F092841490915F14809160147F
:10D57000981791F0DF91CF911F910F91FF90EF904D
:10D58000DF90CF90BF90AF909F908F907F906F90E3
:10D590005F904F900C94B1640E94E26980916F009B
:10D5A000982F927081FF05C080916F008D7F8093CE
:10D5B0006F0040917D1450917E1460917F147091A2
:10D5C00080140091791410917A1420917B14309179
:10D5D0007C14C0907514D0907614E0907714F0907D
:10D5E0007814C092E71CD092E81CE092E91CF092FB
:10D5F000EA1C0093EB1C1093EC1C2093ED1C309361
:10D60000EE1C4093EF1C5093F01C6093F11C709340
:10D61000F21C409181145091821460918314709196
:10D6200084144093F31C5093F41C6093F51C709386
:10D63000F61C992329F080916F00826080936F001F
:10D64000DF91CF911F910F91FF90EF90DF90CF90DE
:10D65000BF90AF909F908F907F906F905F904F9012
:10D660000895CF93DF93C82F0F94950724E0C29FAE
:10D67000E0011124C059D44F0F941B1A288139811D
:10D680004A815B810F947A1ADF91CF91089590912E
:10D690005F1480916014981306C0809118119091C6
:10D6A0001911892B21F080E00E941853F0CF5F9A66
:10D6B000809149138E7F809349138A9A80914913F0
:10D6C0008D7F8093491380910801809581708093AC
:10D6D0000601809149138B7F809349130C940C5061
:10D6E000CF93DF9390916F00292F227091FF05C097
:10D6F00090916F009D7F90936F0094E0899FA001AF
:10D700001124FA01E552F34E608171818281938187
:10D71000222329F020916F00226020936F00EA01FC
:10D72000C059D44F0F941B1A288139814A815B81DB
:10D730000F947A1ADF91CF91089580916F00982FFE
:10D74000927081FF05C080916F008D7F80936F0084
:10D750008091601480935F1480935E1480935D14B5
:10D7600084E680935C1428EE33E030931911209303
:10D770001811992329F080916F00826080936F00C7
:10D7800081E08093DA1C0895CF92DF92EF92FF92AE
:10D79000CF93DF9320915617222331F1EC010896A5
:10D7A0000E9468CB6B017C0120E030E0A9010F945E
:10D7B000141A882361F0CE010E9443BD9B01AC0185
:10D7C000C701B6010F947A1A9B01AC0103C020E097
:10D7D00030E0A901688579858A859B850F94FD20B5
:10D7E000688779878A879B87DF91CF91FF90EF9039
:10D7F000DF90CF900895CF92DF92EF92FF92CF9378
:10D80000DF9320915617222331F1EC0108960E94F4
:10D8100068CB6B017C0120E030E0A9010F94141A61
:10D82000882361F0CE010E9443BD9B01AC01C7017A
:10D83000B6010F947A1A9B01AC0103C020E030E0DE
:10D84000A901688579858A859B850F94FE20688764
:10D8500079878A879B87DF91CF91FF90EF90DF9048
:10D86000CF9008952F923F924F925F926F927F9246
:10D870008F929F92AF92BF92CF92DF92EF92FF92E0
:10D880001F93CF93DF9300D01F92CDB7DEB74A012D
:10D890001901FC014080518062807380FB01C080CF
:10D8A000D180E280F38020913E1730913F17409164
:10D8B000401750914117C301B2010F94141A8111FE
:10D8C0000EC011E0A70196016091421770914317B5
:10D8D00080914417909145170F94141A811110E00C
:10D8E00080E1EEE3F7E1A8ECB6E101900D928A95B4
:10D8F000E1F7F40180809180A280B380209127021B
:10D90000309128024091290250912A02C501B401A8
:10D910000F94141A882379F18092D0169092D11620
:10D92000A092D216B092D31680922702909228022B
:10D93000A0922902B0922A0220E030E040E05FE3AA
:10D9400060914711709148118091491190914A114D
:10D950000F947A1A69837A838B839C83CE01019614
:10D960000E94ACCF80E1EEE3F7E1A8ECB6E10190D4
:10D970000D928A95E1F74092C8165092C9166092AE
:10D98000CA167092CB16C092CC16D092CD16E092E9
:10D99000CE16F092CF16F101208131814281538160
:10D9A0006091D4167091D5168091D6169091D716A5
:10D9B0000F94FE206093D4167093D5168093D616DC
:10D9C0009093D716112379F02AEF3EE74AE25FE3FE
:10D9D00060914B1170914C1180914D1190914E11AD
:10D9E0000F947A1A04C060E070E080EA91E46983E1
:10D9F0007A838B839C83CE0101960E94ACCF80E119
:10DA0000EEE3F7E1A8ECB6E101900D928A95E1F71B
:10DA10000F900F900F900F90DF91CF911F91FF907B
:10DA2000EF90DF90CF90BF90AF909F908F907F90BE
:10DA30006F905F904F903F902F9008950F931F939A
:10DA4000CF93DF93CDB7DEB728970FB6F894DEBF3C
:10DA50000FBECDBF8C010E946CF81D821E821F82FA
:10DA6000188620E030E040E05FE360914617709157
:10DA7000471780914817909149170F94FE206983AA
:10DA80007A838B839C839E012B5F3F4FAE014F5F58
:10DA90005F4F62E477E18EE397E10E94326C1D8272
:10DAA0001E821F82188620E030E040E05FE3F8012C
:10DAB00060857185828593850F94FE2069837A83C2
:10DAC0008B839C83B8016C5F7F4F9E012B5F3F4F20
:10DAD000AE014F5F5F4FC8010E94326C28960FB6AF
:10DAE000F894DEBF0FBECDBFDF91CF911F910F9194
:10DAF00008952F923F924F925F926F927F928F92F2
:10DB00009F92AF92BF92CF92DF92EF92FF920F93CC
:10DB10001F93CF93DF93CDB7DEB7A0970FB6F894DE
:10DB2000DEBF0FBECDBF8C011B0140903E17509051
:10DB30003F17609040177090411780904217909067
:10DB40004317A0904417B0904517DC018D919D912B
:10DB50000D90BC91A02D8D879E87AF87B88B9C01BF
:10DB6000AD01C301B2010F94FD206B017C01D8010E
:10DB700014968D919D910D90BC91A02D898B9A8BBF
:10DB8000AB8BBC8B9C01AD01C501B4010F94FD2092
:10DB90006D8B7E8B8F8B988FD1018D919D910D9088
:10DBA000BC91A02D8D839E83AF83B8879C01AD016E
:10DBB000C301B2010F94FD20698F7A8F8B8F9C8FE8
:10DBC000D10114968D919D910D90BC91A02D8987C6
:10DBD0009A87AB87BC879C01AD01C501B4010F9446
:10DBE000FD206D8F7E8F8F8F98A3A7019601C701AF
:10DBF000B6010F947A1A6B017C012D893E894F89F9
:10DC0000588DCA01B9010F947A1A9B01AC01C70162
:10DC1000B6010F94FE204B015C012D853E854F859A
:10DC200058896D817E818F8198850F94FD202B010D
:10DC30003C0129893A894B895C8969857A858B857C
:10DC40009C850F94FD206B017C01A3019201C3010F
:10DC5000B2010F947A1A2B013C01A7019601C7016A
:10DC6000B6010F947A1A9B01AC01C301B2010F9463
:10DC7000FE200F94AC236B017C01298D3A8D4B8DD6
:10DC80005C8DCA01B9010F947A1A2B013C012D8DCC
:10DC90003E8D4F8D58A1CA01B9010F947A1A9B018C
:10DCA000AC01C301B2010F94FE209B01AC01C50180
:10DCB000B4010F945E231816E4F420E030E0A901CB
:10DCC000C701B6010F945E2387FF04C0C701B601E8
:10DCD000905802C0C701B60120E030E040EA50E4AD
:10DCE0000F945E2318162CF4B801C1010E94796DBF
:10DCF00046C020E030E040E050E4C501B4010F949C
:10DD00005E2318161CF4C8010E941E6D19821A8227
:10DD10001B821C82A801485F5F4FB8016C5F7F4F78
:10DD20009E012F5F3F4FC8010E94326C2DEC3CECEE
:10DD30004CEC5CE3C701B6010F947A1A9B01AC016D
:10DD40006091E00A7091E10A8091E20A9091E30A01
:10DD50000F947A1A69837A838B839C838091D81677
:10DD600081110E9498F8A101485F5F4FB1016C5F7B
:10DD70007F4F9E012F5F3F4FC1010E94326CA096E2
:10DD80000FB6F894DEBF0FBECDBFDF91CF911F91CC
:10DD90000F91FF90EF90DF90CF90BF90AF909F904A
:10DDA0008F907F906F905F904F903F902F9008954D
:10DDB0008C3891051CF02CE880E002C0282F892FB8
:10DDC00020939408809395080C943BDB8091C216B5
:10DDD0009091C316892B39F00E943EB891E08111D1
:10DDE00003C090E001C091E0892F0895CF93DF93A5
:10DDF000C82FD62F0E94D6B8882321F0DF91CF916B
:10DE00000C94E66E8C2F0E948DB8811101C08D2F6D
:10DE1000DF91CF9108952F923F924F925F926F9230
:10DE20007F928F929F92AF92BF92CF92DF92EF92AA
:10DE3000FF920F931F93CF93DF93CDB7DEB7CB56EF
:10DE4000D1090FB6F894DEBF0FBECDBF81EC9CE1C7
:10DE50000E94B2500E94C99081110C94837984E58C
:10DE60000E94D6B8882329F00E9452B881110E94DE
:10DE7000D6D380E090E0A0E8BFE38093E00A9093DF
:10DE8000E10AA093E20AB093E30A8093C416909348
:10DE9000C516A093C616B093C7168DEC9CECACE4E7
:10DEA000BEE38093DC0A9093DD0AA093DE0AB09370
:10DEB000DF0A80E090E0A0E2B1E48093D80A90937A
:10DEC000D90AA093DA0AB093DB0A8CE390E090932E
:10DED000D70A8093D60A8DEC90E09093D50A809370
:10DEE000D40A1092D30A4AE959E969E97EE38FE43A
:10DEF0000E94A5AF29966CAF7DAF8EAF9FAF2997DB
:10DF000060E083E40E94F66EA5968FAFA59760E06F
:10DF10008BE40E94F66EA6968FAFA69782E40E94CD
:10DF2000D6B88823C9F00E9456B80F946A2270931D
:10DF3000D70A6093D60A6115710571F068527109AC
:10DF40006536710548F06CE870E083E99CE10E9459
:10DF5000D7518EE89CE1B0C18CE40E94D6B88823EA
:10DF600001F10E9456B86B017C016093DC0A70934A
:10DF7000DD0A8093DE0A9093DF0A20E030E0A901F9
:10DF80000F945E2387FD0AC020E030E040E050E4BB
:10DF9000C701B6010F94141A18161CF486E69CE10A
:10DFA0008BC181E50E948DB8882351F18091C21602
:10DFB0009091C316892B09F10E9456B86B017C0120
:10DFC0006093C4167093C5168093C6169093C716B7
:10DFD0002DEC3CEC4CE45DE30F945E2387FD0AC01E
:10DFE00020E030E040E751E4C701B6010F94141A75
:10DFF000181634F485E39CE15FC18AE09CE15CC1C2
:10E0000083E50E94D6B88823C9F00E9456B84B0118
:10E010005C012DEC3CEC4CEC5DE30F945E2387FD42
:10E020000AC020E030E040E050E4C501B4010F94A4
:10E03000141A181654F483EE9BE13EC1ADEC8A2EFF
:10E04000ACEC9A2EA92CAEE3BA2E80E50E948DB8D6
:10E05000882371F18091C2169091C316892B19F40F
:10E060008BEA9BE129C18091D30A8F5F8093D30A09
:10E070000E9456B86B017C016093D80A7093D90A4C
:10E080008093DA0A9093DB0A20E030E0A9010F9434
:10E090005E2387FD0AC020E030E048EC51E4C70170
:10E0A000B6010F94141A18161CF483E89BE104C1FE
:10E0B00086E40E94D6B88823C9F00E9456B86B0146
:10E0C0007C0120E030E040E85FE30F945E2387FDB1
:10E0D0000AC020E030E040E850E4C701B6010F94E8
:10E0E000141A18164CF48AE59BE1E6C0C12CD12C19
:10E0F000F0EEEF2EFFE3FF2EA7019601C701B60158
:10E100000F947A1A9B01AC0160E070E084E490E423
:10E110000F94F8212091E00A3091E10A4091E20A3F
:10E120005091E30A0F947A1A2B013C01A501940146
:10E13000C501B4010F947A1AA70196010F947A1AB7
:10E140002CEE31E548EB5DE30F94F8219B01AC0127
:10E15000C301B2010F947A1A6093E00A7093E10A46
:10E160008093E20A9093E30A88E40E94D6B8882359
:10E1700081F00E9456B80F946A227093D50A60937A
:10E18000D40A655A71096838710518F08CE29BE170
:10E1900093C085E50E948DB88823F1F00E947AFA39
:10E1A000611571058105910511F00F94A5158091F8
:10E1B000C2169091C316892B19F00E9456B804C05C
:10E1C00060E070E088E492E46093CF0A7093D00A34
:10E1D0008093D10A9093D20A82E50E948DB8811172
:10E1E00003C088EF9AE168C08091C2169091C3166F
:10E1F000892B61F00E9452B86B969FAF8EAF6B97E0
:10E20000181619064CF084EC9AE156C02AE130E069
:10E210006B963FAF2EAF6B9789E50E94D6B88823E7
:10E2200079F00E9456B82091DE163091DF164091A9
:10E23000E0165091E1160F94FD206B017C0108C09F
:10E24000C0904217D0904317E0904417F0904517C4
:10E2500088E50E94D6B8882369F00E9456B82091BC
:10E26000DA163091DB164091DC165091DD160F94D2
:10E27000FD2008C060913E1770913F1780914017B4
:10E28000909141176093C70A7093C80A8093C90A96
:10E290009093CA0AC092CB0AD092CC0AE092CD0ADF
:10E2A000F092CE0AB701A60187EC9AE00F94E20A39
:10E2B000811106C08AE99AE10E94B2500C948379D8
:10E2C00084E40E948DB891E089270E9460BF20E01D
:10E2D00030E040EA50E46091461770914717809112
:10E2E0004817909149170F94141A87FF1CC0198A78
:10E2F0001A8A1B8A1C8A80E090E0A0EAB0E4898335
:10E300009A83AB83BC83BE016F5E7F4FCE010196C3
:10E310000E9411D180E1E8ECF6E1AEE3B7E10190B3
:10E320000D928A95E1F730916712A7963FAFA797B4
:10E33000109267120E9463C889E79AE10E94B25066
:10E340008091D60A9091D70A8A3191056CF4809118
:10E35000D40A9091D50A0E94E4DB61E080E00E943B
:10E36000E0D5811109C00DC50E94D86E81E00E94E0
:10E3700062D48111ECCF05C510924A1710924B1749
:10E3800010924C1710924D178AE497E10E94F3699E
:10E390008091D30A882309F455C020E030E040E79B
:10E3A00051E460914B1170914C1180914D119091FD
:10E3B0004E110F94F82169837A838B839C8380E1CB
:10E3C000EEE3F7E1A8ECB6E101900D928A95E1F752
:10E3D0002091D80A3091D90A4091DA0A5091DB0A8B
:10E3E0006091D4167091D5168091D6169091D7165B
:10E3F0000F94FE206093D4167093D5168093D61692
:10E400009093D716CE0101960E94ACCF2091D80AE6
:10E410003091D90A4091DA0A5091DB0A6091D41602
:10E420007091D5168091D6169091D7160F94FD2035
:10E430006093D4167093D5168093D6169093D71602
:10E440000E946CF885E0E2ECFAE0DF01282F1D92D3
:10E450002A95E9F7EDEBFAE0DF01282F1D922A95C6
:10E46000E9F7E8EBFAE0DF011D928A95E9F780E130
:10E47000EEE3F7E1A8ECB6E101900D928A95E1F7A1
:10E480008091DC0A9091DD0AA091DE0AB091DF0A4A
:10E490008093D0169093D116A093D216B093D31632
:10E4A00019821A821B821C829E012F5F3F4F40ED12
:10E4B00056E16CEC76E188EC96E10E94326C9E01AC
:10E4C0002B5B3F4F40ED56E16CEC76E188EC96E13A
:10E4D0000E94326CA596BFADA597BB23B9F02091E1
:10E4E0003E1730913F1740914017509141172E969B
:10E4F0002CAF3DAF4EAF5FAF2E97809142179091FA
:10E500004317A0914417B091451716C02091C70A30
:10E510003091C80A4091C90A5091CA0A2E962CAF70
:10E520003DAF4EAF5FAF2E978091CB0A9091CC0A52
:10E53000A091CD0AB091CE0A69968CAF9DAFAEAFD7
:10E54000BFAF6997212C312C9FEF2A969FAF2A9756
:10E55000AFEF6596AFAF6597BFEF6C96BFAF6C97A7
:10E56000EFE4A096EFAFA097F3ECA296FFAFA297CF
:10E5700027E4A3962FAFA39781E090E0A0E0B0E05E
:10E58000022C04C0880F991FAA1FBB1F0A94D2F740
:10E59000AB968CAF9DAFAEAFBFAFAB97A2ECBAE07E
:10E5A0006496BFAFAEAF649700E010E0AC962FAEBC
:10E5B000AC976496EEADFFAD649781916496FFAF22
:10E5C000EEAF649790E0A0E0B0E0AB962CAD3DAD2F
:10E5D0004EAD5FADAB9782239323A423B523892B44
:10E5E0008A2B8B2B09F004C18091D0129091D1120B
:10E5F000289EB001299E700D389E700D11248091C7
:10E60000741190917511680F791F072E000C880BFB
:10E61000990B0F941B1A62966CAF7DAF8EAF9FAFB4
:10E6200062978091D2129091D312089FB001099FF6
:10E63000700D189F700D11248091761190917711B3
:10E64000680F791F072E000C880B990B0F941B1A6B
:10E650006B017C0162962CAD3DAD4EAD5FAD629716
:10E660002E966CAD7DAD8EAD9FAD2E970F94FD2097
:10E670002B013C01A701960169966CAD7DAD8EAD75
:10E680009FAD69970F94FD204B015C01A30192019E
:10E69000C301B2010F947A1A2B013C01A501940128
:10E6A000C501B4010F947A1A9B01AC01C301B201F8
:10E6B0000F94FE200F94AC234B015C0162962CADAD
:10E6C0003DAD4EAD5FAD62976091C70A7091C80ACB
:10E6D0008091C90A9091CA0A0F94FD202B013C0138
:10E6E000A70196016091CB0A7091CC0A8091CD0A66
:10E6F0009091CE0A0F94FD206B017C01A301920141
:10E70000C301B2010F947A1A2B013C01A7019601B3
:10E71000C701B6010F947A1A9B01AC01C301B20183
:10E720000F94FE200F94AC2320E030E040E751E44A
:10E730000F94F821A50194010F94FE206B017C0138
:10E740008090CF0A9090D00AA090D10AB090D20ABF
:10E7500020E030E040E85FE3C501B4010F945E23A0
:10E760001816FCF4C501B4010F946A224B015C0138
:10E7700016161706180619063CF40F945715A5012E
:10E7800094010F948C2003C060E070E0CB010F94E3
:10E790001B1A9B01AC01B601C7010F94FE206B014F
:10E7A0007C016C962FAD6C97A0963FADA097A2967A
:10E7B0004FADA297A3965FADA397B601C7010F9483
:10E7C000141A87FF15C02A960FAF2A97AC963FAD53
:10E7D000AC9765963FAF65976C96CFAE6C97A09659
:10E7E000DFAEA097A296EFAEA297A396FFAEA39737
:10E7F0000F5F1F4F0530110509F0DBCE4FEF241AD4
:10E80000340A55E02516310409F0B6CE65968FAD71
:10E810006597E82FF0E0EE53F54F81E090E02A96FF
:10E820000FAC2A9702C0880F991F0A94E2F79081D3
:10E83000892B808365969FAD65979F3F09F487C2BA
:10E840002A96AFAD2A97AF3F09F481C22091D0122A
:10E850003091D11265964FAD65974203B001439F49
:10E86000700D11248091741190917511680F791FAA
:10E87000072E000C880B990B0F941B1A162F072FCD
:10E88000382E292E862F902FA32DB22D21968CAFB6
:10E890009DAFAEAFBFAF21972091D2123091D3126E
:10E8A0002A965FAD2A975203B001539F700D112431
:10E8B0008091761190917711680F791F072E000CC7
:10E8C000880B990B0F941B1A6B017C0125966CAF7A
:10E8D0007DAF8EAF9FAF2597AB01BC01CE01CD962A
:10E8E0000F94E20A882309F436C220E030E040EABF
:10E8F00050E4612F702F832D922D0F94FE204B0139
:10E900005C01FE01B9968CE0DF011D928A95E9F762
:10E91000C401D50189A79AA7ABA7BCA7CDA6DEA63F
:10E92000EFA6F8AA6596BFAD6597B111B1C22A9658
:10E93000EFAD2A97E1118DC220E030E040EA50E4CB
:10E94000C701B6010F94FE206B017C012A96FFAD32
:10E950002A97FF2309F416C32A963FAD2A9734302D
:10E960000CF010C3E2ED4E2EE3E55E2EEBE76E2ECB
:10E97000E1E47E2E89A49AA4ABA4BCA42DA53EA557
:10E980004FA558A92E962CAF3DAF4EAF5FAF2E9737
:10E9900025966CAD7DAD8EAD9FAD25970F94FD2076
:10E9A00062966CAF7DAF8EAF9FAF6297A501940169
:10E9B00021966CAD7DAD8EAD9FAD21970F94FD205E
:10E9C0006DAB7EAB8FAB98AF62968CAD9DADAEADAF
:10E9D000BFAD629789AF9AAFABAFBCAFA501940151
:10E9E00060913E1770913F178091401790914117A9
:10E9F0000F94FD204B015C012E962CAD3DAD4EAD2C
:10EA00005FAD2E9760914217709143178091441724
:10EA1000909145170F94FD202E966CAF7DAF8EAF71
:10EA20009FAF2E97812F902FA32DB22D89839A838C
:10EA3000AB83BC83CD82DE82EF82F886C090DC0A95
:10EA4000D090DD0AE090DE0AF090DF0AC986DA860F
:10EA5000EB86FC862DEC3CEC4CEC5CE3C301B20194
:10EA60000F947A1A2091E00A3091E10A4091E20A6B
:10EA70005091E30A0F947A1A20914A1730914B175C
:10EA800040914C1750914D170F94FE206D877E8753
:10EA90008F87988BA5019401C501B4010F947A1A50
:10EAA0004B015C012E962CAD3DAD4EAD5FAD2E976A
:10EAB000CA01B9010F947A1A9B01AC01C501B401D6
:10EAC0000F94FE2020E030E040E050E40F945E23FD
:10EAD000181684F420E030E040E05FE3C701B6019F
:10EAE0000F94FE2069AB7AAB8BAB9CABCE018996C1
:10EAF0000E941E6D8091DC0A9091DD0AA091DE0AD1
:10EB0000B091DF0A89AB9AABABABBCAB198A1A8A5E
:10EB10001B8A1C8A9E012F5E3F4FAE014F5C5F4FE8
:10EB2000BE01635D7F4FCE0189960E94326C809159
:10EB3000D81681110E9498F840906B0250906C0298
:10EB400060906D0270906E02E0904311F09044115D
:10EB50000091451110914611A0903F11B0904011C5
:10EB6000C0904111D09042119501A601B701C80192
:10EB70000F945E23181614F4750186012DEC3CECFD
:10EB80004CEC5DE3B701C8010F947A1A60936B02F5
:10EB900070936C0280936D0290936E0240E0BE0110
:10EBA0006B5C7F4FCE0101960E9413E140926B0295
:10EBB00050926C0260926D0270926E0280E1EEE300
:10EBC000F7E1A8ECB6E101900D928A95E1F780910A
:10EBD000DC0A9091DD0AA091DE0AB091DF0A898FEC
:10EBE0009A8FAB8FBC8F8DA39EA3AFA3B8A7CC2465
:10EBF000C394D12CD60111976796BFAFAEAF67977C
:10EC0000812C912C5401839466960FAC669704C0B6
:10EC1000880C991CAA1CBB1C0A94D2F781E090E0D6
:10EC2000A0E0B0E00C2C04C0880F991FAA1FBB1FE6
:10EC30000A94D2F79C01AD01282939294A295B2978
:10EC40006F962CAF3DAF4EAF5FAF6F9781E066968A
:10EC50000FAC669701C0880F0A94EAF7A2968FAFAF
:10EC6000A29748EB5AE064965FAF4EAF64978DEB86
:10EC70009AE02C969FAF8EAF2C97A2ECBAE06096EC
:10EC8000BFAFAEAF6097212C312CA1963FAE2EAE18
:10EC9000A1976096EEADFFAD6097A496FFAFEEAF83
:10ECA000A497FFEF2F1A3F0A6096AEADBFAD6097F5
:10ECB0008C9190E0A0E0B0E06F962CAD3DAD4EADF4
:10ECC0005FAD6F9782239323A423B52328173907B9
:10ECD0004A075B0709F47AC16096EEADFFAD609715
:10ECE00031966096FFAFEEAF6097A496AEADBFAD24
:10ECF000A4978C9190E0A0E0B0E088219921AA210E
:10ED0000BB21892B8A2B8B2B09F052C164962EAD27
:10ED10003FAD64972F5F3F4F64963FAF2EAF649730
:10ED20002C964EAD5FAD2C974F5F5F4F2C965FAF2B
:10ED30004EAF2C9755E02516310409F0A6CF8FEF82
:10ED4000C81AD80A96E0C916D10409F053CF8091A9
:10ED50008511809386116B96AEADBFAD6B97119701
:10ED60006B96BFAFAEAF6B97AB2B59F06596BFAD4F
:10ED70006597BF3F31F02A96EFAD2A97EF3F09F034
:10ED8000A9CB6FEF8EE89AE10E949BFD0E946CF880
:10ED900080E090E0A0EAB0E48093D0169093D11682
:10EDA000A093D216B093D31619821A821B821C82AA
:10EDB0009E012F5F3F4F40ED56E16CEC76E188EC11
:10EDC00096E10E94326C8091CB0A9091CC0AA0917E
:10EDD000CD0AB091CE0A4091C70A5091C80A6091FD
:10EDE000C90A7091CA0A4093C8165093C916609315
:10EDF000CA167093CB168093CC169093CD16A09321
:10EE0000CE16B093CF1619821A821B821C829E01E5
:10EE10002F5F3F4F40ED56E16CEC76E188EC96E1D8
:10EE20000E94326CA796FFADA797F09367120E94DD
:10EE300063C8A6962FADA697211165C210929508BA
:10EE4000109294080E943BDB80E090E00E94E4DB9B
:10EE50005AC2812F902FA32DB22D89A79AA7ABA7B5
:10EE6000BCA720E030E040EA50E4C701B6010F94AF
:10EE7000FD206DA77EA78FA798AB2A962FAD2A9766
:10EE800024300CF459CD182D092D3A2C2B2C7AC096
:10EE900065964FAD659744300CF44CC02A965FAD33
:10EEA0002A9754307CF020E030E040EA50E4612FB3
:10EEB000702F832D922D0F94FD2069A77AA78BA721
:10EEC0009CA728C0812F902FA32DB22D89A79AA788
:10EED000ABA7BCA720E030E040EA50E4C701B60190
:10EEE0000F94FE206DA77EA78FA798AB2A968FADB3
:10EEF0002A9781110FC020E030E040EA50E4612FF2
:10EF0000702F832D922D0F94FD20162F072F382E52
:10EF1000292E38C020E030E040EA50E4C701B601B5
:10EF20000F94FD206B017C012A969FAD2A979430A7
:10EF30004CF518CD2A96AFAD2A97A1110DC020E04F
:10EF400030E040E251E4B401C5010F94FD20162FDA
:10EF5000072F382E292E06CD2A96BFAD2A97B4301A
:10EF6000D4F020E030E040E251E4B401C5010F9458
:10EF7000FD2069A77AA78BA79CA7182D092D3A2CED
:10EF80002B2CF0CC72ED472E73E5572E7BEF672EBE
:10EF900070E4772EEFCC182D092D3A2C2B2C62ED36
:10EFA000462E63E5562E6BEF662E61E4762EE2CC9C
:10EFB000808190E0A0E0B0E088219921AA21BB21C6
:10EFC000892B8A2B8B2B09F0D0C0A0CE2C96AEAD0E
:10EFD000BFAD2C978C9190E0A0E0B0E08821992102
:10EFE000AA21BB21892B8A2B8B2B09F075CE00918E
:10EFF000741110917511E090D012F090D1126796B3
:10F000004EAD5FAD6797E49EB001E59E700DF49E36
:10F01000700D1124600F711F072E000C880B990BC7
:10F020000F941B1A20E030E040E050E40F94FE20E3
:10F030006D8F7E8F8F8F98A3CE9CB001CF9C700D6B
:10F04000DE9C700D1124600F711F072E000C880BC1
:10F05000990B0F941B1A20E030E040E050E40F942D
:10F06000FD20698B7A8B8B8B9C8B4AE351E061E0AE
:10F0700070E0CE014D960F94C6028091D21290910D
:10F08000D312A196AEADBFADA197A89FB001A99F25
:10F09000700DB89F700D11248091761190917711A9
:10F0A000680F791F072E000C880B990B0F941B1A01
:10F0B0002B013C0120E030E040E85FE30F94141A9C
:10F0C00087FD12C020E030E84AE953E4C301B201F1
:10F0D0000F945E23181674F4412C30E8532E3AE94D
:10F0E000632E33E4732E06C0412C512C20E8622E8F
:10F0F0002FE3722E4D8A5E8A6F8A788E49A25AA2B9
:10F100006BA27CA24AE351E061E070E0CE0141963F
:10F110000F94C60249A15AA16BA17CA1CE014D96C4
:10F120000F94E20A882351F04D895E896F89788DAA
:10F13000CE0141960F94E20A81110FC02C96EEADDC
:10F14000FFAD2C978081A296FFADA2978F2B2C96B6
:10F15000AEADBFAD2C978C93BFCDBE016F5E7F4F20
:10F16000CE014D960E94796DE9CF6496EEADFFAD6C
:10F170006497808190E0A0E0B0E088219921AA21E5
:10F18000BB21892B8A2B8B2B09F0C0CD00917611E6
:10F1900010917711E090D212F090D312A196EEADBB
:10F1A000FFADA197EE9DB001EF9D700DFE9D700D1E
:10F1B0001124600F711F072E000C880B990B0F9400
:10F1C0001B1A20E030E040E050E40F94FE2069A3D9
:10F1D0007AA38BA39CA32E9CB0012F9C700D3E9C08
:10F1E000700D1124600F711F072E000C880B990BF6
:10F1F0000F941B1A20E030E040E050E40F94FD2013
:10F200006D8B7E8B8F8B988F8091D0129091D112C5
:10F2100067962EAD3FAD6797289FB001299F700D6F
:10F22000389F700D11248091741190917511680FA1
:10F23000791F072E000C880B990B0F941B1A2B01BA
:10F240003C0120E030E040E85FE30F94141A87FDB2
:10F2500011C020E030E04DE953E4C301B2010F9446
:10F260005E2318166CF4412C512C9DE9692E93E411
:10F27000792E06C0412C512C80E8682E8FE3782E21
:10F28000498A5A8A6B8A7C8A4D8E5E8E6F8E78A2EE
:10F2900045E351E061E070E0CE0181960F94C60233
:10F2A00045E351E061E070E0CE0145960F94C6025F
:10F2B00049A15AA16BA17CA1CE014D960F94E20AFF
:10F2C000882351F04D895E896F89788DCE014196F2
:10F2D0000F94E20A81110FC06496AEADBFAD649782
:10F2E0008C91A296BFADA2978B2B6496EEADFFAD2D
:10F2F000649780830BCDBE016F5E7F4FCE014D962C
:10F300000E94796DE9CFC559DF4F0FB6F894DEBF83
:10F310000FBECDBFDF91CF911F910F91FF90EF9066
:10F32000DF90CF90BF90AF909F908F907F906F9025
:10F330005F904F903F902F900895CF92DF92EF9281
:10F34000FF920F931F93CF93DF936C017A018B0190
:10F35000C0E0D0E0CE15DF0581F0D8016D918D01C0
:10F36000D601ED91FC910190F081E02DC601199537
:10F37000892B11F02196EECF7E01C701DF91CF914D
:10F380001F910F91FF90EF90DF90CF900895089517
:10F3900080E090E00895FC01538D448D252F30E0EE
:10F3A000842F90E0821B930B541710F0CF96089592
:10F3B00001970895FC01918D828D981761F0828DDF
:10F3C000DF01A80FB11D5D968C91928D9F5F9F7399
:10F3D000928F90E008958FEF9FEF0895FC01918D3B
:10F3E000828D981731F0828DE80FF11D858D90E0A8
:10F3F00008958FEF9FEF0895FC01918D228D892F45
:10F4000090E0805C9F4F821B91098F73992708952C
:10F410008BE493E10E94FC7921E0892B09F420E040
:10F42000822F0895FC01848DDF01A80FB11DA35A1E
:10F43000BF4F2C91848D90E001968F739927848F14
:10F44000A689B7892C93A089B1898C918370806437
:10F450008C93938D848D981306C00288F389E02DD8
:10F4600080818F7D80830895EF92FF920F931F9389
:10F47000CF93DF93EC0181E0888F9B8D8C8D981367
:10F4800005C0E889F989808185FD26C0F62E0B8D9F
:10F4900010E00F5F1F4F0F731127E02E8C8DE812C5
:10F4A0000CC00FB607FCFACFE889F989808185FF87
:10F4B000F5CFCE010E94127AF1CF8B8DFE01E80FBD
:10F4C000F11DE35AFF4FF0829FB7F8940B8FEA8942
:10F4D000FB89808180620AC09FB7F894EE89FF891A
:10F4E0006083E889F98980818370806480839FBF0D
:10F4F00081E090E0DF91CF911F910F91FF90EF900D
:10F500000895CF93DF93EC01888D8823C9F0EA89B1
:10F51000FB89808185FD05C0A889B9898C9186FD0C
:10F520000FC00FB607FCF5CF808185FFF2CFA88909
:10F53000B9898C9185FFEDCFCE010E94127AE7CF79
:10F54000DF91CF91089580E090E0892B41F080E039
:10F5500090E0892B21F00E940000811121C080E001
:10F5600090E0892B41F080E090E0892B21F00E940F
:10F570000000811118C080E090E0892B21F00E94EA
:10F58000087A811113C080E090E0892BA1F080E01F
:10F5900090E0892B81F00E94000081110AC008953B
:10F5A0000E940000DCCF0E940000E5CF0E94000016
:10F5B000EACF0C94000008950F941024CF93DF93AA
:10F5C000EC01CB01E881F981608171810E94759223
:10F5D00088819981DC01ED91FC912081AA81BB8118
:10F5E000222369F02C91293650F43196DC01ED93F9
:10F5F000FC93EA81FB8180818F5F8083E9CF8C91CE
:10F60000893670F48FE28083E881F981808191816D
:10F61000019691838083EA81FB8180818F5F808363
:10F62000DF91CF9108951F920F920FB60F92112480
:10F630000BB60F922F933F934F935F936F937F93EC
:10F640008F939F93AF93BF93EF93FF938BE493E1DB
:10F650000E94127AFF91EF91BF91AF919F918F918C
:10F660007F916F915F914F913F912F910F900BBEC2
:10F670000F900FBE0F901F9018951F920F920FB60C
:10F680000F9211240BB60F922F938F939F93EF93AA
:10F69000FF93E0915B13F0915C138081E091611323
:10F6A000F091621382FD12C09081809164138F5F8C
:10F6B0008F7320916513821751F0E0916413F0E08D
:10F6C000E55BFC4E958F8093641301C08081FF91B0
:10F6D000EF919F918F912F910F900BBE0F900FBEC6
:10F6E0000F901F9018958BE1E1E4F4E1A6E2B4E1FC
:10F6F00001900D928A95E1F780917916806280934E
:10F70000791608958091791682FF1FC08DE29EE1DF
:10F710000E94B2506091751670917616809177169E
:10F72000909178164AE00E9430518FE20E94A050DA
:10F730006091711670917216809173169091741683
:10F740004AE00E9430510C94F1528FE39EE10C94F8
:10F75000B2501092E40A809179168F7B8B7F809350
:10F7600079160E945050882321F088EE93E10C9482
:10F77000DB9408958091791683FF03C084608093A1
:10F7800079160895CF92DF92EF92FF920F931F9315
:10F79000CF93DF93CDB7DEB7EDB6FEB6DC010D90AB
:10F7A0000020E9F79D01281B390B2C5F3F4F4DB717
:10F7B0005EB7421B530B0FB6F8945EBF0FBE4DBF32
:10F7C0000DB71EB70F5F1F4F9F938F9389E29DE187
:10F7D0009F938F931F930F930F94AC19680154E07C
:10F7E000C50ED11C0F900F900F900F900F900F909F
:10F7F000F6018081882349F0082E000C990B0F94A4
:10F800001524F60181936F01F3CFC8010E948FDDAB
:10F8100085E29DE10E9481B70FB6F894FEBE0FBE4F
:10F82000EDBEDF91CF911F910F91FF90EF90DF9090
:10F83000CF9008958F929F92AF92BF92CF92DF9216
:10F84000EF92FF92CF9380917916877F80937916FC
:10F8500080914414882321F081E494E10E94DB9498
:10F86000109225141092221485E3809321140E9493
:10F870007AFA6B017C0120EDC20E27E0D21EE11C5A
:10F88000F11CA89561E0809121140E94EDF861E0DF
:10F89000809121140E941CF9209A289A219A239879
:10F8A000229A81E00E94E45A85E0809323140E940A
:10F8B000E45ACAE08FEF0E94D85AC150D9F7A895F0
:10F8C00020E030E0A90160E081E294E10E94BB9376
:10F8D00080932414813061F00E947AFADC01CB011C
:10F8E0008C199D09AE09BF09B7FDEACF81E062C05E
:10F8F000A8952AEA31E040E050E068E081E294E136
:10F900000E94BB93853011F481E00AC0C4E00E94DC
:10F91000DD5A80932414C150D1F78A3A61F482E011
:10F9200080932514A89580912514823081F0812C34
:10F93000912C540111C00E947AFADC01CB018C1980
:10F940009D09AE09BF09B7FDD4CF82E033C0812C39
:10F95000912CA12C80E4B82E20E030E0A90167E3CF
:10F9600081E294E10E94BB93A501940169E281E2E6
:10F9700094E10E94BB9380932414882361F00E9439
:10F980007AFADC01CB018C199D09AE09BF09B7FDDC
:10F99000E3CF8AE00FC080912514823021F520E06A
:10F9A00030E0A9016AE381E294E10E94BB938823DD
:10F9B00061F088E08093221481E294E10E94B39385
:10F9C0000E94D85087E19DE122C00E94DD5A807CD0
:10F9D000803C19F483E0809325140E94DD5A0E9434
:10F9E000DD5A0E94DD5A81E294E10E94B3931092A5
:10F9F000231481E00F94DD0081110CC080E00F948E
:10FA0000DD00811107C00E94D45083E09DE10E9477
:10FA1000B2501AC063E074E181E494E10E9406925E
:10FA2000811105C00E94D45082EF9CE1F0CF8091FB
:10FA300079168860809379160E94D85086EE9CE1F2
:10FA40000E94B2500E944450CF91FF90EF90DF90FF
:10FA5000CF90BF90AF909F908F900C94737BFC01E0
:10FA600080818823E1F0853ED1F08E32C1F0809113
:10FA700066198E32A1F09385892F8A7081F498716E
:10FA800021E0903109F020E08091791620FB84F983
:10FA900080937916903141F08085873411F080E0B1
:10FAA000089581858E37D9F381E008950F931F93D0
:10FAB000CF93DF93CDB7DEB7EB970FB6F894DEBFE9
:10FAC0000FBECDBF86E294E10E94AE938BE1E6E2E9
:10FAD000F4E1DE01919601900D928A95E1F700E044
:10FAE00010E046E659E1BE016F5F7F4FCE0181967F
:10FAF0000E94709618163CF4CE0101960E942F7D4C
:10FB0000080F111DEECFCE0181960E94E494C8012A
:10FB1000EB960FB6F894DEBF0FBECDBFDF91CF914D
:10FB20001F910F910895FC0120E03EE2DB014C9112
:10FB3000403241F0283011F430833196DB014C9192
:10FB4000408331962F5F6F5F7F4F2B3079F71082A4
:10FB500008956F927F928F929F92AF92BF92CF92B1
:10FB6000DF92EF92FF920F931F93CF93DF93CDB766
:10FB7000DEB7C356D1090FB6F894DEBF0FBECDBFB6
:10FB80005C018B016DB67EB67E0187E5E80EF11C47
:10FB900046E659E1BE016F5F7F4FC5010E94709636
:10FBA00018160CF0AFC08C858871803109F06CC0DC
:10FBB0008DB69EB6BE016F5F7F4FC7010E94937DD9
:10FBC0000115110521F0F8018081811191C021E01A
:10FBD00081E090E0F70101900020E9F73197EE19FC
:10FBE000FF09E80FF91F32968DB79EB78E1B9F0B4A
:10FBF0000FB6F8949EBF0FBE8DBFEDB7FEB731961E
:10FC00006F01211102C0B80102C06BEC76E0C601A1
:10FC10000F945C24B701C6010F9446246BEC76E088
:10FC2000C6010F94462419A21CA221E0A701B50128
:10FC3000CE0181960E94DE9881110AC00E94D850A0
:10FC4000B70182ED9CE10E94C1508AE00E94A05061
:10FC50008BE1FE01B196DE01DC9601900D928A9552
:10FC6000E1F7B601CE01CC960E94A97DCE01CC96DB
:10FC70000E94E494CE0181960E94E4940FB6F89419
:10FC80009EBE0FBE8DBE84CFCE0101960E942F7DF9
:10FC9000882309F47DCFBE016F5F7F4F88EA99E129
:10FCA0000E94937D0115110529F488EAC82E89E187
:10FCB000D82E09C06801F60181916F018823A9F34C
:10FCC0000E94A050F8CFF60181916F01882319F0AE
:10FCD0000E94A050F8CF80E20E94A0506D8D7E8DD2
:10FCE0008F8D98A14AE00E9430510E94F15250CF6E
:10FCF000F80101900020E9F73197CF01801B910BAB
:10FD000020E068CF0FB6F8947EBE0FBE6DBECD5911
:10FD1000DF4F0FB6F894DEBF0FBECDBFDF91CF919E
:10FD20001F910F91FF90EF90DF90CF90BF90AF9019
:10FD30009F908F907F906F900895EF92FF920F9316
:10FD40001F93CF93DF93CDB7DEB7A0970FB6F8948C
:10FD5000DEBF0FBECDBF7C018B0146E659E1BE017F
:10FD60006F5F7F4FC7010E9470961816A4F4CE01F2
:10FD700001960E942F7D882381F3BE016F5F7F4F24
:10FD800088EA99E10E94937D68EA79E1C8010F94BD
:10FD90003324892B11F7A0960FB6F894DEBF0FBE5F
:10FDA000CDBFDF91CF911F910F91FF90EF900895FC
:10FDB0000F931F93CF93DF93CDB7DEB76B970FB63B
:10FDC000F894DEBF0FBECDBF8C0186E294E10E94A5
:10FDD000AE938BE1E6E2F4E1DE01119601900D9223
:10FDE0008A95E1F7B801CE0101960E949D7ECE0171
:10FDF00001960E94E4946B960FB6F894DEBF0FBE96
:10FE0000CDBFDF91CF911F910F910895DF92EF92B7
:10FE1000FF920F931F93CF93DF93CDB7DEB7279752
:10FE20000FB6F894DEBF0FBECDBF2091791623FF29
:10FE300037C1F42EE62E8C010E945050882309F41D
:10FE400080C0FF2009F48BC080917016882351F088
:10FE50000E94D45088EE9DE10E94B25080E090E074
:10FE60000E9428EE8AEE9AE09E838D838FE2809333
:10FE7000E90A81E08F83CE0105969A8389830296F1
:10FE80009C838B83F12C9BE1D92E80916F16F81601
:10FE900058F4DF9CB00111246F597A4ECE010196BF
:10FEA0000E94DE7AF394F1CF8F818B3558F468EE9F
:10FEB00073E1CE0101960E94DE7A8D819E810197C9
:10FEC0009E838D83ED81FE811082E091701684E027
:10FED000E89FF0011124EB51F54F80917516909138
:10FEE0007616A0917716B091781680839183A283BD
:10FEF000B3830E94D850B8018FEC9DE10E94C1509D
:10FF00006091701689E6689FB00111246751754FA2
:10FF100084EC9DE10E94C150409175165091761677
:10FF200060917716709178168EEB9DE10E949D513D
:10FF30008AE00E94A050809170168F5F80937016A7
:10FF400026C0FF2039F00E94D8508EEA9DE10E9421
:10FF5000B2501DC01092701682E0F82E02C0FF242D
:10FF6000F3940E94D85089EA9DE10E94B25081E04A
:10FF7000F81609F492C085E99DE10E94B250B801DB
:10FF800081EA9DE10E94C1508AE00E94A0500E9437
:10FF9000A97BB801CE0101960E948FEF8C010097DA
:10FFA00009F47EC069817A81EE2009F44DC021E018
:10FFB000AC0188EE93E10E94DE988823E9F18091FC
:10FFC000F9139091FA13A091FB13B091FC13809355
:10FFD000711690937216A0937316B09374161092C4
:10FFE0007516109276161092771610927816B80140
:10FFF00087E89DE10E94C1504091711650917216A0
:020000021000EC
:1000000060917316709174168FE79DE10E949D5167
:100010008AE00E94A05080E79DE10E94B250C80192
:100020000E94D87E80916619811102C0C80102C069
:1000300086E699E160E02EC0B8018CE59DE10E9462
:10004000C15089E59DE10FC026E5AC0188EE93E142
:100050000E94DE9881110AC0B80185E49DE10E94EA
:10006000C15082E49DE10E94B2501AC0809179167D
:10007000816080937916C8010E94D87E10925F1526
:10008000B80180E39DE10E94C1508AE00E94A05027
:1000900060E0C8010E94F6FD03C08BE99DE16DCFD1
:1000A00027960FB6F894DEBF0FBECDBFDF91CF917C
:1000B0001F910F91FF90EF90DF900895CF92DF9204
:1000C000EF92FF92CF936B017C01C42F80915B195B
:1000D00090915C19A0915D19B0915E198C159D05E8
:1000E000AE05BF05D1F00E946894811102C080E086
:1000F00018C02BE537E1B701A601809164199091F2
:1001000065190E94EA94882391F3C0925B19D092FA
:100110005C19E0925D19F0925E1981E0C111809343
:100120006319CF91FF90EF90DF90CF9008954F9299
:100130005F926F927F928F929F92AF92BF92CF9277
:10014000DF92EF92FF920F931F93CF93DF93EC0117
:10015000423051056105710510F480E069C0898560
:100160009A85AB85BC850196A11DB11D84179507A5
:10017000A607B70790F38F89803149F4852E962E14
:10018000A72EBB248B899C89AD89BE890FC0803284
:1001900021F78B889C88AD88BE88DB01CA01E7E027
:1001A000B695A79597958795EA95D1F7880E991EEC
:1001B000AA1EBB1E280139016A017B0141E0C5016D
:1001C000B4010E945E80882341F29F89903161F4DE
:1001D000DD24EE24FF249601220F331FF901E55A96
:1001E000F84E5182408211C0E894C7F8DD24EE2415
:1001F000FF249601220F331F220F331FF901E55A06
:10020000F84E40825182628273829A89923080F0E5
:100210004D815E816F817885840E951EA61EB71E66
:1002200080925F1990926019A0926119B092621940
:10023000DF91CF911F910F91FF90EF90DF90CF90C2
:10024000BF90AF909F908F907F906F905F904F90F6
:100250000895CF92DF92EF92FF920F931F93CF9367
:10026000DF93FC0181859285A385B4850196A11D4C
:10027000B11D84179507A607B70710F480E061C089
:100280008789803149F4BB27A72F962F852FC388F4
:10029000D488E588F6880FC0803281F783899489F5
:1002A000A589B6896A017B01C7E0F694E794D794E3
:1002B000C794CA95D1F78C0D9D1DAE1DBF1DE901D8
:1002C0006A017B018F0140915B1950915C1960912B
:1002D0005D1970915E1984179507A607B70739F065
:1002E00040E0BC01CD010E945E80882339F2F80114
:1002F0008789803179F4B701A601552766277727CA
:10030000440F551FFA01E55AF84E80819181A0E013
:10031000B0E012C0B701A6014F77552766277727AF
:10032000440F551F440F551FFA01E55AF84E8081BE
:100330009181A281B381BF7088839983AA83BB8393
:1003400081E0DF91CF911F910F91FF90EF90DF90AF
:10035000CF9008954F925F926F927F92AF92BF922B
:10036000CF92DF92EF92FF920F931F93CF93DF9381
:1003700000D01F92CDB7DEB78C0149835A836B83BF
:100380007C835901C12CD12C7601412C82E0582E5E
:10039000612C712C49815A816B817C819E012F5F78
:1003A0003F4FC8010E942981882341F1D301C20136
:1003B000F801058404C0880F991FAA1FBB1F0A9467
:1003C000D2F7C80ED91EEA1EFB1E49815A816B81E5
:1003D0007C818789803139F481E0483F5F4F610536
:1003E000710538F4D7CF81E0483F5F4F6F4F7F40B2
:1003F00088F2F501C082D182E282F3820F900F90E1
:100400000F900F90DF91CF911F910F91FF90EF9080
:10041000DF90CF90BF90AF907F906F905F904F90A4
:1004200008952F923F924F925F926F927F928F9298
:100430009F92AF92BF92CF92DF92EF92FF920F9373
:100440001F93CF93DF93CDB7DEB7CB56D1090FB64D
:10045000F894DEBF0FBECDBF4B015A0169012D9646
:10046000FFAEEEAE2D9720912F11309130114091BB
:10047000311150913211DC016D917D918D919C91E2
:100480000F947A1A0F946B23A3966CAF7DAF8EAF47
:100490009FAFA397209133113091341140913511C2
:1004A00050913611F40160817181828193810F94A2
:1004B0007A1A0F946B23A7966CAF7DAF8EAF9FAF68
:1004C000A7972091371130913811409139115091EF
:1004D0003A11D5016D917D918D919C910F947A1A6D
:1004E0000F946B23AB966CAF7DAF8EAF9FAFAB9786
:1004F00020913B1130913C1140913D1150913E11A2
:10050000F60160817181828193810F947A1A0F9430
:100510006B232B966CAF7DAF8EAF9FAF2B978091E7
:100520001A1183FF0EC02B962CAD3DAD4EAD5FADC5
:100530002B9720938114309382144093831450930B
:1005400084148091181190911911892B11F00C9439
:10055000C08ED8013C901196BC91BDABF801F281E0
:10056000F9AFD80113962C9080915F14909160148C
:10057000891B8F708F3021F480E00E941853F4CFD4
:10058000B0915F14AC96BFAFAC9780915F14E82F29
:10059000F0E0F8A7EFA3F8E58F9FC00111249C01BC
:1005A0002856344F23963FAF2EAF23978091751472
:1005B00090917614A0917714B0917814A3968CAC96
:1005C0009DACAEACBFACA397881A990AAA0ABB0A25
:1005D0008091791490917A14A0917B14B0917C143D
:1005E000A7962CAD3DAD4EAD5FADA797281B390B3F
:1005F0004A0B5B0B2BA33CA34DA35EA380917D1400
:1006000090917E14A0917F14B0918014AB962CAD84
:100610003DAD4EAD5FADAB97281B390B4A0B5B0B65
:1006200029A73AA74BA75CA78091811490918214C7
:10063000A0918314B09184142B96CCACDDACEEACBD
:10064000FFAC2B97C81AD90AEA0AFB0A09F477C04B
:100650008091800B81112DC020E030E0A9016091D4
:10066000850B7091860B8091870B9091880B0F946E
:10067000FE200F946A2220912F02309130026217DF
:100680007307BCF42B968CAD9DADAEADBFAD2B9773
:100690008093811490938214A0938314B093841454
:1006A0000E94D85087E99EE10E94B250C12CD12C03
:1006B0007601C701B6010F941B1A20912B023091CD
:1006C0002C0240912D0250912E020F947A1A2B0188
:1006D0003C0120E030E0A9010F945E2387FF04C0B5
:1006E00077FA709477F8709420E030E04AEF53E4A2
:1006F00060913B1170913C1180913D1190913E11A0
:100700000F947A1AA30192010F94141A87FF17C04D
:100710002B962CAD3DAD4EAD5FAD2B972093811444
:100720003093821440938314509384140E94D850C1
:1007300088E79EE10E94B250C12CD12C7601D501F0
:10074000C4018827B7FD83959927AA27BB27182FAF
:100750002BA13CA14DA15EA157FD126089A59AA5D0
:10076000ABA5BCA5B7FD1460F7FC1860C701B601C6
:100770000F941B1A20912B0230912C0240912D02D4
:1007800050912E020F947A1A6B017C0120E030E028
:10079000A9010F945E2387FF04C0C701B6019058DA
:1007A00002C0C701B60120E030E040E05FE30F94F3
:1007B000FE200F94712269AB7AAB8BAB9CAB88E5C2
:1007C000AFA1B8A58A9FF0018B9FF00D1124E856C8
:1007D000F44F1082EB5BFF4F108329A53AA54BA580
:1007E0005CA527962CAF3DAF4EAF5FAF279757FF65
:1007F0000DC050954095309521953F4F4F4F5F4F1D
:1008000027962CAF3DAF4EAF5FAF27978BA19CA132
:10081000ADA1BEA18DA79EA7AFA7B8ABB7FF0BC078
:10082000B095A095909581959F4FAF4FBF4F8DA7E5
:100830009EA7AFA7B8AB24013501B7FE07C044247B
:1008400055243201481859086A087B082396AEAD32
:10085000BFAD239755964D925D926D927C925897BD
:100860002DA53EA54FA558A959962D933D934D937F
:100870005C935C9727962CAD3DAD4EAD5FAD279751
:100880005D962D933D934D935C939097C501B40174
:100890000F941B1A2091700B3091710B4091720BC9
:1008A0005091730B0F947A1A21966CAF7DAF8EAF77
:1008B0009FAF2197698B7A8B8B8B9C8B6BA17CA1D3
:1008C0008DA19EA10F941B1A2091740B3091750B72
:1008D0004091760B5091770B0F947A1A6BA37CA3FF
:1008E0008DA39EA36D8B7E8B8F8B988F69A57AA528
:1008F0008BA59CA50F941B1A2091780B3091790B36
:1009000040917A0B50917B0B0F947A1A4B015C014A
:10091000698F7A8F8B8F9C8F20917C0B30917D0B10
:1009200040917E0B50917F0BC701B6010F947A1A4C
:100930006B017C016D8F7E8F8F8F98A3B6E04B1675
:100940005104610471049CF52DA53EA54FA558A93D
:10095000263031054105510554F527968CAD9DADE6
:10096000AEADBFAD27970697A105B10504F520E010
:1009700030E0A901C701B6010F945E2387FF04C0D0
:10098000F7FAF094F7F8F09488E5AFA1B8A58A9F3C
:1009900080018B9F100D11240856144F20E030E089
:1009A000A901C701B6010F94FE20F80154C02D968D
:1009B000AEADBFAD2D97CD90DD90ED90FC9020E0D9
:1009C00030E0A901C701B6010F94141A882379F009
:1009D00088E52FA138A5829FF001839FF00D112497
:1009E000E856F44FC586D686E786F08A38C0219649
:1009F0002CAD3DAD4EAD5FAD2197CA01B9010F944D
:100A00007A1A6B017C012BA13CA14DA15EA1CA0108
:100A1000B9010F947A1A9B01AC01C701B6010F947A
:100A2000FE206B017C01A5019401C501B4010F9466
:100A30007A1A9B01AC01C701B6010F94FE200F94F6
:100A4000AC2328E54FA158A5249FF001259FF00D68
:100A50001124E856F44F658776878787908B88E561
:100A6000AFA1B8A58A9FF0018B9FF00D1124E85625
:100A7000F44F29A93AA94BA95CA921A332A343A306
:100A800054A327968CAD9DADAEADBFAD27972DA5D8
:100A90003EA54FA558A982179307A407B50710F4E0
:100AA000DA01C90184159505A605B70510F4D3012F
:100AB000C20129A93AA94BA95CA982179307A407E7
:100AC000B50710F4DA01C90128E54FA158A5249F04
:100AD000F001259FF00D1124E856F44F85A396A34D
:100AE000A7A3B0A70697A105B10510F40C946E8FCB
:100AF000DF01AA5ABF4F80916E0B8C93E95AFF4FCA
:100B000080916F0B808345284628472809F05F981D
:100B100088E5AFA1B8A58A9FF0018B9FF00D112445
:100B2000E856F44F818D928DA38DB48D892B8A2B3D
:100B30008B2B09F08A9888E52FA138A5829FF001B8
:100B4000839FF00D1124E856F44F858D968DA78D67
:100B5000B0A1892B8A2B8B2B29F080910801817001
:100B60008093060189A99AA9ABA9BCA9892B8A2BD4
:100B70008B2B11F40C94C28E80917311882319F081
:100B8000815080937311129880E280937311E090EA
:100B90005B11F0905C1100915D1110915E11970155
:100BA000A801632D7DA989AD922D0F94141A87FF9A
:100BB00004C03E2CFDAA09AF212E88E5AFA1B8A53F
:100BC0008A9FF0018B9FF00D1124E856F44F258584
:100BD00036854785508927962CAF3DAF4EAF5FAF26
:100BE000279760E070E080E89FE30F94F8216BA303
:100BF0007CA38DA39EA3232D3DA949AD522D0F9417
:100C00007A1A6B017C0180915F1490915D14891BAD
:100C10008F7089AFA701960160E074E284E799E4E0
:100C20000F94F8210F946B234B015C0189AD825026
:100C30008630B0F580912B1190912C11A0912D113F
:100C4000B0912E1188169906AA06BB0648F5881998
:100C50009909AA09BB09BC01CD01660F771F881F3E
:100C6000991F49AD042F10E020E030E0A901980160
:100C70000F946A20CA01B9010F94191A0F946B23BB
:100C8000680D791D8A1D9B1D0F94191A9B01AC01DB
:100C900060E074E284E799E40F94F8216B017C0131
:100CA000A701960127966CAD7DAD8EAD9FAD2797C0
:100CB0000F947A1A9B01AC010F947A1A6DAB7EAB3C
:100CC0008FAB98AF88E5AFA1B8A58A9F80018B9FB5
:100CD000100D11240856144F2DA93EA94FA958AD47
:100CE000D80111962D933D934D935C93149795964F
:100CF0004D905D906D907C909897C301B2010F94D8
:100D0000191A69A77AA78BA79CA79B01AC01C701F9
:100D1000B6010F947A1A0F94DC210F947122219658
:100D20006CAF7DAF8EAF9FAF2197F801EA5BFF4FAD
:100D30006083718382839383FE017196FEA7EDA782
:100D40002FE331E161963FAF2EAF6197AE014F5D6A
:100D50005F4F5AA349A300E010E050E8252E6FE34F
:100D6000362EADA5BEA52D913D914D915D91BEA7AD
:100D7000ADA7C701B6010F947A1A4B015C0120E0C0
:100D800030E0A9010F945E2387FF04C0B7FAB09446
:100D9000B7F8B0946196AEADBFAD61972D913D911E
:100DA0004D915D916196BFAFAEAF61972F962CAF1D
:100DB0003DAF4EAF5FAF2F97A50194012F966CAD5D
:100DC0007DAD8EAD9FAD2F970F94141A87FF14C081
:100DD000A50194012F966CAD7DAD8EAD9FAD2F9783
:100DE0000F94F8215B014C019801A1010F94141A92
:100DF00087FF02C085011401EDA5FEA529A13AA136
:100E0000E217F30709F0ADCF20E030E040E85FE300
:100E1000B801C1010F94141A87FF36C028E54FA10D
:100E200058A5249FC001259F900D1124DC01A856D0
:100E3000B44F7D016D01B6E4CB0ED11C21966CAD93
:100E40007DAD8EAD9FAD21970F94191A9801A10128
:100E50000F947A1A0F947122F60160837183828352
:100E600093839801A101B801C1010F947A1A2DA9A9
:100E70003EA94FA958AD0F947A1AD70111966D93D8
:100E80007D938D939C93149729A53AA54BA55CA5BA
:100E90006BA17CA18DA19EA10F947A1A21966CAFB3
:100EA0007DAF8EAF9FAF219788E52FA138A5829F98
:100EB000F001839FF00D1124E856F44F8588968841
:100EC000A788B08C81149104A104B10419F5818D17
:100ED000928DA38DB48D892B8A2B8B2BD9F4858D84
:100EE000968DA78DB0A1892B8A2B8B2B99F42091FD
:100EF0005311309154114091551150915611219632
:100F00006CAD7DAD8EAD9FAD21970F947A1A0F9485
:100F1000DC21FBC189A99AA9ABA9BCA9892B8A2B81
:100F20008B2B49F020914F1130915011409151116C
:100F30005091521108C02091571130915811409191
:100F4000591150915A1121966CAD7DAD8EAD9FAD6A
:100F500021970F947A1A0F94DC210F9471226B0160
:100F60007C0180916A0B90916B0BA0916C0BB091FE
:100F70006D0B2396EEADFFAD2397218D328D438D02
:100F8000548D29AB3AAB4BAB5CAB258D368D478D81
:100F900050A12DA73EA74FA758AB21A132A143A135
:100FA00054A12DAB3EAB4FAB58AF84159505A605AC
:100FB000B70508F4AFC081149104A104B10471F124
:100FC00060915A0B70915B0B80915C0B90915D0B63
:100FD0006C157D058E059F0508F5A30192010F9400
:100FE0005A2069A77AA78BA79CA7A5019401C701DE
:100FF000B6010F945A2029A53AA54BA55CA5261742
:1010000037074807590750F469A57AA58BA59CA511
:10101000A50194010F946A2069017A0129A93AA9CE
:101020004BA95CA9232B242B252B51F160915E0B3E
:1010300070915F0B8091600B9091610B6C157D0539
:101040008E059F05E8F4A30192010F945A204B01ED
:101050005C0129A93AA94BA95CA9C701B6010F9463
:101060005A2086169706A806B90650F4C501B401A1
:1010700029A93AA94BA95CA90F946A2069017A01B0
:101080008DA59EA5AFA5B8A9892B8A2B8B2B51F1D5
:101090006091620B7091630B8091640B9091650B72
:1010A0006C157D058E059F05E8F4A30192010F9450
:1010B0005A204B015C012DA53EA54FA558A9C7019B
:1010C000B6010F945A2086169706A806B90650F462
:1010D000C501B4012DA53EA54FA558A90F946A20BE
:1010E00069017A012DA93EA94FA958AD232B242BC4
:1010F000252B09F40EC16091660B7091670B8091EE
:10110000680B9091690B6C157D058E059F0508F4A1
:1011100043C6FFC081149104A104B104B9F16091E8
:101120005A0B70915B0B80915C0B90915D0B6C1571
:101130007D058E059F0550F50F94191A29A53AA52E
:101140004BA55CA50F947A1A2B013C01C501B40193
:101150000F94191A4B015C01C701B6010F94191ABB
:10116000A50194010F947A1A9B01AC01C301B2014D
:101170000F94141A87FF0AC0A5019401C301B2019C
:101180000F94F8210F9471226B017C0189A99AA90F
:10119000ABA9BCA9892B8A2B8B2BC9F160915E0B63
:1011A00070915F0B8091600B9091610B6C157D05C8
:1011B0008E059F0560F50F94191A29A53AA54BA530
:1011C0005CA50F947A1A4B015C0169A97AA98BA9D5
:1011D0009CA90F94191A2B013C01C701B6010F9469
:1011E000191AA30192010F947A1A9B01AC01C5014F
:1011F000B4010F94141A87FF0AC0A3019201C5011C
:10120000B4010F94F8210F9471226B017C012DA57C
:101210003EA54FA558A9232B242B252BC9F160915E
:10122000620B7091630B8091640B9091650B6C1550
:101230007D058E059F0560F50F94191A29A53AA51D
:101240004BA55CA50F947A1A4B015C016DA57EA598
:101250008FA598A90F94191A2B013C01C701B6015B
:101260000F94191AA30192010F947A1A9B01AC01F1
:10127000C501B4010F94141A87FF0AC0A30192019B
:10128000C501B4010F94F8210F9471226B017C0108
:101290008DA99EA9AFA9B8AD892B8A2B8B2BC9F13B
:1012A0006091660B7091670B8091680B9091690B50
:1012B0006C157D058E059F0560F50F94191A29A5FB
:1012C0003AA54BA55CA50F947A1A4B015C016DA958
:1012D0007EA98FA998AD0F94191A2B013C01C70163
:1012E000B6010F94191AA30192010F947A1A9B0167
:1012F000AC01C501B4010F94141A87FF0AC0A30101
:101300009201C501B4010F94F8210F9471226B0171
:101310007C0188E5AFA1B8A58A9F80018B9F100D45
:1013200011240856144FF801EE5AFF4FC082D182A3
:10133000E282F382C701B6010F94191A21962CADEF
:101340003DAD4EAD5FAD21970F94F8216DA77EA7FF
:101350008FA798ABF801618B728B838B948B298953
:101360003A894B895C896BA17CA18DA19EA10F94C8
:101370007A1A21966CAF7DAF8EAF9FAF21972D89E2
:101380003E894F89588D6BA17CA18DA19EA10F94A0
:101390007A1A2F966CAF7DAF8EAF9FAF2F97298DA6
:1013A0003A8D4B8D5C8D6BA17CA18DA19EA10F947C
:1013B0007A1A63966CAF7DAF8EAF9FAF63972D8D1A
:1013C0003E8D4F8D58A16BA17CA18DA19EA10F9444
:1013D0007A1A67966CAF7DAF8EAF9FAF6797F9AD06
:1013E000FF2309F476C2209161142BA3309162147B
:1013F00039A730906314209064142DEB37E346E84E
:1014000055E36BA179A5832D922D0F94141A87FDB6
:1014100060C28090631190906411A0906511B090AB
:101420006611C0906711D0906811E0906911F0903A
:101430006A1180916B1190916C11A0916D11B09116
:101440006E118DAB9EABAFABB8AF20916F113091E9
:101450007011409171115091721129AF3AAF4BAF99
:101460005CAFC501B401905821962CAD3DAD4EAD99
:101470005FAD21970F947A1A2B013C01C701B60189
:1014800090582F962CAD3DAD4EAD5FAD2F970F947C
:101490007A1A9B01AC01C301B2010F94FE202B010B
:1014A0003C016DA97EA98FA998AD905863962CAD8B
:1014B0003DAD4EAD5FAD63970F947A1A9B01AC01C1
:1014C000C301B2010F94FE202B013C0169AD7AAD3E
:1014D0008BAD9CAD905867962CAD3DAD4EAD5FADDC
:1014E00067970F947A1A9B01AC01C301B2010F9464
:1014F000FE2069AB7AAB8BAB9CAB2FEE3FEF4FE797
:101500005FE30F945E2318160CF4B2C12FEE3FEF89
:101510004FE75FEB69A97AA98BA99CA90F94141ACC
:1015200087FF08C08FEE9FEFAFE7BFEB89AB9AABA9
:10153000ABABBCABA501940121966CAD7DAD8EAD7E
:101540009FAD21970F94FD202B013C0169837A8385
:101550008B839C83A70196012F966CAD7DAD8EADDC
:101560009FAD2F970F94FD206B966CAF7DAF8EAF24
:101570009FAF6B976D837E838F8398872DA93EA93C
:101580004FA958AD63966CAD7DAD8EAD9FAD6397A1
:101590000F94FD206F966CAF7DAF8EAF9FAF6F97AE
:1015A00069877A878B879C8729AD3AAD4BAD5CAD57
:1015B00067966CAD7DAD8EAD9FAD67970F94FD20A6
:1015C00069AF7AAF8BAF9CAF6D877E878F87988B23
:1015D000DE011196BEABADABFE017196FAA3E9A395
:1015E0008D01C12CD12C7601D8018D909D90AD90AC
:1015F000BD908D0120E030E0A901C501B4010F9438
:10160000141A882371F0A5019401C501B4010F9447
:101610007A1A9B01AC01C701B6010F94FE206B0141
:101620007C01E9A1FAA1E017F107F1F6C701B601C3
:101630000F94AC239B01AC0160E070E080E89FE375
:101640000F94F8216B017C019B01AC01C301B20135
:101650000F947A1A69837A838B839C83A7019601FE
:101660006B966CAD7DAD8EAD9FAD6B970F947A1A76
:101670006D837E838F839887A70196016F966CADEB
:101680007DAD8EAD9FAD6F970F947A1A69877A877B
:101690008B879C87A701960169AD7AAD8BAD9CAD18
:1016A0000F947A1A6D877E878F87988B0BE111E1F3
:1016B0004DA46EA45FA478A8ADA9BEA9CD90DD907D
:1016C000ED90FD90BEABADAB20E030E0A901C701CD
:1016D000B6010F94141A882331F1F80160817181E9
:1016E000828193810F94191AA70196010F94F82112
:1016F0006B017C0120E030E0A9010F945E2387FF9D
:1017000004C0F7FAF094F7F8F094242D362D452D07
:10171000572DC701B6010F94141A87FF04C04C2C33
:101720006D2C5E2C7F2C0C5F1F4F29A13AA14DA977
:101730005EA92417350709F0BFCF29A93AA94BA9FB
:101740005CA960E070E080E89FE30F94FD2020E05A
:1017500030E040E05FE30F947A1A0F94AC236B0102
:101760007C012091560B3091570B4091580B5091B2
:10177000590B642D762D852D972D0F947A1AA7017C
:1017800096010F947A1A4B015C01A701960160E063
:1017900070E080E89FE30F94FD209B01AC01C50140
:1017A000B4010F94F8217B018C0120E030E040E887
:1017B0005FE327966CAD7DAD8EAD9FAD27970F94FF
:1017C000141A87FF5BC029A93AA94BA95CA9CA01D1
:1017D000B9010F947A1A23EC38EB42E35FEB0F94D4
:1017E0007A1A23EF36E64FE55FE30F94FD2029A92F
:1017F0003AA94BA95CA90F947A1A2BED3FE049EC6A
:101800005FE30F94FE202CEE31E548E35EE30F9496
:10181000FD204B015C0124EE3BEC46E150E40F94CB
:101820005E2318165CF5A50194016BED7FE089E459
:1018300090E40F94FD209B01AC0127966CAD7DAD2B
:101840008EAD9FAD27970F94F821242D362D452D71
:10185000572D0F947A1A5B016C019B01AC01B70103
:10186000C8010F945E2318164CF47501860106C05A
:101870003BE0E32E47EDF42E03E21BE388E5AFA146
:10188000B8A58A9FF0018B9FF00D1124E856F44F04
:10189000A180B280C380D4809501A6016BA179A5F7
:1018A000832D922D0F945E23181624F4ABA2B9A6B3
:1018B0003C2C2D2C9701A8016BA179A5832D922D8D
:1018C0000F945E2318164CF4EBA2F9A6302E212EAD
:1018D00004C01BA219A6312C212C21962CAD3DADA4
:1018E0004EAD5FAD21972093631130936411409307
:1018F0006511509366112F968CAD9DADAEADBFAD09
:101900002F978093671190936811A0936911B093FA
:101910006A1163962CAD3DAD4EAD5FAD63972093DC
:101920006B1130936C1140936D1150936E1167964B
:101930008CAD9DADAEADBFAD679780936F119093A9
:101940007011A0937111B093721188E5AFA1B8A581
:101950008A9F80018B9F100D11240856144F8BA174
:1019600099A5A32DB22DF80181879287A387B4870B
:101970006DA57EA58FA598A990589B01AC010F94E9
:10198000FE202396AEADBFAD23971D962D913D91C0
:101990004D915C9150970F947A1A9B01AC016BE0CA
:1019A00077ED83E29BE30F94FD202BE0C22E27ED21
:1019B000D22E23E2E22E2BE3F22EF801C582D6824C
:1019C000E782F086B080C180D280E380F480A701F6
:1019D00096010F945E2387FD02C083E001C081E081
:1019E000B82A88E52FA138A5829FF001839FF00DCA
:1019F0001124E856F44FB082C0926114D092621460
:101A0000E0926314F0926414A3968CAD9DADAEADDC
:101A1000BFADA3978093751490937614A093771419
:101A2000B0937814A7962CAD3DAD4EAD5FADA797A2
:101A30002093791430937A1440937B1450937C1440
:101A4000AB968CAD9DADAEADBFADAB9780937D1425
:101A500090937E14A0937F14B09380142B962CAD9A
:101A60003DAD4EAD5FAD2B97209381143093821422
:101A7000409383145093841490915F148091601468
:101A8000981303C084E680935C14AC968FADAC973A
:101A90008F5F8F7080935F1480915F1490915E14BC
:101AA00081508F70891709F491C0F0905F148FEF07
:101AB0008F0D8F708FA3B0905E1480915F14B81655
:101AC00009F45BC0C12CD12C3FA13B1509F455C0D2
:101AD000632E712C48E5469D8001479D100D112411
:101AE0000856144FD8018C9183FD2EC00DA728965F
:101AF0001FAF28971996BC91BBA3F801F285F9A7EF
:101B0000D8011B96BC912296BFAF2297F801F485AD
:101B1000F9ABD80115962D903D904D905C9018979B
:101B2000A20191016BA179A522968FAD22979F2FDB
:101B30000F94141A81114FC1C114D10449F0F60158
:101B4000808180FD48C104C0CDA62896DFAE2897CD
:101B50008FA181508F708FA380915E148B1105C06F
:101B6000CDA42896DFAC2897AFCFFFA1FB1529F0B5
:101B700081E08B0D8F70B82EEFCF20915E142FA3D4
:101B8000C12CD12C80915F143FA18317F9F0832ED3
:101B9000912C48E5489D8001499D100D112408565F
:101BA000144FD8018C9183FD0AC05801C114D1048F
:101BB00039F0C6010F94B207811102C096C15601D7
:101BC0008FA18F5F8F708FA36501DCCFD0906014E1
:101BD00080905F1428E5D81469F08FEF880D8F701E
:101BE000289FF0011124E856F44F908193FF02C022
:101BF000882EF1CF212C312C412C512C1FA21BA25D
:101C0000712C612C00E010E0E12CF12C8D1409F412
